:020000040000FA
:0600000013EFA9F012004D
:020006001200E6
:06000800ACEF93F01200C2
:02000E000202EC
:0100100006E9
:020011000100EC
:020013000000EB
:0600180011EF3DF01200A3
:02001E000B00D5
:100020001A540100000B00004000000002540100BF
:10003000E708000018000000FD530100F709000068
:1000400005000000D1530100C80600002C0000008C
:100050008C5301005D0A0000450000002F53010091
:10006000000A00005D000000C65201008E09000079
:100070006900000013000000F30700000200000008
:100080009B520100C80700002B00000084520100B1
:10009000E20A00001700000011000000FE0400004A
:0400A000020000005A
:0C00A4006DEC2AF0C8EC25F001340FE2EE
:1000B00000501008270E01540AE2100EF36EFD0ED8
:1000C000F3CFDBFF270EF36EFE0EF3CFDBFF54EC16
:1000D0002BF003E3F36AF46A4ED0DE6ADD6AC8EC03
:1000E00025F0013430E20050B808240E01542BE210
:1000F000B80E035D240E04590DE2C8EC25F0B80ECD
:10010000005E240E015A026A036A01AE05D002683D
:10011000036802D024EC26F0280E61EC29F02C0EA6
:100120000026010EFBEC2BF0580E2B6E020E12EC8B
:1001300025F0B80EF36EFD0EF3CFDBFF240EF36E49
:10014000FE0EF3CFDBFF54EC2BF00FE224EC26F095
:10015000B40E61EC29F05C0E0026120EFBEC2BF0C5
:10016000B80E2B6E240E12EC25F070EC24F000C0BB
:10017000F3FF01C0F4FF020EE15C02E2E16AE55226
:10018000E16EEFEF22F0EAEC22F00E0EE126CBEC6E
:1001900024F03EEC26F0040E02C0DBFF050E03C087
:1001A000DBFFE5EC24F0FEEC26F0080E02C0DBFFDE
:1001B000090E84EC24F00A0E00C0DBFF0B0E01C018
:1001C000DBFF0C0E02C0DBFF0D0E03C0DBFFCDC951
:1001D000E6FFCEC9E6FFCFC9E6FFD0C9E6FF060EAF
:1001E000E66EE50EE66E000EF2EC2DF024EC75F0F6
:1001F000DEEC2CF04AEC27F0FE0EE66EE40EE66E26
:10020000000E5CEC2BF0EFEC25F080EC28F05CECC1
:100210002BF079EC26F052EC2CF0D9C9E6FFDAC9C4
:10022000E6FF52EC2CF009019F51D8EC2DF00901AA
:10023000E051D8EC2DF0E3C900F0016A00BE01687E
:100240004CEC23F080EC28F0B5EC22F00901E951E8
:10025000D8EC2DF005EC27F001AE02D0026803685F
:10026000040E5EEC25F0FDE100EC2CF080EC28F0B3
:1002700055EC2CF016EC75F0046E090ECBEC2AF060
:1002800075EC23F0080EDBCF02F0090EDBCF03F094
:10029000A9EC21F0E2EC2CF0EBEC27F0E4EC27F0F9
:1002A000A9EC21F0E2EC2CF051EC23F0C4EC2AF0A4
:1002B00007EC24F0E2EC2CF06A0EE66E090EE66E16
:1002C00045EC2DF0006E0E0EE15C02E2E16AE552B3
:1002D000E16E0050EFEF22F004EC2CF0010EDB6A2F
:1002E000020EDB6ADF6ADF50006E016AFD0EDBCFB3
:1002F00002F0FE0EDBCF03F003500118E8AE02D08F
:10030000013402D003EC26F001E28ED045EC26F059
:10031000BFEC27F004BE056842EC2AF024C003F0CD
:1003200025C004F026C005F0CAEC2CF00800F550FA
:1003300033E1A00E066E3C0E076E010E086E010E34
:10034000DBCF09F0020EDBCF0AF00B6A0ABE0B68A6
:10035000E6EC2CF0ABEC2BF0D4EC84F024C009F0EC
:1003600025C00AF026C00BF006502424F36E075077
:100370002520F46E08502620A7EC29F0A4EC2BF0E1
:100380000BE145EC26F0BFEC27F004BE056841EC1C
:1003900023F0F550DF6E41D0DF50006E016AFD0E94
:1003A000DB5000183AE1FE0EDB50011836E17F0EFB
:1003B0000601C85D23E1010EDBCFE6FF020EDBCFB5
:1003C000E6FFEB0EE66EE40EE66E000EF2EC2DF0AC
:1003D0007FEC2CF0F2EC27F0E90EE66EE40EE66E10
:1003E000000EE66E030EDBCFE6FF040EDBCFE6FF6A
:1003F00025EC22F0F2EC27F08DEC29F0A390A392EB
:10040000010EDBCFE2FA020EDBCFE3FA15D85CD99E
:100410000A01E269E369A382A380010EDB2A020ECE
:1004200001E261D7DB2A5FD7050EE15C02E2E16AF7
:10043000E552E16EEFEF22F004EC2CF00A01800EA1
:10044000E3154DE1A3EC26F008BE09687CEC23F02F
:100450000EBE0F68BBEC23F0030E00C0DBFF040EE2
:1004600001C0DBFFD950030FBDEC2CF0550EEE1888
:1004700009E1010EED1806E1DF6A5FEC2BF004AE36
:1004800004D002D0000E16D1056841EC23F0F5CF60
:1004900040FB030EDB6A040EDB6A030EDBCF00F0C9
:1004A000040EDBCF01F0080EEDEC25F030E2AFECEE
:1004B00026F007BE086876EC25F0030EDBCF09F0C6
:1004C000040E20EC25F0030EDBCFE9FF040E36EC22
:1004D00027F0030EDB2A040EE0E3DB2ADED7010E51
:1004E0006014DF6E0F0E65140B01406F66CF41FB89
:1004F00067CF42FB68CF43FB69CF44FB6ACF45FB24
:100500006BCF46FB6CCF47FB6DCF48FB609EDF5047
:1005100001E0CFD0540E0B01445D01E0CAD045CBC1
:1005200003F0026A465141EC25F02CE20CEC27F076
:10053000026A0234000E021807E6D880400E00540A
:100540009C0E0154000E02541DE3010EDBCF03F993
:10055000020EDBCF04F90901D89004330333D8909D
:10056000043303330351095D04510A5904E203C9FA
:1005700009F904C90AF90551035D0651045902E25B
:1005800053EC27F00F0E0B014215036E026A435124
:1005900041EC25F001E38DD00CEC27F0000E005C5F
:1005A0000F0E015801E385D0010EDBCF15F9020EC5
:1005B000DBCF16F90901D00ED8801557070E165754
:1005C0003E51135D3F51145907E33E51135D006ED8
:1005D00014513F55016E21D0F9EC27F0086A096AE1
:1005E000010E0A6E0B6A3EC90CF03FC90DF00E6A8F
:1005F0000F6A0C50085C046E0D500958056E0E50C1
:100600000A58066E0F500B58076E0450002605500E
:1006100001220650022207500322B2EC2BF013C92C
:100620003EF914C93FF90CEC27F0026A036AB9ECF1
:1006300025F0AEEC24F0163521E215510008000E2D
:1006400016551CE205EC27F001AE02D002680368E3
:10065000B9EC25F0040EC3EC29F0AEEC24F005EC67
:1006600027F001AE02D002680368005062270150F3
:10067000632302506423035065231BD0F3EC26F060
:1006800001AE02D002680368B9EC25F0080EC3EC95
:1006900029F0AEEC24F0F3EC26F001AE02D00268B3
:1006A00003680050662701506723025068230350F7
:1006B0006923010E006E050EE15C02E2E16AE5527B
:1006C000E16E0050EFEF22F0EAEC22F00E0EE12690
:1006D0000A01800EE31570E1A3EC26F008BE09685C
:1006E0007CEC23F00EBE0F68BBEC23F043EC24F04F
:1006F000D7EC22F0900E0016050E0116900E001891
:1007000005E1050E011802E1020E1BD0D7EC22F024
:10071000900E0016060E0116900E001805E1060E4A
:10072000011802E1030E0DD0D7EC22F0500E001696
:10073000050E0116500E001816E1050E011813E102
:10074000040EDF6E0F0EE76E040EDBCF00F0050E19
:10075000E7500016016A010E00C0DBFF5FEC2BF0D2
:1007600004AE04D002D0000EF5D2056841EC23F0AF
:10077000F5CF40FB040EDB6A050EDB6AD7EC22F0F6
:10078000080EEDEC25F041E2AFEC26F007BE08685C
:1007900076EC25F0040EDBCF09F0050E20EC25F0F9
:1007A000040EDBCFE9FF050E36EC27F0040EDB2A42
:1007B000050EE4E3DB2AE2D7070E0F015015DF6ECA
:1007C000E00E5215E00BE838E840006E010E5115BE
:1007D000080DF3500024E76E010EE7CFDBFF0F0E8C
:1007E00055150B01406F56CF41FB57CF42FB58CFF9
:1007F00043FB59CF44FB5ACF45FB5BCF46FB5CCF55
:1008000047FB5DCF48FB0F01509F020EDF5C01E00C
:1008100096D0010EDB500E0A01E177D0070A23E0E3
:100820000E0A01E096D20B0141AB08D0E60E090199
:100830008E6F8F6B09010A0E906F05D009018E6BC8
:100840008F6B0901906B42CB17F90B0148510008DF
:1008500001E37FD2F00E485D01E37BD2280E485DB4
:100860000901C06F76D2600E090117150BE1FF0E6A
:100870000B01465D07E04651000804E246510901BC
:100880000B6F0C6B47CB03F0026A0B014851CFECA6
:100890002AF03EEC26F0D950020FBDEC2CF0FF0EF2
:1008A000EE1802E1FF0EED1801E153D2020EDBCF8C
:1008B00028F0030EDBCF29F009010D51285C006EF2
:1008C0000E512958016EFEEC26F075EC23F0D890FD
:1008D000015004E60A0E005C000E015802E3010E0E
:1008E0000AD075EC23F0013408E30050F608FF0E3F
:1008F000015403E3020E3D6F01D03D6B020EDBCFCE
:100900000DF9030EDBCF0EF924D241CB01F0006AC2
:100910000B01425109010024136F000E0120146FD6
:100920000B014651280808E2F00E465D05E2280E4C
:10093000465D0901C16F0DD20901C16B0AD2030ED8
:10094000DF5C35E1010EDB500F0A01E002D2090144
:10095000B55101E1FED10F0E0B014415300F090115
:10096000AE6F0B0144390F0B300F0901AF6F0F0E43
:100970000B014315300F0901B06F0B0143390F0B09
:10098000300F0901B16F0F0E0B014215300F090135
:10099000B26F0B0142390F0B300F0901B36F0F0E0D
:1009A0000B014115300F0901B46FB56BD2D1040EA4
:1009B000DF5C01E078D1090EFEC0DBFF010EDB50E9
:1009C0000F0A01E125D1010A01E1E5D0090A01E19F
:1009D0009BD0030A6CE0020A01E0BBD1FF0E0B01C1
:1009E000415D01E1B6D17CEC28F001E1B2D147ECE8
:1009F00028F0A7EC25F0FDE10B0142390F0B0001B7
:100A000000108E6F01C08FF013EC27F00001001072
:100A1000966F01C097F07DEC27F0A7EC25F0FDE183
:100A20000B0145390F0B000100109E6F01C09FF0B4
:100A30001AEC27F000010010A66F01C0A7F00B010F
:100A40004751006E016A040EA7EC25F0FDE10B0191
:100A500048390F0B00010010AE6F01C0AFF0090E56
:100A6000DB50FC0B3C0803E13F0EFE6F72D1090E18
:100A7000DB50FC0B01E16DD1090EDB50030B010FC4
:100A8000E76E080EE7CFDBFFDB50030803E1090E3A
:100A9000DB6A06D1080EDBCFE6FF090EDB50FC0B4C
:100AA000E552E710E76E090EE7CFDBFFF9D0FF0E46
:100AB0000B01415D01E14DD17CEC28F001E149D110
:100AC000080EDB6A070EF36E080EDBCFF4FFF3505F
:100AD000F45C13E2080EDB50EA6A410FE96E0B0E7C
:100AE000EA22EF50E66E080EDB50DEEC22F0E55213
:100AF000E750EF6E080EDB2AE5D7090EDB84CFEC5A
:100B000026F001E283D07DD0FF0E0B01415D01E1B3
:100B100020D17CEC28F001E11CD147EC28F0A7ECB7
:100B200025F0FDE10B0142390F0B00010010B66FFB
:100B300001C0B7F013EC27F000010010BE6F01C038
:100B4000BFF07DEC27F0A7EC25F0FDE10B01453966
:100B50000F0B00010010C66F01C0C7F01AEC27F0A0
:100B600000010010CE6F01C0CFF00B014751006EA5
:100B7000016A040EA7EC25F0FDE10B0148390F0BCB
:100B800000010010D66F01C0D7F0090EDB86CFEC54
:100B900026F03CE336D0FF0E0B01415D01E1D9D0D8
:100BA0007CEC28F001E1D5D047EC28F0A7EC25F04B
:100BB000FDE10B0142390F0B00010010DE6F01C097
:100BC000DFF013EC27F000010010E66F01C0E7F042
:100BD0007DEC27F0A7EC25F0FDE10B0145390F0B6B
:100BE00000010010EE6F01C0EFF01AEC27F00001D9
:100BF0000010F66F01C0F7F0090EDB88CFEC26F08D
:100C000005E33F0EF36E090EF3CFDBFF090E48D06C
:100C1000FF0E0B01465D01E19CD07CEC28F001E168
:100C200098D04651026E036A040ED89002360336FD
:100C3000E804FBE10B0147390F0B00010210006EC5
:100C40000A0E00C0DBFF0B0E03C0DBFF0F0E0B0113
:100C50004715036E026A485100010210006E0C0E27
:100C600000C0DBFF0D0E03C0DBFF00EC28F00A0E16
:100C7000DB5000240001606F0B0EDB5000010120EF
:100C80000001616FD89061336033090EDB8ACFECCD
:100C900026F005E33F0EF36E090EF3CFDBFF090EDE
:100CA000DBCFFEF056D0050EDF5C53E1010EDB50CA
:100CB000070A4FE146CB00F0016A026A036A040E9C
:100CC00007EC28F0FDE145CB04F0056A066A076AE7
:100CD000040E1F0B03E0B1EC24F0FDE10450001200
:100CE00005500112065002120750031244CB08F0BF
:100CF000096A0A6A0B6A0C0E1F0B07E0D8900836C7
:100D000009360A360B36E806F9E108500012095098
:100D100001120A5002120B50031243CB0CF00D6A61
:100D20000E6A0F6A140E1F0B07E0D8900C360D36B2
:100D30000E360F36E806F9E100500C1009010F6F6E
:100D400001500D10106F02500E10116F03500F1054
:100D5000126F010E006E0E0EE15C02E2E16AE552D6
:100D6000E16E0050EFEF22F004EC2CF009EC2CF0D7
:100D70007F0E0601C85D04E0200EC85D01E0B0D022
:100D8000030EE66EAFEC27F06FEC2CF0E50EE66E8E
:100D9000E40EE66E000ECFEC25F005E0010EF36EDA
:100DA000020EF3CFDBFFE20EE66EE40EE66E000EFF
:100DB000CFEC25F005E0010EF36E030EF3CFDBFF61
:100DC000090118A11ED0030EDB500CE00A015D5191
:100DD00009E00A015E5106E19DEC2BF0CD0EB9EC65
:100DE0002BF01891020EDB500CE03EEC27F0CEEC1D
:100DF0001CF001EC2EF0000902E01DEC59F0090195
:100E00001891090118A322D0030EDB5010E00A014B
:100E10005D510DE00A015E510AE19DEC2BF0CF0E11
:100E200075EC26F089EC0EF083EC27F01893020E97
:100E3000DB500CE03EEC27F05EEC0EF001EC2EF007
:100E4000000902E01DEC59F009011893090118A9E5
:100E50000CD00A015D0509E10A015E5106E19DEC35
:100E60002BF0CE0EB9EC2BF01899090118A524D05F
:100E70000A015D0521E10A015E511EE1020EF36ED9
:100E8000040EF3CFDBFFD00EE66EE66A040EDBCF76
:100E9000E6FF86EC27F04CEC28F0DBCFE6FFC3EC56
:100EA00000F0E5524CEC28F0DB50020802E02AEC9E
:100EB0002EF0090118951889090118A711D00A0107
:100EC0005D050EE10A015E510BE1020EE66EC3EC18
:100ED00000F0E552020802E02AEC2EF00901189712
:100EE000050EE15C02E2E16AE552E16EEFEF22F00D
:100EF0003BDF010CEAEC22F0070EE1260501EF5181
:100F0000DE6EDD6AF051E66ED950020F4FEC25F02F
:100F1000F151E66ED950040F4FEC25F04B0E07014E
:100F2000CB5D38E151EC23F0013418E261EC26F09E
:100F300015E221EC27F0033402E2A0EC27F003E3F2
:100F4000006A016A09D051EC23F0ADEC29F066EC9F
:100F500026F0FDE16BEC26F03EEC26F0D7EC22F01B
:100F6000013418E261EC26F015E2C4EC2AF00334F7
:100F700002E2A0EC27F003E3006A016A09D0D7EC93
:100F800022F0ADEC29F066EC26F0FDE16BEC26F0EA
:100F900043EC24F00901A52B000EA623A723A823C8
:100FA000320E0901016A0325006E04510122640E0C
:100FB000E9EC29F028C0A0F95CEC27F067EC2BF0F5
:100FC000D880000E2654000E2754000E2854000E20
:100FD000295406E30901CD6BCE6BCF6BD06B2AD0C1
:100FE0000FC900F010C901F011C902F012C903F0D5
:100FF000ADEC2CF05CEC27F0E3EC2DF0ADEC2CF03C
:10100000C6EC22F0050E005E000E015A025A035A89
:10101000040E07EC28F0FDE100C0CDF901C0CEF9C7
:1010200002C0CFF903C0D0F90901CD2B000ECE23A9
:10103000CF23D023B3EC27F027E1320E0901036A56
:101040000D25026E0E510322640E2D6E2E6A02C013
:1010500028F003C029F0CEECA8F028C002F029C087
:1010600003F0000ED8802854000E295403E3006AD0
:10107000016A0CD0D4EC2CF0ADEC29F066EC26F033
:10108000FDE16BEC26F002D0D4EC2CF000C09FF90F
:101090000901000ED8808E55000E8F5505E209011A
:1010A000998709019D8904D00901999709019D99A2
:1010B000600E09011715200804E109019985998935
:1010C00002D009019999090117A910D0090199BF06
:1010D0002ED0998F0901A96BAA6BAB6BAC6B010E7B
:1010E000B8EC24F001EC15F087D921D0090199AFB3
:1010F0001ED0999FA5C9A9F9A6C9AAF9A7C9ABF994
:10110000A8C9ACF90901A907000EAA5BAB5BAC5BEF
:10111000010EB8EC24F0D880E40E09011D55570EDD
:101120001E55000E1F55000E205501E2188390EC4D
:1011300015F06ED9090199A9E0D0640E006E016A1C
:101140000EEC2CF02D6E01C02EF0CEECA8F0060EA9
:1011500028C0DBFF0901000ED8800755000E085596
:101160003FE2000ED8800355000E045539E2000E10
:10117000D8800555000E065533E2A5EC22F00EECA2
:101180002CF08EEC82F06BEC29F0A8EC83F044ECB0
:1011900085F028C00BF929C00CF90901000ED88090
:1011A0002854000E29540EE2D5EC26F004E3090180
:1011B000A36BA46B07D066EC2DF066EC26F0FDE186
:1011C000C7EC27F0D7EC22F0013406E261EC26F000
:1011D00003E2F8EC22F004D0A3C9A1F9A4C9A2F952
:1011E000150E0901945D03E1040EB8EC24F0090129
:1011F0009451020808E2010E946F03C909F904C969
:101200000AF9FAD861D00901000ED8800355000E02
:1012100004552CE270EC24F0013428E261EC26F055
:1012200025E2060EDB50026E036ADECF04F0DDCF4E
:1012300005F003500518E8AE02D0053404D0045080
:10124000025C0550035812E30051066E076ADECFB8
:1012500008F0DDCF09F007500918E8AE02D00934D4
:1012600004D00850065C0950075828E3D5EC26F056
:101270002DE2020EDBCF0AF0030EDBCF0BF00B34B6
:1012800025E20A500008000E0B5420E2020EDBCFCC
:101290000CF0030EDBCF0DF009010C50A15D0D50D9
:1012A000A25914E3020EDBCF0EF0030EDBCF0FF0DA
:1012B00009010E50015D0F50025908E20901020EAA
:1012C000946F040EB8EC24F0020E0DD0020E09014A
:1012D000945D0BE00901B80E035D240E045905E38B
:1012E0000901020E946FB8EC24F0060EDBCF00F972
:1012F000A1C901F9A2C902F947D00901D5EC26F02C
:101300001CE2D5EC26F004E30901A36BA46B07D023
:1013100066EC2DF066EC26F0FDE1C7EC27F0D7EC8B
:1013200022F0013406E261EC26F003E2F8EC22F050
:1013300004D0A3C9A1F9A4C9A2F9090194510208D2
:1013400013E30901100E095D270E0A5903E3090191
:10135000040E02D00901150E946F040EB8EC24F0AF
:10136000020EB8EC24F010D009019951800B0CE06A
:101370009951100B09E19951040B06E09995090167
:10138000040E946F53EC27F00901000ED8800D5520
:10139000000E0E5516E20501ED51000812E2C8C715
:1013A00000F0C9C701F0050E2D6E2E6AC8C728F0DF
:1013B000C9C729F0CEECA8F02450251002E109019C
:1013C0001887000E006E070EE15C02E2E16AE5524A
:1013D000E16E0050EFEF22F0090117BF08D0400E78
:1013E000176F09018E6B8F6B0901906B000C179FB3
:1013F000000C09011885000CA39098EC2AF013C981
:101400003EF914C93FF98AEC25F0A380A3EF2AF036
:10141000EAEC22F0100EE126090117A9EFD009012C
:10142000E35103E197EC26F0E9D009015C515D112D
:101430005E115F1107E180EC26F0A3908AEC25F0A5
:10144000A380DCD05C0EE96E090EEA6EEE500F5DF3
:10145000266EEE501059276EEE501159286EEE5040
:101460001259296EADEC2CF0F0ECA7F022C0DEFF93
:1014700023C0DEFF24C0DEFF25C0DDFFDD52DD52CC
:1014800025EC2AF0D890030EEB50000A08E6640E13
:10149000EE5C000EEE58000EEE58000EEE5801E223
:1014A000ADD0A390080E62C9DBFF090E63C9DBFF54
:1014B0000A0E64C9DBFF0B0E65C9DBFF0C0E66C9A3
:1014C000DBFF0D0E67C9DBFF0E0E68C9DBFF0F0ED9
:1014D00069C9DBFF09018AEC25F0A380605109018D
:1014E000DB5D006EDC5109016155016E43EC24F0B7
:1014F000D7EC22F0026A036A01AE02D002680368E8
:10150000640E61EC29F0B6EC29F055EC84F0060E7F
:1015100026C0DBFF070E27C0DBFF80EC26F075EC52
:1015200023F0D890015002E651EC28F02BE3DF5075
:1015300009014027010EDB504123020EDB504223FC
:10154000030EDB504323BFEC2BF0285044272950D7
:101550004523080EDB504627090EDB5047230A0EB1
:10156000DB5048230B0EDB5049230C0EDB504A277F
:101570000D0EDB504B230E0EDB504C230F0EDB50B9
:101580004D233CD075EC23F0013438E30050FF08C4
:10159000FF0E015433E3DF5009014E27010EDB50EB
:1015A0004F23020EDB505023030EDB5051232868DB
:1015B0002968040EDBCF2DF0050EDBCF2EF089EC71
:1015C00084F026500901522727505323080EDB5080
:1015D0005427090EDB5055230A0EDB5056230B0E01
:1015E000DB5057230C0EDB5058270D0EDB505923D0
:1015F0000E0EDB505A230F0EDB505B23100EE15C06
:1016000002E2E16AE552E16EEFEF22F0EAEC22F04D
:10161000190EE1260C0EDB6A0D0EDB6A0E0EDB6A7C
:10162000CBEC24F000C0DFFF010E01C0DBFF020E97
:1016300002C0DBFF030E03C0DBFF8DEC26F013ECD2
:101640002CF007E1010EDE6EDE6ADE6ADD6ADD5235
:10165000DD52E5EC24F043EC24F0060E02C0DBFF83
:10166000070E84EC24F0080E00C0DBFF090E01C059
:10167000DBFF0A0E02C0DBFF0B0E03C0DBFF19C944
:1016800000F01AC901F01BC902F01CC903F09FEC5D
:101690002CF019C926F01AC927F01BC928F01CC95B
:1016A00029F018EC2CF00C0E26C0DBFF25C900F049
:1016B00026C901F027C902F028C903F09FEC2CF0DD
:1016C00025C926F026C927F027C928F028C929F0FE
:1016D00018EC2CF00D0E26C0DBFF31C900F032C92A
:1016E00001F033C902F034C903F09FEC2CF031C98A
:1016F00026F032C927F033C928F034C929F018EC94
:101700002CF00E0E26C0DBFF28EC2BF083EC2CF027
:10171000FE0EDB50740801E0C3D0D7EC22F028ECB9
:1017200027F0A9EC21F0DA0EE66EE40EE66E000E6C
:1017300010EC22F00EEC28F00A0EDBCF02F00B0EBC
:10174000DBCF03F006EC29F0010EE66EE66A8DECC5
:1017500026F0E80E2B6E030E2C6E93EC28F0B3EC03
:101760002CF0D20EE66EE40EE66E000E67EC2CF066
:10177000B1EC2DF00FEC2BF00C0EC6EC2CF0C60EDD
:10178000E66EE40EE66E000E9DEC28F01DC900F03A
:101790001EC901F01FC902F020C903F007EC2AF0AE
:1017A00000EC2DF006EC29F00D0EC6EC2CF0B60E78
:1017B000E66EE40EE66E000E9DEC28F029C900F0FE
:1017C0002AC901F02BC902F02CC903F007EC2AF05A
:1017D0002DC900F02EC901F02FC902F030C903F065
:1017E00006EC29F00E0EC6EC2CF0AA0EE66EE40E06
:1017F000E66E000E9DEC28F035C900F036C901F008
:1018000037C902F038C903F007EC2AF039C900F0F3
:101810003AC901F03BC902F03CC903F006EC29F0DB
:10182000ADEC2AF0A10EE66EE40EE66E000E10ECB2
:1018300022F046C900F047C901F048C902F049C981
:1018400003F0FDEC2AF04AC900F04BC901F04CC985
:1018500002F04DC903F006EC29F0B6EC2AF0920E26
:10186000E66EE40EE66E000E10EC22F054C900F0B5
:1018700055C901F056C902F057C903F0FDEC2AF032
:1018800058C900F059C901F05AC902F05BC903F008
:1018900006EC29F08E0EE66EE40EE66E000E42D1E6
:1018A00025EC2AF0150EEECFDBFF160EEECFDBFF98
:1018B000170EEECFDBFF180EEECFDBFFDAEC28F0D1
:1018C000D7EC22F028EC27F013EC2CF011E0150EE9
:1018D000DBCF04F0160EDBCF05F0170EDBCF06F0E2
:1018E000180EDBCF07F0045005100610071006E1B4
:1018F000580EE66EE40EE66E000E14D1BFEC28F032
:10190000100E2B6E270E46EC29F04C0EE66EE40E00
:10191000E66E000EB6EC21F098EC28F0040E1DC91E
:10192000DBFF050E1EC9DBFF060E1FC9DBFF070E1E
:1019300020C9DBFF080E21C9DBFF090E22C9DBFF2E
:101940000A0E23C9DBFF0B0E24C9DBFF150E19C9D4
:10195000DBFF160E1AC9DBFF170E1BC9DBFF180EC3
:101960001CC9DBFF18EC22F00DE26AEC23F00AE25E
:101970000C0EC6EC2CF0370EE66EE40EE66E000E92
:1019800058EC2CF0040E29C9DBFF050E2AC9DBFF39
:10199000060E2BC9DBFF070E2CC9DBFF080E2DC975
:1019A000DBFF090E2EC9DBFF0A0E2FC9DBFF0B0E72
:1019B00030C9DBFF150E25C9DBFF160E26C9DBFF7C
:1019C000170E27C9DBFF180E28C9DBFF18EC22F021
:1019D0000DE26AEC23F00AE20D0EC6EC2CF02B0EA1
:1019E000E66EE40EE66E000E58EC2CF0040E35C9DF
:1019F000DBFF050E36C9DBFF060E37C9DBFF070E1E
:101A000038C9DBFF080E39C9DBFF090E3AC9DBFF15
:101A10000A0E3BC9DBFF0B0E3CC9DBFF150E31C9BB
:101A2000DBFF160E32C9DBFF170E33C9DBFF180EC2
:101A300034C9DBFF18EC22F00DE26AEC23F00AE275
:101A40000E0EC6EC2CF0220EE66EE40EE66E000ED4
:101A500058EC2CF0040E46C9DBFF050E47C9DBFF2E
:101A6000060E48C9DBFF070E49C9DBFF080E4AC94D
:101A7000DBFF090E4BC9DBFF0A0E4CC9DBFF0B0E67
:101A80004DC9DBFF150E40C9DBFF160E41C9DBFF58
:101A9000170E42C9DBFF180E43C9DBFF18EC22F01A
:101AA0000EE26AEC23F00BE254EC28F01C0EE66E1A
:101AB000E40EE66E000EEFEC2CF098EC28F0040E2D
:101AC00054C9DBFF050E55C9DBFF060E56C9DBFF07
:101AD000070E57C9DBFF080E58C9DBFF090E59C9AD
:101AE000DBFF0A0E5AC9DBFF0B0E5BC9DBFF150ECD
:101AF0004EC9DBFF160E4FC9DBFF170E50C9DBFFC7
:101B0000180E51C9DBFF18EC22F00EE26AEC23F04C
:101B10000BE259EC28F0110EE66EE40EE66E000EB4
:101B2000EFEC2CF098EC28F0190EE15C02E2E16A8F
:101B3000E552E16EEFEF22F0EAEC22F0020E9FECAC
:101B400026F0D00EEE1801E0AED0ED5001E0ABD0A3
:101B5000F10EE66EE30EE66E000E0FEC29F019C9E9
:101B6000E6FF1AC9E6FF1BC9E6FF1CC9E6FF06EC43
:101B700022F01DC9E6FF1EC9E6FF1FC9E6FF20C906
:101B8000E6FF06EC22F021C9E6FF22C9E6FF23C9E1
:101B9000E6FF24C9E6FF06EC22F025C9E6FF26C9C8
:101BA000E6FF27C9E6FF28C9E6FF06EC22F029C9AF
:101BB000E6FF2AC9E6FF2BC9E6FF2CC9E6FF06ECC3
:101BC00022F02DC9E6FF2EC9E6FF2FC9E6FF30C976
:101BD000E6FF06EC22F031C9E6FF32C9E6FF33C961
:101BE000E6FF34C9E6FF06EC22F035C9E6FF36C948
:101BF000E6FF37C9E6FF38C9E6FF06EC22F039C92F
:101C0000E6FF3AC9E6FF3BC9E6FF3CC9E6FF06EC42
:101C100022F040C9E6FF41C9E6FF42C9E6FF43C9D9
:101C2000E6FF06EC22F0ADEC2AF0E2EC2CF046C91F
:101C3000E6FF47C9E6FF48C9E6FF49C9E6FF06ECEB
:101C400022F04AC9E6FF4BC9E6FF4CC9E6FF4DC981
:101C5000E6FF06EC22F04EC9E6FF4FC9E6FF50C989
:101C6000E6FF51C9E6FF06EC22F0B6EC2AF0E2EC02
:101C70002CF054C9E6FF55C9E6FF56C9E6FF57C91F
:101C8000E6FF06EC22F058C9E6FF59C9E6FF5AC93B
:101C9000E6FF5BC9E6FF06EC22F06C0EE66E090E6D
:101CA000E66E37EC24F0FE0EDB50B7EC27F002E2D4
:101CB000E16AE552E16E0050EFEF22F0EAEC22F02B
:101CC000E652FE0EDB500FE00501F3B50CD0B2EC8E
:101CD00029F003E058EC23F008E1A1EC28F003E040
:101CE00058EC23F002E1000E11D0F1EC2AF004E0F0
:101CF00056EC25F0200901D0650EDF6E0601006B61
:101D0000DFCFE6FF83DCE55209EC2DF0E552EFEF83
:101D100022F0EAEC22F0030E9FEC26F0D00EEE1833
:101D200011E1ED500FE1FE0EDB5005E05AEC25F01D
:101D300086EC27F020D065EC27F086EC27F002082F
:101D400029E026D0F5EC2AF005E065EC25F0EF500F
:101D5000200901D0650EE76E020EE7CFDBFFDAEC5B
:101D600029F0020EDBCFE6FF51DCE552FE0EDB5020
:101D70000BE03AEC2EF0EFEC29F00FEC2DF06CECD0
:101D80002DF0F7EC2CF006D00DEC2EF03AEC2EF006
:101D90002AEC2EF0010E006E030EE15C02E2E16A15
:101DA000E552E16E0050EFEF22F06DEC2AF0FE0EEE
:101DB000DBCFE6FF76EC31F0E552E76EFE0EE7CFC3
:101DC000DBFF93EC2CF003E04CEC26F003D0C80EC4
:101DD000006E016A10EC2AF00901175165EC2AF037
:101DE00086EC22F00901995172EC2DF009019D5108
:101DF00072EC2DF009019451D8EC2DF00DC9E6FFDD
:101E00000EC9E6FF52EC2CF015C9E6FF16C9E6FF35
:101E100052EC2CF069EC27F006EC22F063EC28F091
:101E200052EC2CF068EC28F052EC2CF06DEC28F021
:101E300052EC2CF00BC9E6FF0CC9E6FF52EC2CF07B
:101E400007C9E6FF08C9E6FF52EC2CF0A3C9E6FF7C
:101E5000A4C9E6FF52EC2CF0A1C9E6FFA2C9E6FF37
:101E600052EC2CF00701CA51D8EC2DF08EEC27F083
:101E700002E1010E02D0FE0EDB50B7EC27F002E2C9
:101E8000E16AE552E16E0050EFEF22F0EAEC22F059
:101E9000E150FA0F9EEC22F00AE065EC25F0EF50DD
:101EA00006E0F6EC29F093EC25F072EC27F0FE0E3C
:101EB000DB5006E05AEC25F078DFE552E552E552BA
:101EC000010EEFEF22F06DEC2AF0F1EC2AF009E0C0
:101ED00056EC25F006E0BFEC24F093EC25F072EC14
:101EE00027F00501F3B50CD0B2EC29F003E058EC73
:101EF00023F008E1A1EC28F003E058EC23F002E124
:101F0000000ECFD0FE0EDB5002E06EEC23F072EC40
:101F100028F009011751E66EE66ACD0EE66EE30E73
:101F2000E66E000E86EC22F069EC27F0C70EE66E36
:101F3000E30EE66E000E04EC2AF0DEEC2CF0F9EC79
:101F400027F000EC2CF0C20EE66EE30EE66E000EFB
:101F5000BBEC22F03EC900F03FC901F0026A036AFF
:101F600000EC2CF0BD0EE66EE30EE66E000EBBEC50
:101F700022F00901E951E66EE66AB80EE66EE30E5C
:101F8000E66E000E43EC29F08DEC29F07F0E060181
:101F9000C85D35E172EC28F00901E051E66EE66AB1
:101FA000B00EE66EE30EE66E000E43EC29F04AEC4E
:101FB00027F0AA0EE66EE30EE66E000E71EC2BF033
:101FC000EFEC25F0A40EE66EE30EE66E000E71EC6B
:101FD0002BF079EC26F09E0EE66EE30EE66E000E18
:101FE00043EC29F0D9C9E6FFDAC9E6FF980EE66EA0
:101FF000E30EE66E000E43EC29F08DEC29F072EC56
:1020000028F066C0E6FF67C0E6FF910EE66EE30EBD
:10201000E66E000E86EC22F068C0E6FF69C0E6FFBF
:102020008C0EE66EE30EE66E000E86EC22F06AC0C1
:10203000E6FF6BC0E6FF860EE66EE30EE66E000E70
:1020400086EC22F000016C51E66EE66A810EE66EC7
:10205000E30EE66E000E86EC22F000016D51E66E96
:10206000E66A7C0EE66EE30EE66E000E86EC22F06B
:1020700000016E51E66EE66A760EE66EE30EE66EDF
:10208000000E86EC22F00001FE51E66EE66A710E4B
:10209000E66EE30EE66E000E86EC22F08DEC29F083
:1020A000010EB7EC27F002E2E16AE552E16E005062
:1020B000EFEF22F06DEC2AF028EC2BF06FEC2CF017
:1020C000090199A53FD009019451040A10E0060ABC
:1020D00008E0030A12E1680EE66EE30EE66E000EFB
:1020E00011D0520EE66EE30EE66E000E0BD0440EDB
:1020F000E66EE30EE66E000E05D0330EE66EE30EDE
:10210000E66E000E86EC28F000EC2DF0A9EC21F034
:102110002B0EE66EE30EE66E000EBBEC22F08E0E8A
:10212000E66EE40EE66E000E86EC28F0040E090161
:10213000945D1EE0A8EC23F0220EE66EE30EE66E40
:10214000000E14D00F0EE66EE30EE66E000E86EC67
:1021500028F00901100E035D270E045909E2A8ECCE
:1021600023F0FF0EE66EE20EE66E000E78EC2DF028
:10217000B3EC27F01CE1A3C9E6FFA4C9E6FFF50E06
:10218000E66EE20EE66E000E43EC29F0A1C9E6FF12
:10219000A2C9E6FFF10EE66EE20EE66E000E43EC1B
:1021A00029F0ED0EE66EE20EE66E000E27D0A3C912
:1021B00000F0A4C901F0040EA7EC25F0FDE1ECEC61
:1021C0002DF0F50EE66EE20EE66E000EB5EC22F096
:1021D000A1C900F0A2C901F0040EA7EC25F0FDE1B1
:1021E000ECEC2DF0F10EE66EE20EE66E000EB5ECB4
:1021F00022F0E90EE66EE20EE66E000E86EC28F0A6
:10220000020EE66EE66A03C900F004C901F0026A34
:10221000036A63EC28F00DEC25F0E10EE66EE20EA9
:10222000E66E000E5DEC24F0020EE66EE66A05C96D
:1022300000F006C901F0026A036A68EC28F00DECB0
:1022400025F0DD0EE66EE20EE66E000E5DEC24F08B
:10225000020EE66EE66A09C900F00AC901F0026AD8
:10226000036A6DEC28F00DEC25F0D90EE66EE20E57
:10227000E66E000E5DEC24F0D60EE66EE20EE66E23
:10228000000E86EC28F0B3EC27F01DE1CDC900F07C
:10229000CEC901F0CFC902F0D0C903F008EC26F096
:1022A00049EC2CF0B6EC2DF0B3EC2CF0CE0EE66E33
:1022B000E20EE66E000EBBEC22F0ED0EE66EE20ED4
:1022C000E66E000E2FD0CDC904F0CEC905F0CFC9FF
:1022D00006F0D0C907F008EC26F026C004F027C0AD
:1022E00005F028C006F029C007F0040E1F0B49ECCA
:1022F0002CF003E05EEC25F0FDE1050E07EC24F088
:10230000CE0EE66EE20EE66E000E04EC2AF0086ECB
:10231000090EE15E08506FEC2CF0E90EE66EE20E5D
:10232000E66E000E86EC28F0020EE15C02E2E16A45
:10233000E552E16EEFEF22F0EAEC22F0FE0EDB5008
:102340000FE00501F3B50CD0B2EC29F003E058EC36
:1023500023F008E1A1EC28F003E058EC23F002E1BF
:10236000000E05D00601006BA5DE09EC2DF0EFEFA5
:1023700022F0EAEC22F0DAEC29F09CDE3AEC2EF0C6
:10238000010EEFEF22F06DEC2AF093EC2CF003E05D
:102390004CEC26F003D0C90E006E016A10EC2AF056
:1023A0000501F15165EC2AF043EC29F08EEC27F0A1
:1023B00002E1010E02D0FE0EDB50B7EC27F002E284
:1023C000E16AE552E16E0050EFEF22F0EAEC22F014
:1023D000E1502DEC2BF0CA0EEE1815E1ED5013E193
:1023E000F5EC2AF009E065EC25F0EF5005E0F6EC9D
:1023F00029F015EC28F002D00501F16BF6EC29F07C
:102400001C0E6CEC25F0FE0EDB5006E05AEC25F0BD
:10241000BADFE552E552E552010EEFEF22F029EC6A
:102420002CF028E0B2EC29F003E058EC23F006E1B0
:10243000A1EC28F01FE058EC23F01CE0F5EC2AF0AA
:1024400016E0050E74EC2BF012E0F1EC2AF008E037
:1024500056EC25F005E0BFEC24F015EC28F002D096
:102460000501F16BBFEC24F01C0E6CEC25F00501AE
:10247000F3A502D0000E31D06EEC23F0BC0EE66E58
:10248000E20EE66E000E0FEC29F00501F1510AE1B3
:10249000B60EE66EE20EE66E000E55EC2CF025EC64
:1024A00022F016D0F151D6EC2AF0B3EC27F006E179
:1024B000ED0E006EE20E016E000E05D0E90E006E0C
:1024C000E20E016E000E026E4CEC23F0BBEC26F027
:1024D0006FEC2CF08DEC29F0010EB7EC27F002E246
:1024E000E16AE552E16E0050EFEF22F0EAEC22F0F3
:1024F000080EE126020EDB6A1CEC28F0050133EC25
:1025000026F02DEC2CF00501F151000807E2F15105
:10251000E66ED950060F4FEC25F02AD0090105517F
:1025200006110AE00751081107E0A5EC22F0C4ECFF
:1025300026F0DCEC2AF004D0060EDB6A070EDB6A1C
:10254000B3EC27F015E128EC27F0033402E2A0EC0D
:1025500027F003E3006A016A09D075EC23F0ADECC3
:1025600029F066EC26F0FDE16BEC26F0FEEC26F09F
:10257000D950060F21EC2AF00FE0060EDBCF08F051
:10258000070EDBCF09F00A6A0B6A09AE02D00A68AF
:102590000B6822EC23F002D0006A016A43EC24F0BD
:1025A00093EC2CF003E04CEC26F003D0CB0E006E45
:1025B000016A10EC2AF00501F05165EC2AF043ECB9
:1025C00029F00501EF51D8EC2DF0040EDBCFE6FF2A
:1025D000050EDBCFE6FF52EC2CF00EEC24F052ECB3
:1025E0002CF0A8EC23F080EC28F0B5EC22F08EEC77
:1025F00027F002E1010E02D0FE0EDB50006E080E45
:10260000E15C02E2E16AE552E16E0050EFEF22F098
:10261000EAEC22F0040E9FEC26F0CC0EEE1845E119
:10262000ED5043E1DE6ADD6A09EC2CF0F5EC2AF0AE
:1026300016E065EC25F0EF5012E080EC28F0E66E35
:10264000F6EC29F023EC28F06FEC2CF080EC28F06D
:10265000E66E9DEC2BF023EC28F02DEC2CF025EC15
:102660002AF0EE50ED1005E0E7EC2DF093EC25F0AC
:1026700002D0006A016A00C0F0F5D950020F21ECC7
:102680002AF005E00EEC24F093EC25F002D0006A6D
:10269000016A00C0EFF5E7EC2DF01B0E6CEC25F0A5
:1026A0000EEC24F01A0E6CEC25F0FE0EDB5006E06A
:1026B0005AEC25F01BDFE552E552E552010E006EA3
:1026C000040EE15C02E2E16AE552E16E0050EFEFD8
:1026D00022F0EAEC22F0100EE126FE0EDB5068E05C
:1026E000B2EC29F003E058EC23F006E1A1EC28F06D
:1026F0005FE058EC23F05CE0F5EC2AF056E0020EC7
:1027000074EC2BF052E0060EDB6A27EC28F0050192
:10271000EF6BF06BF1EC2AF03EE056EC25F03BE07D
:10272000BFEC24F0DFEC89F0E552E5522DEC2CF003
:10273000BFEC24F0A3EC98F01DEC2AF00006000E8C
:10274000015AF80EDB500024E96EF90EDB5001202F
:10275000EA6E040EEFCFDBFFDB50250808E12EEC1C
:1027600028F0DCEC2AF0020EDBCFEFF507D02EECE0
:1027700028F035EC28F0020EDBCFF0F5BFEC24F0AA
:102780006EEC5AF0E552E552F80EF3CFDBFFF90E8E
:10279000F4CFDBFFBFD7C6EC2BF01A0E6CEC25F0A4
:1027A000E3EC2AF01B0E6CEC25F00501F3A502D03A
:1027B000000EFED06EEC23F0A70EE66EE20EE66E83
:1027C000000E0FEC29F00501EF5108E1F05106E190
:1027D000A30EE66EE20EE66E000EDCD013EC2BF0DC
:1027E000EF51000813E233EC26F00A0EF3CFDBFFC3
:1027F0000B0EF4CFDBFF0501EF51D6EC2AF0400EB3
:10280000E66EE40EE66E000E86EC28F00501F0514F
:10281000000801E384D0F151000807E2F151E66EAF
:10282000D9500E0F4FEC25F03AD009010551061191
:102830000EE0075108110BE0A5EC22F0C4EC26F0E5
:102840000E0E28C0DBFF0F0E29C0DBFF04D00E0EDA
:10285000DB6A0F0EDB6AB3EC27F021E10E0EDBCF53
:1028600002F00F0EDBCF03F0033402E2A0EC27F0FE
:1028700003E3006A016A0DD00E0EDBCF00F00F0EED
:10288000DBCF01F0ADEC29F066EC26F0FDE16BEC5E
:1028900026F00E0E00C0DBFF0F0E01C0DBFFD9508B
:1028A0000E0F21EC2AF00FE00E0EDBCF08F00F0E1A
:1028B000DBCF09F00A6A0B6A09AE02D00A680B681E
:1028C00022EC23F002D0006A016A0C0E00C0DBFF8C
:1028D0000D0E01C0DBFF0501EF51000807E29E0E5F
:1028E000E66EE20EE66E000E86EC28F00501F05171
:1028F000D6EC2AF0B3EC27F006E1ED0E006EE20E06
:10290000016E000E05D0E90E006EE20E016E000EA3
:10291000026E4CEC23F0BBEC26F06FEC2CF000ECDC
:1029200028F0013420E261EC26F01DE2D9500A0FB4
:1029300021EC2AF013E0E4EC27F00A0EDBCF04F0E0
:102940000B0EDBCF05F003500518E8AE02D00534BE
:1029500004D00450025C0550035805E20C0EDBCF96
:10296000E6FF0D0E0BD0EBEC27F0013411E261EC29
:1029700026F00EE20A0EDBCFE6FF0B0EDBCFE6FF02
:10298000950EE66EE20EE66E000EE66EF4EC21F0B9
:1029900094EC27F086EC28F0A8EC23F0850EE66E88
:1029A000E20EE66E000E78EC2DF08DEC29F0010EB3
:1029B000006E100EE15C02E2E16AE552E16E005049
:1029C000EFEF22F0EAEC22F0E652090117AD02D057
:1029D000010E14D00B0EDF6E3F0E0001FE5D08E00D
:1029E000DF50000805E2010EA5EC27F0DF06F4D762
:1029F0003F0EFE5D02E0000E01D0010EE552EFEF4A
:102A000022F06DEC2AF0DEDFDE6ADD6A72EC2AF07D
:102A100002E632EC2CF02EE229EC22F0030EC1EC9F
:102A200022F0FDE18EEC2CF0C1EC22F0FDE1F3ECA4
:102A300022F0040E75EC24F029EC22F0030EC1EC18
:102A400022F0FDE18EEC2CF0C1EC22F0FDE1D4ECA3
:102A50002DF075EC24F029EC22F0030EC1EC22F0ED
:102A6000FDE1EBEC2CF057EC26F0DF2A010ECEE373
:102A7000DB2ACCD7DE6ADD6A72EC2AF002E64DEC86
:102A80002BF013E216EC2DF0CAEC26F016EC2DF02C
:102A900079EC27F019EC29F062EC2DF033EC27F0FB
:102AA000DF2A010EE9E3DB2AE7D7DE6ADD6A72EC92
:102AB0002AF002E651EC28F029E2F5EC2DF0020EA6
:102AC00075EC24F0F5EC2DF0040E75EC24F015EC0B
:102AD00029F00F0EBBEC2DF0110E35EC2DF00C0E85
:102AE00035EC2DF00D0E35EC2DF0060EBBEC2DF077
:102AF000080EBBEC2DF00E0E35EC2DF00A0E57EC47
:102B000026F0DF2A010ED3E3DB2AD1D70001FE6BCA
:102B1000020EE15C02E2E16AE552E16EEFEF22F0C3
:102B2000EAEC22F0180EE1263F0E0001FE5D01E006
:102B3000E6D3ACEC25F070EC24F0070EEDEC25F0BC
:102B400001E397D029EC22F0020EC1EC22F0FDE166
:102B5000B5EC28F0EF5001E18CD029EC22F0020E08
:102B6000C1EC22F0FDE153EC26F0F00E005C01E335
:102B700080D029EC22F0020EC1EC22F0FDE1B5EC90
:102B800028F0EE52EF5014E029EC22F0020EC1ECD6
:102B900022F0FDE153EC26F029EC22F0020EC1EC0C
:102BA00022F0FDE1B5EC28F0EE52EF50005C0DE2B2
:102BB00029EC22F0020EC1EC22F0FDE14CEC2DF0EC
:102BC000C1EC22F0FDE179EC27F029EC22F0020EB5
:102BD000C1EC22F0FDE1B5EC28F0020ED9EC23F0B7
:102BE00016E029EC22F0020EC1EC22F0FDE153ECDC
:102BF00026F029EC22F0020EC1EC22F0FDE1B5EC4A
:102C000028F0020ED9EC23F0D88000540DE229EC14
:102C100022F0020EC1EC22F0FDE14CEC2DF0C1ECF3
:102C200022F0FDE1CAEC26F029EC22F0020EC1EC04
:102C300022F0FDE153EC26F0016A80EC2AF0020E4E
:102C4000C1EC22F0FDE13CEC28F0096A0A6A0B6A4B
:102C500029EC22F0020EC1EC22F0FDE1B5EC28F0E7
:102C6000EFCF04F0056ADDEC23F001E264D7DB2A44
:102C700062D725EC2AF0070EEE1801E03FD1ED50A7
:102C800001E03CD115EC24F0E00E2E6E400E14EC69
:102C900026F04BEC2AF01DEC85F07FEC82F01DEC69
:102CA00029F033EC2BF0BFEC82F0BAEC28F02C6A60
:102CB0002D6A200E2E6E420E2F6EBEEC82F01DECA1
:102CC00085F029C0C2F90901780EE26F20EC24F0EA
:102CD000E00E2E6E400E40EC22F005E1010EF36E88
:102CE00070EC26F0DB6A51EC23F000017151026EAA
:102CF000036A03EC26F016E2020EDBCF71F0DBCFA5
:102D000000F0030EDBCF01F0EDEC25F003E3800EC5
:102D10006D6F08D051EC23F0020EEDEC25F002E3CC
:102D2000800E6C6FDE6ADD6A70EC24F0070EEDEC4D
:102D300025F001E3E3D029EC22F0020EC1EC22F0F1
:102D4000FDE13CEC28F008C029F07DEC82F047EC76
:102D500027F0DBCF09F0150EDBCF0AF0160EDBCF24
:102D60000BF0170EDBCF0CF0EAEC2AF00CC02FF0C2
:102D70007EEC2DF0020EC1EC22F0FDE1B5EC28F066
:102D8000EFCF15F015C029F07DEC82F027C011F0CF
:102D900028C012F029C013F02AC014F0140EDBCFA3
:102DA00016F0150EDBCF17F0160EDBCF18F0170E4E
:102DB000DBCF19F016C02CF017C02DF018C02EF084
:102DC00019C02FF0AAEC85F0010A05E00D6A0E6A21
:102DD0000F6A3F0E04D00D6A0E6A0F6ABF0E106EA6
:102DE0000DC02CF00EC02DF00FC02EF09FEC24F083
:102DF00003E0CDEC2BF002D075EC23F043EC24F093
:102E0000800E00016D150CE039EC2BF009E3010E8A
:102E1000DF5211E0DFCFF3FFDCEC27F0FDE10BD058
:102E200039EC2BF00BE3010EDF5205E0DFCFF3FFAF
:102E3000DCEC27F0FDE100016D131FD0800E6C1556
:102E40000FE0D7EC22F0020EEDEC25F009E3010EC5
:102E5000DF5211E0DFCFF3FFDCEC27F0FDE10BD018
:102E6000D4EC2BF00AE2010EDF5205E0DFCFF3FFD6
:102E7000DCEC27F0FDE100016C13D7EC22F029EC2B
:102E800022F0020EC1EC22F0FDE162EC2DF0C3EC69
:102E900029F0EFCF04F004340DE329EC22F0020E08
:102EA000C1EC22F0FDE162EC2DF0D9EC23F0FF0D36
:102EB000F3500AD029EC22F0020EC1EC22F0FDE121
:102EC00062EC2DF0D9EC23F0026E036A02BE0368B7
:102ED00003EC26F00DE229EC22F0020EC1EC22F008
:102EE000FDE162EC2DF0C3EC29F0060EDBCFEFFF25
:102EF000DF2A010E01E218D7DB2A16D70001625142
:102F0000631105E06251605D6351615904E260C084
:102F100062F061C063F06451651105E06051645D69
:102F20006151655904E260C064F061C065F0ACECC9
:102F300025F070EC24F00E0EEDEC25F001E399D0B5
:102F400029EC22F0030EC1EC22F0FDE1F3EC22F0BB
:102F5000EE50ED1001E18DD029EC22F0030EC1EC12
:102F600022F0FDE102EC29F0000E005C0F0E01588A
:102F700001E37FD029EC22F0030EC1EC22F0FDE149
:102F8000D4EC2DF09DEC25F012E029EC22F0030E9C
:102F9000C1EC22F0FDE18EEC2CF0C1EC22F0FDE161
:102FA000D4EC2DF0DCEC25F0AAEC27F00FE229ECB4
:102FB00022F0030EC1EC22F0FDE18EEC2CF0C1EC0E
:102FC00022F0FDE1D4EC2DF075EC24F029EC22F098
:102FD000030EC1EC22F0FDE1F3EC22F0040E9DECB7
:102FE00025F013E029EC22F0030EC1EC22F0FDE104
:102FF0008EEC2CF0C1EC22F0FDE1F3EC22F0040E9B
:10300000DCEC25F003EC26F010E229EC22F0030EB4
:10301000C1EC22F0FDE18EEC2CF0C1EC22F0FDE1E0
:10302000F3EC22F0040E75EC24F029EC22F0030EF0
:10303000C1EC22F0FDE102EC29F080EC2AF0030E55
:10304000C1EC22F0FDE1DAEC2BF00A6A0B6A29EC04
:1030500022F0030EC1EC22F0FDE1F3EC22F0EECF02
:1030600004F0EFCF05F0DDEC23F001E262D7DB2ABC
:1030700060D725EC2AF00E0EEE1801E031D1ED50AC
:1030800001E02ED115EC24F0600E2E6E410E14ECF2
:1030900026F020EC24F0600E2E6E410E40EC22F063
:1030A00005E1010EF36E70EC26F0DB6A51EC23F0C3
:1030B000000100506F5D0150705918E2020EDBCF25
:1030C0006FF0030EDBCF70F051EC23F0050EEDEC4A
:1030D00025F004E3686B800E696F08D051EC23F093
:1030E000EDEC25F003E3666B800E676FDE6ADD6A48
:1030F00070EC24F00E0EEDEC25F001E3F1D029EC9C
:1031000022F0030EC1EC22F0FDE1DAEC2BF008C056
:1031100028F009C029F08EEC82F047EC27F0DBCFD5
:103120000AF0150EDBCF0BF0160EDBCF0CF0170EEE
:10313000DBCF0DF00AC02CF00BC02DF00CC02EF030
:103140000DC02FF07EEC2DF0030EC1EC22F0FDE15E
:10315000F3EC22F0EECF16F0EFCF17F016C028F008
:1031600017C029F08EEC82F027C012F028C013F0AF
:1031700029C014F02AC015F0140EDBCF18F0150E7C
:10318000DBCF19F0160EDBCF1AF0170EDBCF1BF0DA
:1031900018C02CF019C02DF01AC02EF01BC02FF053
:1031A000AAEC85F0010A05E00E6A0F6A106A3F0E6C
:1031B00004D00E6A0F6A106ABF0E116E0EC02CF09A
:1031C0000FC02DF010C02EF09FEC24F003E0CDECEA
:1031D0002BF002D075EC23F043EC24F00001695190
:1031E000800B0CE0D7EC22F0EDEC25F007E3E2ECED
:1031F00025F010E05EEC25F0FDE10CD0D7EC22F0DC
:10320000060EEDEC25F00CE3E2EC25F003E05EECBD
:1032100025F0FDE1005000016813015069131BD037
:103220006751800B0AE039EC2BF007E3E2EC25F064
:103230000DE05EEC25F0FDE109D0D4EC2BF00BE2C3
:10324000E2EC25F003E05EEC25F0FDE1005000012A
:10325000661301506713D7EC22F029EC22F0030E1D
:10326000C1EC22F0FDE1EBEC2CF0C3EC29F0EECF49
:1032700004F0EFCF05F00001800E05140EE029ECFC
:1032800022F0030EC1EC22F0FDE1EBEC2CF0DCECC3
:1032900025F0026C031E03220AD029EC22F0030E53
:1032A000C1EC22F0FDE1EBEC2CF0DCEC25F003ECC2
:1032B00026F010E229EC22F0030EC1EC22F0FDE131
:1032C000EBEC2CF0C3EC29F0060EDBCFEEFF070E83
:1032D000DBCFEDFFDF2A010E01E20AD7DB2A08D798
:1032E00000016A51681906E16B51691903E16E51D9
:1032F0006D5D03E0110E090118130001FE6B180E3D
:10330000E15C02E2E16AE552E16EEFEF22F0EAEC05
:1033100022F0080EE126D950FB0F9EEC22F002E0CD
:10332000A00E01D0C70E006E016A43EC24F028EC19
:103330002BF0E3EC22F07D0EE66EE20EE66E000E60
:10334000AFEC28F08BEC28F00F0E2AEC2AF08BEC77
:1033500028F0080E4FEC2BF003E035EC25F008D0F8
:103360008BEC28F0060E4FEC2BF004E03BEC25F044
:10337000AFEC28F00EEC24F089EC2AF084EC2DF070
:103380008BEC28F0080E9DEC25F00EE18BEC28F07C
:10339000060E9DEC25F008E16D0EE66EE20EE66E7F
:1033A000000EAFEC28F05CD0DE6ADD6A72EC2AF029
:1033B00002E632EC2CF054E234EC2CF00C0E9AECD9
:1033C00027F0E8AE02D0033402D0AAEC27F001E3E4
:1033D00099D08BEC28F0080E77EC2AF0DF501F0B09
:1033E00003E0B1EC24F0FDE160EC23F003E035EC08
:1033F00025F010D08BEC28F0060E77EC2AF0DF5089
:103400001F0B03E0B1EC24F0FDE160EC23F023E0BE
:103410003BEC25F0AFEC28F029EC22F0030EC1ECD8
:1034200022F0FDE1EBEC2CF02AEC2AF0E1EC2BF0A1
:10343000670EE66EE20EE66E000E8AEC2DF005E1F8
:103440000EEC24F0E1EC26F004D00EEC24F05BEC62
:1034500026F084EC2DF0DF2A010EA8E3DB2AA6D7A4
:1034600034EC2CF0140E9AEC27F0E8AE02D00334C2
:1034700002D0AAEC27F046E25A0EE66EE20EE66EA5
:10348000000EAFEC28F08BEC28F0110ED9EC23F0F5
:10349000E66ED950020F4FEC25F030EC2DF0800B8A
:1034A00003E035EC25F006D0BFEC2DF0800B04E0F6
:1034B0003BEC25F0AFEC28F00EEC24F089EC2AF080
:1034C00090EC2DF030EC2DF009E1BFEC2DF006E191
:1034D0006D0EE66EE20EE66E000E19D0DE6ADD6A53
:1034E00072EC2AF002E64DEC2BF05AE234EC2CF0B0
:1034F000080E9AEC27F0E8AE02D0033402D0AAEC12
:1035000027F008E3690EE66EE20EE66E000EAFEC01
:1035100028F046D0010EDF5205E0DFCFF3FFDCECF0
:1035200027F0FDE1006E30EC2DF0001403E035ECE7
:1035300025F00FD0010EDF5205E0DFCFF3FFDCEC0A
:1035400027F0FDE1006EBFEC2DF0001424E03BEC11
:1035500025F0AFEC28F019EC29F062EC2DF0A2EC8C
:1035600025F0016A00BE01683EEC26F0E1EC2BF08C
:10357000550EE66EE20EE66E000E8AEC2DF005E1C9
:103580000EEC24F0E1EC26F004D00EEC24F05BEC21
:1035900026F090EC2DF0DF2A010EA2E3DB2AA0D763
:1035A000080EE15C02E2E16AE552E16EEFEF22F023
:1035B000EAEC22F00A0EE126E2EC14F0000905E143
:1035C000FE0EDB50000801E2AED1D9502DEC2BF0FD
:1035D000CD0EEE1830E1ED502EE1DF6A010EDF5C1A
:1035E00001E3A1D12EEC22F0080E9DEC25F003E1C1
:1035F0003EEC2BF013E0DAEC29F09DEC2BF0DFCF62
:10360000E6FFCFEC27F0016ADF34FE0B0136006ED7
:103610006E0E0026090E43EC2BF00BD0EA6ADF3465
:10362000FE0BEA36E96E6E0EE926090EEA22EE6A14
:10363000ED6ADF2AD3D7020EDB681CEC28F0010EFE
:10364000DB6A070E40EC28F02DE2F9EC2AF0EF508F
:10365000006E016AD950040FD5EC27F0F9EC2AF07E
:10366000EE52EFCF00F0020EDB50005C06E2F9EC08
:103670002AF0EE52020EEFCFDBFFF9EC2AF0020E39
:10368000A2EC25F0030EDB50D880005408E2F9ECE0
:103690002AF0020EC3EC29F0030EEFCFDBFF010E80
:1036A000DB2ACFD7040EDBCF28F0050EF3EC23F096
:1036B000040E28C0DBFF050E29C0DBFFDF6A010E08
:1036C000DF5C01E330D12EEC22F0080E9DEC25F0FA
:1036D00002E0030E09D02EEC22F0060E9DEC25F040
:1036E00002E0020E01D0010EF36E060EF3CFDBFFF7
:1036F0003EEC2BF002E0030E08D02EEC22F046EC5C
:103700002CF002E0020E01D0010E91EC29F0DF282E
:10371000E66EE66A3D0EE66EE20EE66E000E1EEC0A
:1037200022F00E0E06EC2BF0010EE66EE66A8AEC35
:103730002CF0DCEC2DF063EC28F08AEC2CF068EC3B
:1037400028F08AEC2CF06DEC28F08AEC2CF02EECB2
:1037500022F0B8EC2CF019EC2AF0B8EC2CF02BECA1
:1037600029F02EEC22F0020E8EEC22F019EC2AF059
:10377000020E8EEC22F02BEC29F02EEC22F0040E3F
:103780008EEC22F019EC2AF0040E8EEC22F02BECD9
:1037900029F0D7EC22F0E7EC2BF0EBEC21F0020E55
:1037A0008FEC2AF0EBEC21F0030E8FEC2AF0C3EC47
:1037B0002DF00F0E26EC29F0C3EC2DF0110ED9ECF4
:1037C00023F0E66EE66A8AEC2CF0016ADF34FE0B29
:1037D0000136006E700E0026090E43EC2BF0010E30
:1037E000DB6A0E0E40EC28F001E39BD02EEC22F0B9
:1037F000080E77EC2AF0DB501F0B03E0B1EC24F04D
:10380000FDE160EC23F002E0030E11D02EEC22F07B
:10381000060E77EC2AF0DB501F0B03E0B1EC24F02E
:10382000FDE160EC23F002E0020E01D0010EF36E28
:10383000060EF3CFDBFFE0EC27F0016E010E015224
:1038400004E0E846FE0B0106FCE1006E3EEC2BF0C6
:10385000001402E0030E14D0E0EC27F0016E010E1C
:10386000015204E0E846FE0B0106FCE1006E2EEC7E
:1038700022F046EC2CF0001402E0020E01D0010E02
:1038800091EC29F0010EDB28E66EE66A2C0EE66E5E
:10389000E20EE66E000E1EEC22F0DF2806EC2BF0A6
:1038A000DCEC2DF0010EDB50080DC1EC2CF002EC2D
:1038B00029F0050EC7EC2DF09FEC29F0020E26EC46
:1038C00029F09FEC29F0040E26EC29F09FEC29F05A
:1038D000060E26EC29F096EC2DF0EF50E3EC29F0E3
:1038E000EE52EF50E3EC29F0020ED9EC23F0E3ECBA
:1038F00029F0030EA2EC25F0016A00BE01684CEC31
:1039000023F0EBEC21F0010E016ADB34FE0B0136F3
:10391000006E720E0026090E43EC2BF0010EDB2A1E
:1039200060D7DF2ACCD6FE0EDB50006E0A0EE15CBB
:1039300002E2E16AE552E16E0050EFEF22F029EC7D
:103940002CF019E05AEC25F033DE94EC2AF0B2ECBE
:1039500029F003E04CEC26F003D0CE0E006E016A95
:103960004CEC23F00FEC2DF086EC29F06FEC2CF0F2
:10397000F7EC2CF009D065EC27F01ADE94EC2AF075
:10398000020802E02AEC2EF0010EB7EC27F002E26A
:10399000E16AE552E16E0050EFEF22F0EAEC22F02E
:1039A0000D0EE126FE0EDB500FE00501F3B50CD045
:1039B000B2EC29F003E058EC23F008E1A1EC28F088
:1039C00003E058EC23F002E1000E03D2E2EC14F025
:1039D0006EEC23F0F1EC2AF004E056EC25F020091F
:1039E00001D0000E4CEC28F0DB5009E0010EE76E30
:1039F000EDEC2BF0E750D9EC23F0200901D0000EBC
:103A0000E76E050EE7CFDBFF040EDB50760A01E11F
:103A1000F4D0020A0FE0060A01E0C7D101EC15F06C
:103A20000901150EFC6FE20EFD6F000EFE6F54ECE7
:103A30003EF0CED1060EDB6827EC28F009EC2CF026
:103A400038EC2CF002E64DEC2BF030E298EC22F052
:103A5000EF50006E016AD950080FD5EC27F098ECB2
:103A600022F0EE52EFCF00F0060EDB50005C06E2D3
:103A700098EC22F0EE52060EEFCFDBFF98EC22F02E
:103A8000020EA2EC25F0070EDB50D880005408E2AD
:103A900098EC22F0020EC3EC29F0070EEFCFDBFF0B
:103AA000020EDB2A030ECCE3DB2ACAD7080EDBCFDB
:103AB00028F0090EF3EC23F035EC28F0FAEC25F0B1
:103AC000050EDB5064081CE100016DAF03D035EC3E
:103AD00025F004D06CAF04D03BEC25F039EC2DF090
:103AE00000017151E66EE66A89EC2AF0E66EA6ECFA
:103AF0002CF07FEC2CF03CEC29F0E7EC26F024D005
:103B00000EEC28F0E7EC2BF0120EE66EE20EE66EFD
:103B1000000EA1EC2BF0060E8FEC2AF00E0EE66ED6
:103B2000E20EE66E000EA1EC2BF0070E8FEC2AF0F1
:103B30000A0EE66EE20EE66E000EA1EC2BF0060E0B
:103B4000E66EE20EE66E000E3DEC2DF0DB6A030E33
:103B5000DB6A38EC2CF002E64DEC2BF001E322D1CD
:103B6000010EF36E020EDB5004E0D890F336E80647
:103B7000FCE1F35000016D1503E035EC25F00FD0AA
:103B8000010EF36E020EDB5004E0D890F336E80627
:103B9000FCE1F35000016C1504E03BEC25F039EC3E
:103BA0002DF0C7EC29F015E148EC2BF000340AE2C7
:103BB00048EC2BF0016A00BE01684CEC23F0E1EC0C
:103BC00026F010D048EC2BF0016A00AE07D0016857
:103BD00005D098EC22F0EF504AEC24F04CEC23F0A6
:103BE0005BEC26F0A1EC2BF0E7EC26F03DEC2DF0A1
:103BF000DB2A030EAEE3DB2AACD7FAEC25F0DE6A53
:103C0000DD6A72EC2AF002E651EC28F001E3CAD03A
:103C1000050EDB5064081FE115EC29F0080E4FEC8F
:103C20002BF003E035EC25F008D015EC29F0060E5A
:103C30004FEC2BF004E03BEC25F039EC2DF015ECCB
:103C400029F00F0E26EC29F089EC2AF0A1EC2BF0DC
:103C5000DBEC26F011D0020EE66EE66A15EC29F0D8
:103C6000B8EC2CF00A0E1CEC2BF0120EE66EE20EF5
:103C7000E66E000EFEEC24F03DEC2DF0DB6A030E48
:103C8000DB6A38EC2CF002E632EC2CF001E384D055
:103C90000B0EDBCF00F00C0EDBCF01F0A00E026E9E
:103CA000060E036E0D0E025E000E035A03EC26F0A4
:103CB00009E28DEC29F01DEC59F01E0E1CEC2CF0E5
:103CC000FAEC25F015EC29F0080E77EC2AF0020E3C
:103CD000DB501F0B03E0B1EC24F0FDE160EC23F0BE
:103CE00003E035EC25F011D015EC29F0060E77EC49
:103CF0002AF0020EDB501F0B03E0B1EC24F0FDE1D3
:103D000060EC23F004E03BEC25F039EC2DF0C7EC3F
:103D100029F029E1FDEC29F0C1EC22F0FDE1EBEC0A
:103D20002CF08EEC22F00001800E01140CE1FDEC71
:103D300029F0C1EC22F0FDE1EBEC2CF026EC29F0AF
:103D4000E1EC26F00BD0FDEC29F0C1EC22F0FDE116
:103D5000EBEC2CF026EC29F05BEC26F0A1EC2BF040
:103D6000DBEC26F011D0030EE66EE66AFDEC29F0DE
:103D7000C1EC22F0FDE102EC29F0050E1CEC2BF069
:103D80005BEC26F0FEEC24F03DEC2DF0DB2A030E7C
:103D900001E277D7DB2A75D7DF2A010E01E231D79E
:103DA000DB2A2FD78DEC29F013D00601006B010E12
:103DB000E66EE66A000EE66ECFEC27F020EC2CF003
:103DC0008DEC29F068C06AF069C06BF06DC06EF0D0
:103DD000010E006E0D0EE15C02E2E16AE552E16E59
:103DE0000050EFEF22F0EAEC22F0FC0EDBCF28F0DF
:103DF000FD0EDBCF29F0CF0E281801E1295040E05D
:103E0000D00E281801E129503BE0CD0E281801E121
:103E1000295033E0CE0E281801E129502EE0CB0EB8
:103E2000281801E1295025E0CC0E281801E129507D
:103E300020E0C90E281801E1295017E0CA0E281801
:103E400001E1295012E0C80E281801E1295009E0CB
:103E5000060E28181BE1295019E19EDBB9EC11F080
:103E600012D09ADB46EC0FF00ED096DBE6EC11F0A8
:103E70000AD092DB08EC13F006D08EDB60DD03D0B5
:103E80008BDB89EC0EF07BEC2AF001D0000EA7D37F
:103E9000A1DB030EE126DE6ADD6A51EC24F004BEEC
:103EA0000568040EEDEC26F0FDE163EC24F001E181
:103EB000E3D0840E066E3E0E076E010E086EDECF56
:103EC00009F0DDCF0AF00B6A0ABE0B68040ED89029
:103ED00009360A360B36E806FAE106500924036E65
:103EE00007500A20046E08500B20056E03C0E6FF41
:103EF00004C0E6FFE66EB1EC98F094EC2AF09CEC7E
:103F00002DF00006000E015A025AC6DB840E0F6E19
:103F10003E0E106E010E116EDECF12F0DDCF13F0EB
:103F2000146A13BE1468040ED89012361336143671
:103F3000E806FAE10F5012240C6E105013200D6E9B
:103F4000115014200E6E0C2A000E0D220E220CC0F1
:103F5000E6FF0DC0E6FF0EC0E6FFF90EDBCFE6FF81
:103F6000FA0EDBCFE6FF91EC97F0156E070EE15EDF
:103F70001550000901E07AD0FE0EDB5030E0F70E5C
:103F8000DBCFE6FFF80EDBCFE6FF27EC5AF0E55279
:103F9000E552F70EF3CFDBFFF80EBBEC27F0F70F7F
:103FA000E66EFF0EDA20E66EFB0EDBCFE6FFFC0EC0
:103FB000DBCFE6FF51EC24F004BE0568040EEDEC07
:103FC00026F0FDE163EC24F0E66E03EC61F0066E92
:103FD000050EE15E0650000902E1000E4ED0DECF74
:103FE000E9FFDDCFEAFF030EEA02F3CFEAFFE902C1
:103FF000F3CFE9FFF450EA26E40EE9260A0EEA229E
:10400000EECF00F0EECF01F0EFCF02F0F70EDBCFF6
:10401000E6FFF80EDBCFE6FFF90EDBCFE6FFFA0E88
:10402000DBCFE6FFFB0EDBCFE6FFFC0EDBCFE6FFD0
:10403000FD0EDBCFE6FF06D002C0FBFF01C0FAFF9A
:104040000050F96EF9DF036E070EE15E0350E76E74
:10405000020EE7CFDBFFFD0EDB5005E0020EDB506A
:1040600002E01DEC59F0020EDB5007D0DF2A010EF2
:1040700001E213D7DB2A11D7000E006E030EE15CBC
:1040800002E2E16AE552E16E0050A9D2A3DABFEC88
:1040900024F082DAE66A84EF2BF09CDAF90EDBCFAB
:1040A000E6FF7ADA010EE66EE66E84EF2BF029EC7D
:1040B0002CF003E10501F3A502D0000E3AD009016E
:1040C000F00EFC6FE10EFD6F000EFE6F54EC3EF043
:1040D000DE6ADD6AE6DB04BE0568040EEDEC26F060
:1040E000FDE1F1DB25E00901EE0EFC6FE10EFD6F55
:1040F000000EFE6F54EC3EF0D4DB04BE0568040EE7
:10410000EDEC26F0FDE1005003240901FC6F0150A5
:104110000420FD6F02500520FE6FFC2B000EFD23D6
:10412000FE2354EC3EF0DF2A010ED4E3DB2AD2D783
:10413000010EB7EC27F002E2E16AE552E16E0050B1
:104140004ED248DAE652520E0501C85D06E1540E21
:10415000C95D03E1CA5101E178D0520EC86F540E17
:10416000C96FCA6BCB6BCC6B0901400E176F880E01
:10417000036F130E046F100E056F270E066F096B89
:104180000A6B0901320EA06F0901006B0B6F0C6BFB
:10419000640E076F086B016B026B0D6B0E6B156B7A
:1041A000166B0F6B106B116B126B136B146B120E83
:1041B00075EC26F0600EE66E000E60DB0001E80E86
:1041C000626F030E636F1C0E75EC26F0720EE66EC6
:1041D000000E54DBDF6A070EDF5C0BE2DF50EED926
:1041E000280EEF6EDF50EAD9EE52F00EEF6EDF2AA6
:1041F000F2D7700E75EC26F08E0EE66E000E3EDBEA
:10420000DF6A0E0EDF5C0EE2DF50080DC1EC2CF011
:10421000D4EC2DF0C3EC29F0D00EEE6E070EED6E4F
:10422000DF2AEFD798EC2AF03E6B3F6BA3EC2AF025
:104230008AEC25F0186B0901A56BA66BA76BA86B20
:104240000901A96BAA6BAB6BAC6B0001FE6B900E06
:104250006F6E6EAEFED7606A0F011869E00E196FBF
:104260002A0E006FA00E016F046B056B506BFE0EE3
:104270001C6F1D6BB20E086F096BD20E0C6F0D6BAD
:10428000AA0E106F116BBA0E146F156B706ABF0E09
:10429000716E020E726E200E736E0501F4510008ED
:1042A00002E26F6A02D0600E6F6E07018E0ECC6F55
:1042B0003C0ECD6F010ECE6F0701940ECF6F3C0EFA
:1042C000D06F010ED16F0701380ED56F040ED66F77
:1042D000000ED76F0701C80ED86F060ED96F000EFB
:1042E000DA6F0701F00EF06F0E0EF16F000EF26F35
:1042F0000701F40EDB6F0E0EDC6F000EDD6F0701A1
:10430000D80EDE6F130EDF6F000EE06F0701F20EA6
:10431000E16F130EE26F000EE36F0B018C0E4C6F1A
:10432000400E4D6F000E4E6F0B019A0E4F6F400EF8
:10433000506F000E516F0B01E60E496F3D0E4A6F34
:10434000000E4B6F0601EE81EE83EE85010EE55205
:1043500046D1F20E00262B0EFBEC2BF0E40E2B6E5A
:10436000570E2C6E93EC28F0B3EF2CF067EC2CF08A
:1043700016EC75F0086E090E24EC2BF058EC2AF0C0
:104380009FEC2CF004C026F078EC29F0040EDBCF73
:104390002BF0050EDBCF2CF0060EDBCF2DF0070E39
:1043A000DBCF2EF0E3EC2DF024EC2CF054EC2DF0D0
:1043B000420EE66EE40EE66E000E67EC2CF007ECA3
:1043C00075F0086E070E24EC2BF0400EE66EE40E3E
:1043D000E66E000E120080EC28F0E66EE3EC2AF0A8
:1043E00086EC29F08CEF2BF0E7EC2DF06CEF2DF044
:1043F000120EEA02F3CFEAFFE902F3CFE9FFF4502D
:10440000EA26600EE926000EEA22120080EC28F06F
:1044100004EC2AF0DEEF2CF09DEC28F0BFEF28F042
:1044200067EC2CF024EC75F0046E090E0FEF2BF006
:10443000DAEC28F0D950040F37EF2AF0E66EE3ECFF
:104440002AF07FEC2CF08CEF2BF0D8EC74F07BEFA3
:104450002AF0DECFE9FFDDCFEAFF1200DF50120DB8
:10446000C1EC2CF0600EE926000EEA2212000102D7
:10447000F3CF01F00002F3CF00F0F4500126120058
:104480002F6ECBEC2DF04BEC2AF0140EDBCF2CF082
:10449000150EDBCF2DF0160EDBCF2EF0170EDBCF77
:1044A0002FF0A8EC83F06BEC29F0BEEC82F0100E3C
:1044B00027C0DBFF110E28C0DBFF120E29C0DBFF77
:1044C000130E2AC0DBFFD950100FBDEC2CF0EECF3D
:1044D000E6FFEECFE6FFEECFE6FFEFCFE6FF70ECB4
:1044E00095F094EC2AF0E55249EC2CF033EC2BF0EB
:1044F00026C027F0BFEC2AF0020E28C0DBFF030E17
:1045000029C0DBFFD950020F21EF2AF055EC2CF027
:1045100067EC75F0006E070E38EF29F0C3EC29F058
:10452000B8EF2CF0A6EC2CF086EC29F03CEF29F04B
:10453000FDEC29F0A3EC2DF0B5EF28F0E96EFF0EAD
:10454000DA20EA6EEE50ED10120007C928F008C913
:1045500029F08EEC82F01DEC29F005C928F006C97F
:1045600029F04DEC29F0CBEF2DF055EC2CF086EC3A
:1045700029F06FEF2CF004EC2AF0046E090ECBEF5B
:104580002AF0D890E936EA36E8061200F0ECA7F0F7
:1045900022C000F0F4EF2BF0F6EC29F0EFEC29F05C
:1045A000FE0EDBCFE6FF1200E66EC6EF2BF0040E28
:1045B000DBCF00F0050EDBCF01F01200040DC1ECE3
:1045C0002CF0B5EF28F0060EF3CFDBFF070EF4CF8B
:1045D000DBFF1200D9CFE6FFE1CFD9FF1200E55291
:1045E000E7CFD9FF12008E0EE926000EEA22120054
:1045F000BFEC2BF090EC82F01DEC29F00EEC2CF0CF
:104600004DEC29F0A8EC83F0BAEC28F08DEC2BF0FF
:1046100055EC83F044EC85F028C0A1F929C0A2F93B
:104620001200B6EC29F059ECA8F0050E2626000E73
:1046300027222822292267EF2BF0000EE66E060EB5
:10464000E66E1200F0C504F0056A066A076A100EED
:104650002B6E270E2C6E2D6A2E6AF0C526F078EC94
:1046600029F008C02BF0EAEC2AF055EC84F026C0C3
:1046700002F027C003F0B6EC2DF052EC00F01DEF75
:104680002AF042EC2AF0CAEC2CF0020EF626000EBC
:10469000F722F8220800120000C0E6FF01C0E6FF82
:1046A0001200020EDBCF00F0030EDBCF01F0120090
:1046B000FC0EDBCFE9FFFD0EDBCFEAFFEF5012006F
:1046C0000450001605500116065002160750031636
:1046D00013EF2CF0D950150F37EF2AF0EFEC29F03B
:1046E000F6EC58F0E552E5521200060EDBCF00F072
:1046F000070EDBCF01F01200E6EC2CF007C027F02C
:1047000008C028F009C029F0D4EC84F024C007F0D8
:1047100025C008F026C009F004502424F36E05508B
:104720002520F46E06502620A7EC29F00800F5CFCE
:1047300002F002C003F0026AA00E0A6E3C0E0B6E7D
:10474000010E0C6EE2CA0DF0E3CA0EF00F6A120001
:10475000100EE66E270EE66E52EC00F01DEC2AF00D
:104760003DEF2CF001C029F0CEECA8F028C000F0FD
:1047700029C001F01200E6EC2CF00DC027F00EC0AD
:1047800028F00FC029F0D4EC84F024C00DF025C02F
:104790000EF026C00FF00A502424F36E0B50252093
:1047A000F46E0C502620A7EC29F0A4EC2BF0CFEFF0
:1047B0002AF0C3EC29F0EF501200066A076A9BEC5E
:1047C0002CF008C02BF0EAEC2AF0F0ECA7F0F4ECA7
:1047D0002BF0D9500C0FBDEC2CF0225095EC2BF0A7
:1047E000DF2A010E1200DBCF29F090EC82F01DECE5
:1047F00029F02C6A2D6AE00E2E6E400E2F6ECBEC47
:104800002DF033EC2BF0BFEC82F044EF85F0002666
:10481000000E012254EC2DF0B3EF2CF0020EDBCF92
:10482000E6FF030EDBCFE6FF120058EC2AF09BEC0C
:104830002CF0A3EC82F0BAEC28F02C6A2D6A12005E
:104840000C0EDBCF08F00D0EDBCF09F00E0EDBCF28
:104850000AF00F0EDBCF0BF008C026F0ABEC2BF00C
:10486000A3EC82F01DEC29F02C6A2D6A120045ECB5
:104870002DF0E76EFE0EE7CFDBFF1200E66EDBECFD
:1048800097F07BEF2AF0040E00C0DBFF050E01C09D
:10489000DBFF1200006E016A280E005E000E015A56
:1048A0001200840E006E3E0E016E010E026EDECF0F
:1048B00003F0DDCF04F0056A120055EC2CF0B1ECEA
:1048C0002DF0CBEF2AF000500324F36E01500420AA
:1048D000F46E02500520A7EC29F00800F5501200F4
:1048E000DECF00F0DDCF01F01200C3EC29F000C0F4
:1048F000EEFF01C0EDFF1200026A036A010E046EB2
:10490000056A066A076A120003C0DBFF2D0EE96E16
:10491000090EEA6E2151EE24006E2251EE20016E46
:104920002351EE20026E2451EE20036E39510026F1
:104930003A5101223B5102223C51032212002F6EB8
:1049400000C027F0BFEC2AF0DCEC2AF0060E070EC0
:10495000DBCF03F00001800E03141200005095EF2E
:104960002BF0D8900436053606360736E8061200D6
:10497000E66EE66AFEEC3EF0E552E5521200F80EF5
:10498000DBCFE6FFF90EDBCFE6FF1200F3CFE6FF49
:1049900001C0E6FF1200250EE96E090EEA6E09015C
:1049A0001951EE24006E1A51EE20016E1B51EE20BB
:1049B000026E1C51EE20036E31510026325101224D
:1049C00033510222345103221200290EE96E090EDE
:1049D000EA6E1D51EE24006E1E51EE20016E1F5135
:1049E000EE20026E2051EE20036E35510026365126
:1049F000012237510222385103221200E66EA6EC42
:104A00002CF0B1EC2DF0E15E04503CEC29F0030EEB
:104A1000E66EE20EE66E000E120002C0E6FF03C074
:104A2000E6FF12002C6E74EC2CF055EC84F027C0DD
:104A300001F025EC2AF02650EE260150ED2212005E
:104A4000DBCF0AF0030E0926000E0A220B6A005083
:104A50000924F36E01500A20F46E02500B20A7ECDB
:104A600029F00800F550E66E12007B0EE66EE20EAD
:104A7000E66E000E1200790EE66EE20EE66E000E95
:104A80001200CFEC2AF0B2EC2BF0D950010FBDECA4
:104A90002CF0000ED880EE54000EED541200BDEC48
:104AA0002CF0E552E750EE6EED6A1200EDEC2BF0C3
:104AB000EF501200EFEC29F0E66A1200D8900036B1
:104AC000013602360336E8061200FA0EDBCFE9FFA4
:104AD000FB0EDBCFEAFF1200E66ECAEC9FF094EF0C
:104AE0002AF0A3EC3EF0E552E5521200E6EC2CF081
:104AF00006C027F007C028F008C029F0D4EC84F0E5
:104B000003502424006E04502520016E05502620F9
:104B1000026E1200626B636B646B656B666B676B36
:104B2000686B696B1200DFEC89F01DEF2AF0050E4F
:104B3000005E000E015A040E1200C3EC29F0EE5084
:104B4000ED101200C3EC29F0EFCF00F01200D89066
:104B500000360136E8041200080EDB6A090EDB6A33
:104B600013EC2BF00E0EDB6A0F0EDB6ADE6ADD6AD9
:104B700012003D510C0DC1EC2CF0190EE926090E66
:104B8000EA221200000E005E060E015AC4EF2AF05F
:104B9000FD0EDBCF00F0FE0EDBCF01F0120055EC76
:104BA0002CF02FEC99F0026E050EE15E0250CFEC76
:104BB0002DF0F350F4101200E6DBEECF02F0EFCF51
:104BC00003F01200010E006E016A026A036ADF50F0
:104BD0001F0B120051DB020E120041EF2DF0DEEC34
:104BE0002CF0D5C9E6FFD6C9E6FFD7C9E6FFD8C97C
:104BF000E6FF1200D9500B0FBDEC2CF0000EEE6E4C
:104C0000060EED6E12000050025C015003581200B7
:104C1000ADEC2CF0CDC926F0CEC927F0CFC928F0D5
:104C2000D0C929F059EFA8F02F6E55EC83F0140E7F
:104C300027C0DBFF150E28C0DBFF160E29C0DBFFE7
:104C4000170E2AC0DBFF1200FD0EDBCF28F0FE0E90
:104C5000DBCF29F00351285C006E04512958016E06
:104C6000026A036A1200EF51640DCFEC2DF03DECA7
:104C70002CF052EC00F0E552E5521200020E00C09A
:104C8000DBFF030E01C0DBFF1200A00E006E3C0E26
:104C9000016E010E026E1200FC0EDBCF00F0FD0E65
:104CA000DBCF01F0120061DAEFCF00F012006BDB16
:104CB000EE6AED6A1200620EE66EE20EE66E000E1D
:104CC000120000500008000E01541200D89001326A
:104CD0000032E8041200010E0026000E012212002C
:104CE000020EF3CFDBFF030E1200E66EE66AE66A01
:104CF0001200DEEC2CF0DBC9E6FFDCC9E6FF120097
:104D00000FC95CF910C95DF911C95EF912C95FF9E3
:104D1000DBC960F9DCC961F9120097DBEECF00F066
:104D2000EECF01F0EECF02F0EFCF03F01200090159
:104D30005C6B5D6B5E6B5F6B606B616B1200E126A1
:104D4000D9502DEF2BF0A00E046E3C0E056E010E17
:104D5000066EE2CA07F0E3CA08F0096A1200A00E64
:104D6000036E3C0E046E010E056EE2CA06F0E3CA45
:104D700007F0086A120055EC2CF0D8EC74F0036EC2
:104D8000050EE15E035012008DEC2BF0A8EC83F0D1
:104D900044EF85F0EAD9020EF6DA42EF2CF0DB5050
:104DA0003F0B006E3D0E005C1200000ED8800B55CC
:104DB000000E0C551200710EE66EE20EE66E000E4D
:104DC0001200640EE66EE20EE66E000E1200570E42
:104DD000E66EE20EE66E000E1200D8900336043640
:104DE0000536E806120015C900F016C901F0006C7E
:104DF000011E000E0122026A036A1200060E00C0A4
:104E0000DBFF070E01C0DBFF120015C900F016C959
:104E100001F0026A036A1200010EDBCF00F0020EFD
:104E2000DBCF01F012000F0E0B014215016E006A7C
:104E3000435112000F0E0B014515016E006A4651D9
:104E40001200020EDBCF02F0030EDBCF03F01200E4
:104E5000060EDBCF02F0070EDBCF03F012008AEC68
:104E600098F07BEF2AF08FDAEF6A1200DBCFEAFFCF
:104E7000410EE9260B0EEA2242EF2CF09DEC2BF0BE
:104E8000E66EE66AE66EE66A010EE66E1200D5D9B7
:104E9000140E1200D1C9E6FFD2C9E6FFD3C9E6FF5E
:104EA000D4C9E6FF120003C905F904C906F90BC904
:104EB00007F90CC908F912000FC926F010C927F02C
:104EC00011C928F012C929F0120089DA020EE66E23
:104ED00012000FC9E6FF10C9E6FF11C9E6FF12C9AB
:104EE000E6FF12003DEC2CF06CEC01F0E552E552CF
:104EF00012003BD9EE5242EF2CF00B014451006EF0
:104F0000016A040E1200F7DA090112009CEC0DF0A0
:104F100094EF2AF035EC98F094EF2AF03AEC2EF06A
:104F2000FE0EDB50020812001C0EE66EE30EE66E6B
:104F3000000E1200025E000E035A01500318120008
:104F400002500008000E03541200E66EBFEC72F02F
:104F5000E55212000250005C03500158120083EC2D
:104F60009FF0E55212004D0E0701CB5D1200006E5E
:104F7000020EE15C1200F4CFDBFFD9501200010EEB
:104F8000DBCF03F0020EDBCF04F0056A1200010E46
:104F900009010024A36F000E0120A46F1200E66A2D
:104FA00087EC19F0C1DAE5521200BDEC2CF000508C
:104FB000EE260150ED221200E846FE0BF306120029
:104FC000010EDB407F0B12000C0EDBCF02F00D0E4A
:104FD000DBCF03F012000A0EDBCF00F00B0EDBCFAD
:104FE00001F01200030EF3CFDBFF040EF4CFDBFF62
:104FF000120013C900F014C901F0026A036A12001A
:105000000C0EDBCF00F00D0EDBCF01F01200D890BC
:105010000332023201320032E8061200080EDBCF02
:1050200000F0090EDBCF01F01200DFEC89F0E55251
:10503000E552F3CFF1F51200030EDB6A040EDB6AD2
:10504000050EDB6A12004AECA4F07BEF2AF0070E93
:10505000DB6A080EDB6A090EDB6A1200F80EDBCF92
:1050600028F0F90EDBCF29F01200080E28C0DBFF74
:10507000090E29C0DBFF120078D8EFCF08F012002C
:10508000F36E010EDBCFF4FFF350F45C12004151DC
:10509000006E016A040E1200E76E040EE7CFDBFF1C
:1050A0001200010E41EF2DF044C9E6FF45C9E6FFAD
:1050B000120052C9E6FF53C9E6FF1200C6EC74F0B5
:1050C000E552E552120003C9E6FF04C9E6FF1200EB
:1050D00005C9E6FF06C9E6FF120009C9E6FF0AC9CD
:1050E000E6FF1200000EDE6E060EDD6E1200020EEE
:1050F000E126FE0EDB501200090EDB503F081200C5
:10510000FC0EE66EE40EE66E000E1200CEDB25EC21
:1051100022F06FEF2CF0FD0EDBCFE9FFFE0EDBCFB0
:10512000EAFFF8EF21F0E0DBE3EC2DF0B6EF2DF035
:10513000CEDB25EC22F083EF2CF0C9DBE0DB83EF44
:105140002CF0E66A0CDFFC0EF3CFDBFFFD0E13DF65
:10515000FC0F9EEF22F0E66EF9DB25EF22F0D4EC97
:1051600022F025EC22F0E3EF22F0720EE926000E89
:10517000EA2212009CEC2DF02AC003F01200110E5E
:10518000DBCF04F0120EDBCF05F0130EDBCF06F001
:10519000140EDBCF07F0CFDB150EDBCF2BF0160E96
:1051A000DBCF2CF0170EDBCF2DF0180EDBCF2EF05F
:1051B000E3EF2DF0040EDBCF04F0050EDBCF05F09E
:1051C000060EDBCF06F0070EDBCF07F0D950080F35
:1051D000D4DBEE50045C006EEE500558016EEE50CC
:1051E0000658026EEE500758036E110E00C0DBFF2A
:1051F000120E01C0DBFF130E02C0DBFF140E03C052
:10520000DBFF1200F3EC22F0B8EF2CF0A9EC21F058
:10521000D70EE66EE40EE66E000E10EF22F0F2EC12
:105220002DF025EC22F06FEF2CF029EC22F0F8EFB6
:1052300021F029EC22F0A3EF2DF027C004F028C0C4
:1052400005F029C006F02AC007F012008EEC22F00B
:10525000050EC7EF2DF00A0E37EC22F00E0E2D6E64
:105260002E6AF3CF28F0B2EC23F07DDBEBEF21F0D8
:10527000E15E00506FEF2CF00B0EF3CFDBFF0C0E56
:10528000F4CFDBFF1200E66EF4EF21F02C6E2D6AF6
:105290002E6AC6EC22F0A9EF21F08EEC82F027C036
:1052A00008F028C009F029C00AF02AC00BF0C6DBBC
:1052B00004C027F005C028F006C029F007C02AF076
:1052C00012002B6E2C6A10DBC6EF22F0D4EC22F019
:1052D00016DBE3EF22F027C00CF028C00DF029C048
:1052E0000EF02AC00FF0AADB00C027F0AAEF2DF0C5
:1052F000FAEC2DF0F0ECA7F022C004F023C005F08A
:1053000024C006F025C007F027EF2DF007EC75F05C
:10531000026E070EE15E025012001DEC23F071EFE9
:1053200025F0F36E070EF3CFDBFF4E0EE66EE20EB6
:10533000E66E000EF2EC2DF025EC22F0BCD3EBEC87
:1053400021F0010EDB50080D1CDBF3EF22F0F86EAC
:10535000F4CFF7FFF3CFF6FF12000A0E37EC22F07E
:1053600097EF25F0D950FC0F9EEF22F070DBDFCFD6
:105370002BF0010EDBCF2CF0020EDBCF2DF0030E55
:10538000DBCF2EF01200E926000EEA221200010EF9
:10539000E76E51EC23F0E7500026000E01224CECA2
:1053A00023F0E66AE66AE66A92EC22F0050EDB502C
:1053B00064081200DF0EE66EE30EE66E000EF2ECFD
:1053C0002DF02FEF27F04AEC24F04CEC23F096EF71
:1053D0002DF02D6E2E6A00C028F0B2EF23F0FC0EE7
:1053E000DBCFE6FFFD0EDBCFE6FF1200FA0EDBCFD0
:1053F000E6FFFB0EDBCFE6FF1200020EDBCFE9FF7C
:10540000030EDBCFEAFF120050DA24EF75F0A9ECAF
:1054100021F0C20EE66EE40EE66E000E10EF22F0F2
:105420004CEC23F0D70EE66EE30EE66E000EB5EF01
:1054300022F00A0EACDBC3EF2DF0E552E552CFEFC0
:105440002DF09BDAEE50ED101200D9CFE9FFDACF44
:10545000EAFF12008EEC22F0050E0102F3CF01F0FC
:105460000002F45001263CDC01C0DBFF120085DAAB
:10547000D880000EEE54000EEE54000EEE54000ED6
:10548000EE541200A3DA03C027F004C028F005C0D0
:1054900029F0D4EF84F0140EDBCF27F0150EDBCF0C
:1054A00028F0160EDBCF29F0170EDBCF2AF0120002
:1054B000080EDBCF04F0090EDBCF05F00A0EDBCFC0
:1054C00006F00B0EDBCF07F01200E66EE66AD30E95
:1054D000E66EE30EE66E000E1200EAEC22F0020E1B
:1054E000E126120070EC24F0D890015012008EECEE
:1054F00022F07CEF24F0006E050EE15E00501200F9
:10550000026A036AD950080F38DAAEEC24F029EFAA
:1055100022F0750EE66EE20EE66E000E1200DB5013
:105520004AEC24F04CEF23F0E552E552E55212002C
:10553000240E75EC26F0190EE66E090E3EEC24F0F2
:1055400009013D6B12001C0E75EC26F0400EE66E54
:10555000090E3EEC24F097EF26F044C900F045C94F
:1055600001F0026A036AA0DD0DEF25F052C900F0D8
:1055700053C901F0026A036A9CDD0DEF25F0EADAF7
:10558000BFEC82F044EF85F0040EDBCF02F0050E95
:10559000DBCF03F01200E15E04506FEF2CF000014E
:1055A0000224006E000E0320016E120075EC26F03E
:1055B000E66AE66AF4EF21F0060E28C0DBFF070E6C
:1055C00029C0DBFF1200080EDBCFE6FF090EDBCFA0
:1055D000E6FF120009C02CF00AC02DF00BC02EF01F
:1055E0001200D950F80F9EEF22F0D950FA0F9EEF1B
:1055F00022F0010EDB50DEEF22F0A9EC21F09D0E2F
:10560000E66EE40EE66E000E10EF22F0E66EE66A3D
:10561000FE0EE66EE40EE66E000E1EEF22F0E15E78
:10562000045083EF2CF00A0EDB6A0B0EDB6A0C0EC3
:10563000DB6A0D0EDB6A120037EC22F0026A036AA5
:10564000C6EC24F00DEF25F0E15E085083EF2CF05E
:10565000E66A1DEC23F08AEF27F0FC0FE96EFF0EDF
:10566000DA20EA6E12002C6A2D6A2E6A3F0E2F6E27
:105670001200D7EC22F0030EEDEF25F02EEC22F015
:105680000D0ED9EF23F001224CEC23F037EF24F07C
:1056900098EC22F0030EA2EF25F0070EF2D18EEC6B
:1056A00022F00150800B1200C8EC25F009010050D7
:1056B000035D015004591200F8D860EF76F045EC14
:1056C00026F0E2CA03F0E3CA04F0056A120045D9E5
:1056D00059EFA8F0190EE66EE40EE66E000EB6EF76
:1056E00021F0E3D8B3EF75F0E76E65EC25F0E750F5
:1056F000D9EC23F03F081200E3EC22F051EC23F048
:105700000001800E0114120048EC1FF0006E080E1C
:10571000E15E0050EFEF22F0CED12C6A400E2D6EEC
:105720001C0E2E6E460E2F6E1200EE260150EE223B
:105730000250EE220350EE221200000EE66EE66AE0
:105740001200E66E92EF22F0F62A000EF722F822FF
:105750000800F550120009C027F00AC028F00BC05D
:1057600029F01200010E00C0DBFF020E01C0DBFFBA
:10577000120075EC26F09FEC1CF083EF27F0040E6E
:10578000DBCF28F0050EDBCF29F01200060EDBCFB1
:10579000E6FF070EDBCFE6FF120075EC23F0006C8E
:1057A000011E000E01221200D7EC22F021EC27F09E
:1057B00003EF26F0F3EC22F0EECF08F0EFCF09F084
:1057C000120070EC24F06BEC26F04CEF23F0280E66
:1057D000005E000E015A4CEF23F0F80EDBCFE9FF1C
:1057E000F90EDBCFEAFF120023C001F024C002F063
:1057F00025C003F012000122000E02220322120033
:105800004CEC23F00DEF25F0EAEC22F0050EE1263A
:105810001200020EDB6A030EDB6A120003C928F0D5
:1058200004C929F0120000500110021003101200E8
:10583000C6EC22F011EF23F0A5EC27F06EEF23F079
:105840001DEC23F05EEF28F0050E0026000E01226D
:105850001200EAEC22F077EF28F070EC26F0F4CF9B
:10586000DBFF12000E0E0DD175EC23F0C2EF25F018
:1058700051EC23F0D89001501200F3CFE6FFF4CFA3
:10588000E6FF1200E552E750EF6E12000C0ED9EF62
:1058900023F026C000F027C001F028C002F029C084
:1058A00003F012002DDC43EF29F0E66EE7EF2DF058
:1058B0000CEC22F0100E2B6E270EE8DC340EE66E98
:1058C000E40EE66E000EB6EC21F098EF28F0E66EDE
:1058D0000F0EDBCFE6FF100EDBCFE6FF1200F3CF9B
:1058E000DEFFF4CFDDFF12002D6A2E6A00C026F025
:1058F00001C027F002C028F003C029F0120007EC15
:1059000075F001EF2EF00F0EF3CFDBFF100EF4CF8A
:10591000DBFF120080EC28F01EEF22F073DC29EC94
:1059200022F0030E1200D90EE66EE30EE66E000EB4
:1059300076DCB2EF29F004C026F0FAEF2DF0E80E85
:105940002B6E030E2C6E2D6A2E6A12000B0EDBCF0F
:10595000E6FF0C0EDBCFE6FF12000A0E2B6E2C6A60
:105960002D6A2E6A120028C0E6FF29C0E6FF120049
:10597000EECF00F0EFCF01F01200E96EDACFEAFFD0
:105980001200F3CFE9FFF4CFEAFF1200DBCFE6FF0E
:10599000E66A120000502424F36E01502520F46EB4
:1059A00002502620A7EF29F0320E0901016A0D25C9
:1059B000006E0E510122640EE9EF29F0006E090E0F
:1059C00038EF29F080EC28F0BBEF22F00B0E2C6EA4
:1059D0002D6A2E6A1200F3EC22F0060E12000CEC77
:1059E00022F0E80E2B6E030E51DC6AEF2BF0E70E6F
:1059F000E66EE30EE66E000E86EC28F03AEF2EF02F
:105A000021C900F022C901F023C902F024C903F022
:105A1000120016DF020E10DF80DC010E1200EA0E0B
:105A2000E66EE30EE66E000EF2EF2DF019EC29F0B3
:105A3000B5EC28F0EF50E66E19EF29F027C02CF0F6
:105A400028C02DF029C02EF02AC02FF0120022C04D
:105A500026F023C027F024C028F025C029F012002A
:105A60008BEC28F00D0ED9EF23F033EC27F015EF77
:105A700029F0ABEC28F03CEF29F0ABEC28F0EAEF92
:105A800025F0005C000E01581200FE0EDBCFE6FF91
:105A900034EC2FF094EF2AF0B5EC28F0EF50E66EDE
:105AA00029EC22F0020E1200022203220A0E2B6EB3
:105AB0002C6A93EF28F0080EF3CFDBFF090EF4CF2A
:105AC000DBFF1200B5EC28F0030E12000BC900F04A
:105AD0000CC901F0ADEF29F007EC75F0006E070E70
:105AE00038EF29F0E66EE66A80EC28F086EF22F0C7
:105AF000B5EC22F094EC27F086EF28F0BEEC82F0B3
:105B0000BAEC28F029EF22F066EC29F0DBEC26F065
:105B1000AFEF28F0D4EC22F086EC29F07CEF2BF0EC
:105B200066EC29F0E7EC26F0AFEF28F0EBEC21F083
:105B3000E0EC27F0DEEF22F027C000F028C001F0F3
:105B400029C002F01200D890E936EA36D890E9363A
:105B5000EA36120001C028F002C029F003C02AF082
:105B60001200F9EC75F0046E0B0E120026C0E6FF71
:105B700027C0E6FF120057EC26F015EF29F08BEC5A
:105B800028F046EF2CF0EBEC21F02EEF22F037EC72
:105B900022F0C6EF24F055EC83F0BAEF28F0F3CFF3
:105BA00000F0F4CF01F01200F3EC22F0020E12002C
:105BB000E66EE66A52EF2CF0060EE8DEABDE070E6C
:105BC000E5DE8AEF2CF059ECA8F049EF2CF0DECF9F
:105BD000E6FFDDCFE6FF120037DE0A0EE9EC29F022
:105BE000B3EF2CF0E66E1DEF23F015EC29F0C0DECC
:105BF00015EF29F005C027F006C028F007C029F0EE
:0C5C00001200006E070EE15E0050120062
:045C0C000A019E6B80
:105C10009F6B12000A015D6B12007F0E0601C85DCA
:105C200008E10901660EFC6FDD0EFD6F000EB2EF9C
:105C30003AF00A01010E5E6F050EE1EC3BF009013E
:105C40005A0EFC6FDD0EFD6F000EB2EC3AF00A0E3C
:105C5000E1EF3BF07F0E0601C85D04E10901FAECBB
:105C60003AF006D00901550EFC6FDD0EFD6F000EF7
:105C7000B2EF3AF07DEC3CF07F0E0601C85D05E125
:105C800078EC3BF0A3EC3EF05AD00A018D0549E1D7
:105C9000450E0601055D45E0410E055D42E0610EE1
:105CA000055D3FE0670E055D3CE0500E055D39E0A7
:105CB000020E05C6DBFF060EE66E060EE66E000E51
:105CC000E66E050E14EC3BF0DCEC39F019EC3AF022
:105CD00002E600EC3BF005E2EFEC3BF0F7E3DB2AF9
:105CE000F5D7000EE66E050EE66EEAEC3CF0000E0F
:105CF000E66E050E6CEC39F04D0EE66EDD0EE66ECE
:105D0000000E5FEC39F0020EDBCF07F6080EE66EF0
:105D1000060E00EC3DF0000EE66E050EE66E2BEC76
:105D20003BF078EC3BF0EAEC3CF013EC3AF06CEC36
:105D30003BF078EC3BF0D6EC90F0E552E552E552C2
:105D4000E5520901FAEC3AF0B2EC3AF0030EE15CEC
:105D500002E2E16AE552E16E68EF39F063EC39F096
:105D6000050EE126D650016E006A030E00C0DBFF6F
:105D7000040E01C0DBFFD75092EC3AF0DF6A080E48
:105D8000DF5C0BE2DF50EA6A410FE96E0B0EEA229C
:105D9000EF5092EC3AF0DF2AF2D7030EDBCFE6FFAA
:105DA000040EDBCFE6FF6EEC8CF0E552E552DF6AC5
:105DB000160EDF5C11E26EEC39F004BE05682CECC7
:105DC0003AF0DF50EA6A5F0FE96E0A0EEA22E55206
:105DD000E750EF6EDF2AECD70A01756B090E27EC4E
:105DE0003CF0CAEC39F0D80EE66E040EE66ECEEC4E
:105DF00039F0F7EC3CF0CEEC39F0160EE66EE66AC0
:105E000005EC3BF074ECA1F0026E0A0EE15E02506C
:105E10000901450EFC6FDD0EFD6F000EB2EC3AF08D
:105E200005EC3BF084EC3AF03DEC3CF024EC3AF02D
:105E3000D6EC90F02CEC3CF009013DEC3CF0080E67
:105E400027EC3CF0CAEC39F0CEEC39F084EC3AF0B7
:105E5000FAEC3AF0B2EC3AF0050EE15C02E2E16AEB
:105E6000E552E16E68EF39F0CEEC3BF078EC3BF0B8
:105E7000F7EC3CF078EC3BF076EC74F0E552E55250
:105E8000C6EC39F0FE0EDB50020A11E0030A03E013
:105E9000010A1EE109D07AEC3AF032EC3BF003E162
:105EA000DE52DD50011814E011EC3CF011D07AEC18
:105EB0003AF032EC3BF003E1DE52DD50011808E02D
:105EC000ACDE11EC3CF0010EF36EFE0EF3CFDBFF07
:105ED000FE0EDB50006E020EE15C02E2E16AE5526A
:105EE000E16E005068EF39F081EC3CF0020E27ECD7
:105EF0003CF0E1EC3AF03C0EE66EDD0EE66E000E94
:105F000025EC39F082EC3BF06CEC3BF066EC3BF0BE
:105F1000E66E020EDBCFE6FF030EE4EC3AF082EC15
:105F20003BF08EC9E6FF8FC9E6FFFCEC38F00901B3
:105F30009051E6EC3BF0090194510F0A20E0020A6F
:105F400018E0090A10E0060A08E0030A1EE1300E14
:105F5000E66EDD0EE66E000E1DD0280EE66EDD0E3E
:105F6000E66E000E17D0220EE66EDD0EE66E000E17
:105F700011D0190EE66EDD0EE66E000E0BD0100E7F
:105F8000E66EDD0EE66E000E05D0070EE66EDD0E47
:105F9000E66E000E04EC3AF009019651040A18E08E
:105FA000070A10E0020A08E0010A18E1FD0EE66E99
:105FB000DC0EE66E000E14D0F40EE66EDC0EE66E1D
:105FC000000E0ED0ED0EE66EDC0EE66E000E08D072
:105FD000E00EE66EDC0EE66E000E02D066EC3BF0E4
:105FE00004EC3AF0FEEC39F04D080FE1A1C9E6FFF0
:105FF000A2C9E6FFFCEC38F0A3C9E6FFA4C9E6FF9E
:10600000B6EC3CF089EC3BF01AD0A1C900F0A2C973
:1060100001F0040E0AEC3BF0FDE12BEC39F041EC11
:1060200039F082EC3BF0A3C900F0A4C901F0040EE2
:106030000AEC3BF0FDE12BEC39F041EC39F082EC5D
:106040003BF009019151E6EC3BF092C9E6FF93C9A0
:10605000E6FFFCEC38F009019751E6EC3BF0090152
:106060009851E6EC3BF009019551E6EC3BF0090153
:106070009451E6EC3BF009019651E6EC3BF0DDC9AA
:1060800000F0016A00BE0168EFEC3CF0DEC9E6FFFB
:10609000DFC9E6FFFCEC38F0E5C900F0016A00BE9C
:1060A0000168EFEC3CF05DEC3AF0B6EC3CF0C0EC93
:1060B0003AF082EC3BF08E0EE66E0A0E48EC39F0B8
:1060C000040EE15C02E2E16AE552E16E005068EF25
:1060D00039F0CEEC3BF0E8EC3AF0D90EE66EDC0E8F
:1060E000E66E000EBAEC3CF099EC39F09AEC3CF01C
:1060F00000BE016814EC39F0900EE66E0A0E85ECD5
:106100003CF002E2E16AE552E16E005068EF39F0DE
:1061100063EC39F0070EE126D20EE66EDC0EE66E79
:10612000000EFBEC39F0CAEC39F0DF6A040EDF5CDC
:106130006FE239EC3BF0EFCF00F0000EE76E001895
:10614000E8AE02D0003403D0E750D880005452E2C9
:10615000DF50EA6AC70FE96E090EEA22EFCF04F0BA
:1061600004C029F07DEC82F027C000F028C001F0C7
:1061700029C002F02AC003F0560E2C6E0E0E2D6EB2
:106180008D0E2E6E3E0E2F6E55EC83F073EC85F067
:10619000030E26C0DBFF040E27C0DBFF050E28C060
:1061A000DBFF060E29C0DBFF010EE66EE66AD95062
:1061B000030F9CEC3AF0E66AE66AE66ACEEC39F048
:1061C000F9EC75F0006E0B0EE15E0050CAEC39F090
:1061D00039EC3BF0EF50D80F006E016A00BE016849
:1061E000EAEC3BF066EC3BF0E66EF3EC3CF066EC80
:1061F0003BF005D0CD0EE66EDC0EE66E000EE66ED0
:10620000CEEC39F0CBEC3BF0CAEC39F0DF2A8ED77C
:10621000E4C900F0016A00BE0168EAEC3BF0E66AFE
:10622000E66AE66AF3EC3CF0920EE66E0A0E48EC83
:1062300039F0070EE15C02E2E16AE552E16E0050DE
:1062400068EF39F07DEC3CF0010EF36E020EF3CFF7
:10625000DBFFF36EDB6EB5EC3AF0C60EE66EDC0EDD
:10626000E66E000EDFEC3CF00F0EF66E000EF76EE1
:10627000000ED8EC39F0100EF66E000EF76E000E20
:10628000D8EC39F009EC3AF06CEC3BF040EC3BF028
:106290007DEC3BF0020E19EC3CF000EC3DF0FAEC2A
:1062A0003CF0AE0EE66E090E94EC39F00901E951AE
:1062B000ACEC3BF00501F451ACEC3BF0C80EE66EE3
:1062C000050E94EC39F0EC0EE66E090E94EC39F004
:1062D000940EE66E0A0E48EC39F0030EE15C02E221
:1062E000E16AE552E16E005068EF39F063EC39F095
:1062F000060EE1260901A951AA11AB11AC1109E161
:10630000020EDB6A030EDB6A040EDB6A050EDB6A33
:106310001DD0A90EE96E090EEA6EEE500901A55DC9
:10632000006EEE50A659016EEE50A759026EEE5067
:10633000A859036E020E00C0DBFF030E01C0DBFF95
:10634000040E02C0DBFF050E03C0DBFF09019951FB
:10635000E66EE66AB80EE66EDC0EE66E000EDFEC68
:106360003CF009019A51ACEC3BF009019E51ACECB8
:106370003BF0C0C900F0016A00BE016814EC39F0BE
:106380000901C151ACEC3BF0C2C900F0016A00BE8A
:10639000016814EC39F0CBC9E6FFCCC9E6FFF9EC93
:1063A00038F0CDC9E6FFCEC9E6FFCFC9E6FFD0C9B8
:1063B000E6FFF6EC39F009019F51ACEC3BF0D95007
:1063C000020F9CEC3AF0F6EC39F0ADC900F0016A2E
:1063D00000BE016814EC39F009019B51ACEC3BF0B4
:1063E000E2C900F0016A00BE016814EC39F0E1C9AD
:1063F00000F0016A00BE016814EC39F0A9EC39F034
:1064000066EC3BF0B6EC39F009019C51ACEC3BF08A
:106410003DEC3AF066EC3BF0B6EC39F009019D51E9
:10642000ACEC3BF0960EE66E0A0E48EC39F0060E28
:10643000E15C02E2E16AE552E16E005068EF39F09A
:10644000CEEC3BF0B10EE66EDC0EE66E000EFBEC21
:1064500039F07DEC3BF00701CF51D011D11116E09E
:10646000CFC7F6FFD0C7F7FFD1C7F8FF0800F55038
:106470000DE0CFC7E6FFD0C7E6FFD1C7E6FF44EC8B
:1064800039F066EC3BF0E66E44EC39F0A10EE66EB6
:10649000DC0EE66E000EE66E44EC39F09C0EE66E05
:1064A0000A0E85EC3CF002E2E16AE552E16E005032
:1064B00068EF39F0CEEC3BF047EC3BF09A0EE66E1D
:1064C000DC0EE66E000EBAEC3CF0FFEC3BF0E1ECCB
:1064D0003AF0F9EC38F009019F51ACEC3BF09AEC42
:1064E0003CF000BE016814EC39F0E8EC3AF0B0EC96
:1064F0003CF099EC39F0FD0EDB0404E1980EE66EF9
:106500000A0E03D09A0EE66E0A0E85EC3CF002E20B
:10651000E16AE552E16E005068EF39F063EC39F062
:10652000090EE126010EF36E080EF3CFDBFF020E1B
:10653000F36E080EF3CFDBFFC7EC3AF0EE50ED1030
:1065400001E138D1FD0EDBCFDEFFDBCFDDFFFEEC5E
:1065500039F009E0FEEC39F0200805E0DF2A010EF1
:10656000F6E3DB2AF4D7FEEC39F0200801E022D173
:106570004EEC3BF001E3DB2AEF6A1EEC39F005EC50
:106580003BF019EC3BF001E115D1090EE66EE7ECAA
:1065900039F0D80EE66E040E5AEC39F01EEC39F0E4
:1065A000ECEC39F01EEC39F0CEEC3AF078EC3BF044
:1065B00024EC3AF02BEC3BF078EC3BF06CEC3BF04D
:1065C00019EC3BF001E0F6D01EEC39F0000EE66E5F
:1065D000060E14EC3BF005EC3BF0C1EC39F0D80EA4
:1065E000E66E040E5AEC39F078EC3BF0ECEC39F046
:1065F00078EC3BF0CEEC3AF024EC3AF044EC3CF092
:10660000A6EC3AF068EC3AF002E600EC3BF00AE265
:10661000D4EC3CF016EC3AF0060EDB2A070EF2E35F
:10662000DB2AF0D724EC3AF04CEC3CF0A6EC3AF044
:1066300068EC3AF002E600EC3BF00AE2D4EC3CF005
:1066400013EC3AF0060EDB2A070EF2E3DB2AF0D752
:106650000A01010E5D6F0A0EE66EE7EC39F028ECD8
:1066600039F050084EE10A018D5127E1060EDB6A30
:10667000070EDB6A68EC3AF004E6160E005C000ECA
:10668000015819E26EEC39F004BE05682CEC3AF0C2
:10669000060EDBCFE9FF070EDBCFEAFF760EE92619
:1066A0000A0EEA22E552E750EF6E060EDB2A070ECD
:1066B000E1E3DB2ADFD70A018C6B8D6B920EE66E6D
:1066C000DC0EE66E000E5FEC39F05CEC3BF0C1ECEA
:1066D00039F00DEC2EF04AEC3AF00A01010E8D6F04
:1066E000E66EE7EC39F0E80EE66E040E5AEC39F08F
:1066F0005CEC3BF0ECEC39F05CEC3BF0CEEC3AF0CF
:1067000002D00A018D6B0501F69FB5EC3AF0700ED0
:10671000E66EDC0EE66E000EFDEC3CF00F0EF66E43
:10672000000EF76E000EC0EC3BF019EC39F0100EC5
:10673000F66E000EF76E000EC0EC3BF019EC39F06F
:1067400009EC3AF0DAEC3BF040EC3BF08DEC3BF03E
:106750000701CC51CD11CE110CE0CCC7E6FFCDC75F
:10676000E6FFCEC7E6FFDAEC3BF0CBEC3BF08DEC7E
:106770003BF0080E19EC3CF019EC39F00501F5512D
:10678000ABEC3CF00501F651E66EE66A66EC3BF0D8
:10679000E66EDAEC3BF067EC75F0E2EC3CF08DEC89
:1067A0003BF00501F751ABEC3CF0140ED5EC39F0A1
:1067B0004AEC3AF0090EE15C02E2E16AE552E16E70
:1067C00068EF39F07DEC3CF00A015D511AE1070EEB
:1067D000E66EE66A680EE66EDC0EE66E000EB3EC60
:1067E0003CF01EEC3BF001E0B9D0070EB9EC39F0FB
:1067F00095DEE552E5520601060ED06F0E0ED16F02
:10680000ADD0F7EC3BF078EC3BF01EEC39F070ECDF
:106810003CF06CEC3BF016EC3AF0050EE66EE66AE6
:10682000620EE66EDC0EE66E000EBAEC3CF01EEC7C
:106830003BF006E0400EE66EB7EC3FF0E5528ED03E
:10684000D950FD0F96EC3CF0050EEE6E060EED6E87
:106850001DEC3AF0EF50450835E154EC3CF04D08A2
:1068600031E1C7EC3AF0020EEE26000EED22F7EC15
:106870003BF0010EE66E050EE66E010EB9EC39F046
:1068800070EC3CF0DCEC39F019EC3AF002E600EC8C
:106890003BF005E2EFEC3BF0F7E3DB2AF5D76CECDD
:1068A0003BF0010EE66E050E6CEC39F01DEC3AF093
:1068B000EFCF00F5D950FD0F96EC3CF0000EEE6ED8
:1068C000050EED6E0501F6BF03D00501150EF76F3D
:1068D0001DEC3AF0EF50430A37E0190A11E01B0AA9
:1068E0003DE15B0EE66EDC0EE66E000E5FEC39F00D
:1068F0000A015E5133E10DEC2EF03AEC2EF01ED081
:1069000054EC3CF030081DE00901010EE86F0A016B
:106910005E5124E10DEC2EF0E66A74EC2FF0E552A6
:10692000E66A69EC30F0E552E66A88EC30F0E55250
:10693000E66A88DCE552E66AD9DCE5522AEC2EF0FC
:106940000DD00901E86B0AD0010EB9EC39F00ED870
:10695000E552E5520A015E5101E1DBD9030EE15C2B
:1069600002E2E16AE552E16E68EF39F081EC3CF059
:10697000FD0EDBCFDEFFDBCFDDFFFEEC39F009E003
:10698000FEEC39F02C0805E0DF2A010EF6E3DB2AE5
:10699000F4D7FEEC39F02C0805E14EEC3BF001E3B6
:1069A000DB2AEF6A1EEC39F0DFEC89F0E552E552A4
:1069B000F3CF9EFAF4CF9FFADECFA0FADDCFA1FA93
:1069C000040EE15C02E2E16AE552E16E68EF39F043
:1069D00063EC39F0060EE126020EE1EC3BF0310EDD
:1069E0000A019E1901E19F5101E173D1290E9E19FF
:1069F00001E19F5101E15BD1280E9E1901E19F51F8
:106A000001E128D1060E9E1901E19F5101E11ED13D
:106A1000050E9E1901E19F5101E10FD1040E9E194F
:106A200001E19F5101E1C0D0030E9E1901E19F5188
:106A300001E182D0020E9E1901E19F512AE0010E70
:106A40009E1901E19F5102E0000E5AD1DE6ADD6A13
:106A500019EC3AF004E6100E005C000E015801E358
:106A60004ED16CEC3BF0500EE66EDC0EE66E000E86
:106A7000FDEC3CF0100EABEC3CF0F1EC3AF0EF50DA
:106A8000ABEC3CF03AEC2EF0DF2A010EE1E3DB2A1E
:106A9000DFD7D5EC3AF0DCDB09E03AEC3CF006E07D
:106AA000020EDB2A030EF7E3DB2AF5D73AEC3CF0C3
:106AB00001E0BCD08AEC3AF001E3DB2A0AEC3CF0BE
:106AC00001E0AED055EC3BF004E6100E025C000E87
:106AD000035801E3A5D071EC3BF0DFEC89F0E552FF
:106AE000E552F350E66EF1EC3AF0E552E750EF6E06
:106AF00019EC3AF004E6080E005C000E015810E3B1
:106B000071EC3BF089EC3CF0080E005E000E015A7F
:106B1000180E0024E66ECAEC9FF0E552E552E552ED
:106B20000FEC3BF00F0EEE1804E1ED5002E107EC24
:106B300093F0ACEC3AF07FD0DE6ADD6A19EC3AF003
:106B400004E6200E005C000E015801E3D8D0DFCF30
:106B5000E6FFE7EC39F00FEC3BF0090EEE1804E12C
:106B6000ED5002E128EC3BF06CEC3BF0450EE66E9C
:106B7000DC0EE66E000EFDEC3CF0200EABEC3CF0C3
:106B800071EC3BF066EC3BF0E66E040EDBCFE6FF0B
:106B9000050EE4EC3AF08DEC3BF03AEC2EF0DF2AF7
:106BA000010ECCE3DB2ACAD7D5EC3AF051DB09E081
:106BB0003AEC3CF006E0020EDB2A030EF7E3DB2A98
:106BC000F5D73AEC3CF032E18AEC3AF001E3DB2A0B
:106BD0000AEC3CF025E155EC3BF004E6180E025CB3
:106BE000000E03581DE271EC3BF0DFCFE6FFCAEC6C
:106BF0009FF0E552E552E552ACEC3AF001DB0FECC8
:106C00003BF0020EEE1801E1ED5007E00FEC3BF017
:106C10000E0EEE181CE1ED501AE107EC93F017D0C0
:106C20003D0EE66E4E0EE66E010E05D0110EE66EBE
:106C30004E0EE66E010EE4DA0AD0ACEC3AF08EECC1
:106C40003CF0040EE66EB7EC3FF058D063DA3AEC55
:106C50002EF055D0D5EC3AF0FBDA09E03AEC3CF0F6
:106C600006E0020EDB2A030EF7E3DB2AF5D73AEC47
:106C70003CF015E18AEC3AF001E3DB2AEF6ADCEC48
:106C80003AF0F6EC58F0E552E55271EC3BF084EC4A
:106C90003AF0550EFC6FDD0EFD6F000E23D00DECAB
:106CA0002EF0110EE66E4E0EE66E010E21D0090199
:106CB000390EFC6FDC0EFD6F000EB2EC3AF0DCEC2E
:106CC0003AF084EC3AF0330EFC6FDC0EFD6F000EF0
:106CD00009D0DCEC3AF084EC3AF0310EFC6FDC0EBB
:106CE000FD6F000EB2EC3AF0050E5FDBACEC3AF053
:106CF0008EEC3CF0020EE66EBFEC72F0E552010E37
:106D0000006E060EE15C02E2E16AE552E16E0050BF
:106D1000DFD20501F6BF03D00501160EF76F020E94
:106D2000E1EC3BF0280E0A019FAF02D0D89003D0CF
:106D30009E5D000E9F5907E39F3507E29E51310883
:106D4000000E9F5502E20DEC2EF00B0149514A1145
:106D50004B1119E0A0CAE6FFA1CAE6FF9ECAE6FFF2
:106D60009FCAE6FF010EE66E07D04BCBFBFF4ACB76
:106D7000FAFF0B014951F96EF8DF006E050EE15E76
:106D8000005000090AE124DE000907E1AC0EE66EBE
:106D90004E0EE66E010E8EEC3CF02AEC2EF00A014F
:106DA0009E6B9F6BA0CAE9FFA1CAEAFFEF6A1200BF
:106DB0008ADA0A015D512CE05E51000829E3020ED7
:106DC000F4DA290EE66EDC0EE66E000E78DA1E0EA0
:106DD000E66EDC0EE66E000EBAEC3CF092DB2EDACC
:106DE000D0DA150EE66EDC0EE66E000EBAEC3CF064
:106DF00088DBAA0EE76EFB0EDBCFE9FFFC0EDBCFD4
:106E0000EAFF61EC3BF0EF6A47EC3BF0BADA42DBB9
:106E10005FD281EC3CF0020EDB6A030EDB6A0A01F2
:106E20005D516EE0B4DBEE50ED106AE0220EB3EC83
:106E30003CF035EC98F0E552E552E55282EC3BF03F
:106E4000F3CF00F0F4CF01F0F350F41022E0020E83
:106E5000DB2ADBCF00F0030E01E3DB2ADBCF01F0FE
:106E6000FD0E00C0DBFFFE0E01C0DBFFF1D910E01C
:106E7000EFD922080DE03AEC3CF004E103EC3CF0E1
:106E80002E0EEF6E020EDB2A030EF0E3DB2AEED7A6
:106E9000DFDB290EE66EE66A690EE66EDD0EE66E53
:106EA000000EDFEC3CF0D950020F96EC3CF0EE50B7
:106EB000ED100DE0C3D9110EE66EDC0EE66E000E8D
:106EC00000EC3DF001EC75F0006E070E0BD0FA0EF1
:106ED000E66EDB0EE66E000E00EC3DF0D8EC74F0D2
:106EE000006E050EE15E00507DEC3BF00A015E5144
:106EF000000803E2140EE1EC3BF00DEC2EF0CADAD0
:106F0000040EE15C02E2E16AE552E16EE1D1DBD917
:106F1000090199A552D009019651040A18E0070AFF
:106F200010E0020A08E0010A18E1EE0EE66EDB0E40
:106F3000E66E000E11D0E30EE66EDB0EE66E000E7E
:106F40000BD0DA0EE66EDB0EE66E000E05D0CB0E31
:106F5000E66EDB0EE66E000EE7DB090194510F0AC8
:106F600026E0020A1EE0090A16E0060A0EE0030AFD
:106F700006E0710EE66EDB0EE66E000E23D0C20E4A
:106F8000E66EDB0EE66E000E1DD0AC0EE66EDB0E7E
:106F9000E66E000E17D09E0EE66EDB0EE66E000E5D
:106FA00011D0940EE66EDB0EE66E000E0BD0820E54
:106FB000E66EDB0EE66E000E05D0640EE66EDB0EAE
:106FC000E66E000EB1DB4D0E0701CB5D12E1A3C9E9
:106FD000E6FFA4C9E6FF03EC3DF09BDB64D9A1C941
:106FE000E6FFA2C9E6FF0AEC3DF093DB5AEC3CF069
:106FF00019D0A3C900F0A4C901F0040E0BDBFEE117
:107000002AD903EC3DF0A1DB4ED9A1C900F0A2C9F9
:1070100001F0040EFFDAFEE11ED90AEC3DF095DB2B
:1070200061EC3CF081DB91EC3CF0460EE66EDB0E51
:10703000E66E000EB3EC3CF06CDB35D9440EE66E28
:10704000DB0EE66E000E70DB4D0E0701CB5D0EE130
:10705000CDC900F0CEC901F0CFC902F0D0C903F00C
:107060001DDA7EDB8DDA5AEC3CF039D0CDC904F064
:10707000CEC905F0CFC906F0D0C907F00FDA26C097
:1070800004F027C005F028C006F029C007F0040E60
:107090001F0B27DA07E0D890003601360236033698
:1070A000E806F9E1050E0026000E01220222032265
:1070B0000A0E2B6E2C6A2D6A2E6A00C026F001C0C3
:1070C00027F002C028F003C029F059ECA8F048DBF3
:1070D00024EC75F0086E090EE15E0850F2DBB3ECAB
:1070E0003CF0D8EC74F0050EE15EDDD80901F551F5
:1070F000F6110AE0E2D9340EE66EDB0EE66E000E03
:10710000B3EC3CF03DDACFD8F1DB00C0F3FF01C0B7
:10711000F4FFDED043DB55DB290EE66EDC0EE66EB7
:10712000000E69D9EADAD8DAF2DEE552E552020E4B
:10713000E15C02E2E16AE552E16ECAD0E7EC3CF0C4
:10714000120EE66EDB0EE66E000EB9D88FDB02E2A1
:10715000E16AE552E16EBCD0E7EC3CF0E70EE66E8A
:10716000DA0EE66E000EABD881DB02E2E16AE55290
:10717000E16EAED0E7EC3CF0D4DBB70EE66EDA0E93
:10718000E66E000EDFEC3CF0B00EE66EDA0EE66E58
:10719000000EE66E79D86ADB02E2E16AE552E16E42
:1071A00097D0E7EC3CF00701CAA307D0D2D8890EEC
:1071B000E66EDA0EE66E000E06D0CBD8710EE66EE5
:1071C000DA0EE66E000ED6DBDEDB57D9690EE66E10
:1071D000DA0EE66E000ECAD8660EE66EDA0EE66EBF
:1071E000000EE66E51D842DB02E2E16AE552E16E42
:1071F0006FD0B6DBFAEF3CF0B9DB8BDA82EF3BF015
:10720000E66E9ECAE6FF9FCAE6FF070EE66E4E0ECA
:10721000E66E010EAFDB99DA8FDAD8EC74F0036E0C
:10722000050EE15E03501200D5DA9ADB8EDA7DEFAF
:107230003BF0E66EBFDA6DDA8DEF3BF0FD0EDBCF93
:10724000E6FFFE0EDBCFE6FF120094DB89EF3BF09A
:10725000DADAEF501200050E0026000E01220A0EA7
:107260002D6E2E6A00C028F001C029F0CEECA8F0E7
:1072700028C000F029C001F028C0E6FF29C0E6FFC1
:10728000120074DBA5EF3BF027DA85DA7DEF3BF0E7
:10729000E66EFE0EDBCFE6FF34EC2FF0E552E55252
:1072A000E552006E1200FD0EF3CFDBFFFE0EF4CFB1
:1072B000DBFF1200E66E15DA9ADB71EF3BF05ADB6A
:1072C0008AEC98F077D3D9CFE6FFE1CFD9FF12004F
:1072D000E552E7CFD9FF12005EDB64D24E0E006E9E
:1072E0004F0E016E010E026E75DAE66E75EC8CF0D3
:1072F000E552E7CF02F0E552E7CF01F0E552E7CFE4
:1073000000F0F3CF03F0F4CF04F0400E2D6E2E6AA0
:10731000F3CF28F0F4CF29F02FEC84F024C003F051
:1073200025C004F0056A1200E66E1ADB68DA7DEF0C
:107330003BF060EC76F021DBD5C9E6FFD6C9E6FF6D
:10734000D7C9E6FFD8C9E6FF0BDB60EC76F0BDEFEE
:107350003CF0010EE66EE66AEAC900F0016A026AD4
:10736000036AEAC9E6FF01C0E6FF6CD249DBC3EF5E
:107370003CF0E76EBBDAE7500026000E0122EAEF90
:107380003BF0B6D9F5EC97F02CEF3CF0E552E55226
:107390007DEF3BF0DE52B1D9DD521200010EDBCFA2
:1073A000E6FF020EDBCFE6FF12000BDA0DEF2EF048
:1073B000E7D926DBFAEF3CF0100EE66EE66AE80E3F
:1073C000E66E040EE8DA84DADE6ADD6A120083EC27
:1073D0009FF0E55282EF3BF044DAF3CF02F0F4CFB6
:1073E00003F0F3CFE6FFF4CFE6FF1200B9DA24ECA6
:1073F00075F0BDEF3CF0BEDACBEF3BF0DECFE9FF3E
:10740000DDCFEAFFEF501200E66E6BD9C4D982EFF0
:107410003BF00E0E1CDA90D9C20EE66EDC0EE66E64
:10742000000EE66E120064D937DABCD161D92CDACD
:10743000B9D16FDAD89001501200FD0EDBCFE9FF11
:10744000FE0EDBCFEAFF1200100EE66EE66AD80EE3
:10745000E66E040EE66E120000500324F36E015037
:107460000420F46E02500520F86EF4CFF7FFF3CF3E
:10747000F6FF0800F550E66E1200010EE66EE66AB1
:10748000EBC900F0016A026A036AEBC9E6FF01C0BA
:10749000E6FFD8D13AEC2EF02AEF2EF00A0E2B6E32
:1074A0002C6A2D6A2E6ACDC926F0CEC927F0CFC925
:1074B00028F0D0C929F059EFA8F0F5C900F0F6C9B5
:1074C00001F0026A036AF5C9E6FFF6C9E6FFBAD120
:1074D000060EDBCF00F0070EDBCF01F0D890015095
:1074E000120026C000F027C001F028C002F029C019
:1074F00003F01200FC0EDBCFE9FFFD0EDBCFEAFF4D
:10750000120019EC98F056D2A3EC3EF0E552E55289
:1075100009011200020EDBCFE9FFDB2A030EDBCFED
:10752000EAFF1200006E016AD950030FFFD9005024
:10753000EE260150ED221200F9D9EECFE6FFEECF94
:10754000E6FFEECFE6FFEFCFE6FF1200C1D9060E51
:10755000DB6A070EDB6A12000E0EE66E4E0EE66E5A
:10756000010E1200FE6F54EF3EF00E0EF66E000E8E
:10757000F76E000EF86E0800F550E66EE66A12002F
:1075800024EC75F0046E090EE15E04501200D9502F
:10759000FD0FE96EFF0EDA20EA6E120074ECA1F026
:1075A000046E0A0EE15E04501200020EA0CADBFF58
:1075B000030EA1CADBFF1200A0CAE6FFA1CAE6FFC4
:1075C00012009BD891EF3CF0DBCFE6FFFFEF3BF0E2
:1075D000D1C9E6FFD2C9E6FFD3C9E6FFD4C9E6FFA9
:1075E0001200DECFE9FFDDCFEAFFE50EE926050E4A
:1075F000EA221200570EFC6FDD0EFD6F000E120026
:10760000000E005C040E015812005F0EE66E0A0EBA
:10761000E66E1200D89000360136E8041200D9CF89
:10762000E9FFDACFEAFF1200E66E69EC98F02CEF82
:107630003CF049EC98F010D90009120091EC97F059
:10764000C1D90009120065D90001800E0114120091
:10765000DAD8EF6A120081EC90F0006E060EE15E5F
:1076600000501200EECF00F0EFCF01F0DF50001815
:107670001200DF50EA6AC30FE96E090EEA22120017
:1076800001EC75F0026E070EE15E02501200FB0E77
:10769000DBCFE6FFFC0EDBCFE6FF1200DFCFE9FF1A
:1076A000DF2A010EDBCFEAFF1200DECF02F0DDCFD2
:1076B00003F0D89003501200760EE66E0A0EE66EC6
:1076C0001200E750E926000EEA2212003A0EE66E9A
:1076D000DD0EE66E000E1200DECFE6FFDDCFE6FF28
:1076E0001200020EDBCFE6FF030EDBCFE6FF120037
:1076F000000EE66E060EE66E1200F3CFDEFFF4CF4C
:10770000DDFF1200020EF3CFDBFF030EF4CFDBFF31
:10771000120007EC75F0E2EF3CF0040EF3CFDBFF54
:10772000050EF4CFDBFF12001ED9D8EC74F0006E0A
:10773000050EE15E53EF39F0F3CF00F0F4CF01F026
:10774000F3CFE6FFF4CFE6FF120007EC75F0026E10
:10775000070EE15E02501200E66EE66AF9EF38F0BD
:10776000C0DE26C0E6FF27C0E6FF28C0E6FF29C02E
:10777000E6FF3C0EE66EDB0EE66E000EB3EF3CF06D
:10778000F86E0800F550E66EE66AC40EE66EDC0E92
:10779000E66E000E1200D8EC74F00CD194DD020EEF
:1077A000E1261200E66E96EC9DF0006E080EE15E9A
:1077B00000501200040EDBCFE6FF050EDBCFE6FF24
:1077C0001200E66EBFEC72F0E5521200E66EE66A59
:1077D000FCEF38F000C0E6FF01C0E6FF1200E4D87D
:1077E000000EE66E060E78DDDF2A010E1200570E3F
:1077F000E66EDD0EE66E000EB6D881EF3AF001ECD3
:1078000075F0E2EF3CF0020EDBCFE9FF030EDBCFB9
:10781000EAFF1200EF6AD0DEDFEC89F0B7DD23EF7C
:107820003BF03AEC2EF066DEDECFEEFFDDCFEDFF73
:107830001200DBCFE6FFE66ABF0EE66EDC0EE66EF8
:10784000000E120002C0E6FF03C0E6FF1200E66E63
:1078500083EC9FF0E5521200E552E552E552E55205
:107860001200A3EC98F0E552E552120013DE020E6E
:10787000E15C1200EDDC2C081200430EFC6FDD0E03
:10788000FD6F000EB2EF3AF0000EE66E020EE66EED
:10789000FA0EE66E040E1200000EE66E010EE66EA3
:1078A000F80EE66E040E1200010EE76EC6DD09DF6B
:1078B000EF501200F8DC520EE66EDB0EE66E000EA4
:1078C0001200F1DC4E0EE66EDB0EE66E000E1200CC
:1078D000E66EEDEC9CF0006E080EE15E00501200CA
:1078E0003DEC91F0E552E552C6EF39F0FD0EDBCFED
:1078F00000F0FE0EDBCF01F01200E5DC030EE12606
:107900001200E1DC040EE1261200C2DC020EE15C92
:107910001200DECF00F0DDCF01F0120071DC3AEF93
:107920002EF00901A051E66EE66A1200E96EDACF88
:10793000EAFF1200D9C9E6FFDAC9E6FF5ADCDBC963
:10794000E6FFDCC9E6FF55DC0901E05105DFE3C9CC
:1079500000F0016A1200E66EE66AB8DE19EF39F04F
:10796000B5DE00EF3DF0E66E1EEF39F0AFDEE66EFD
:1079700071EF3BF0E66E78EF3BF0006E090EE15ED2
:1079800000507DEF3BF0F9EC75F0046E0B0EE15EFC
:1079900004507DEF3BF0E66E000EE66E030EE66EE1
:1079A000FC0EE66E040E12000601006B010EE66E80
:1079B000E66A1200006E050EE15E0050120045DC22
:1079C0007DEF3BF0006E070EE15E00501200E6DE38
:1079D000D5EF39F0A3EC98F0D9DC6CEF3BF0FADE90
:1079E00050DC82EF3BF0DADCB0DECAEF39F039DF91
:1079F0009CEF3BF08EDE7DEF3BF027DC8DEF3BF024
:107A0000E66E6CEF3BF05A0EE66EDB0EE66E000E95
:107A1000B3EF3CF0560EE66EDB0EE66E000EB3EFF3
:027A20003CF038
:0E7A2200D8CFE4FFE0CFE4FFE46EDACFE4FF5C
:107A3000E2CFDAFFE9CFE4FFEACFE4FFF6CFE4FFDD
:107A4000F7CFE4FFF8CFE4FFF5CFE4FFF3CFE4FF97
:107A5000F4CFE4FFFACFE4FFFBCFE4FF00EE20F029
:107A6000140EE80403E3EECFE4FFFBD700EE00F0D2
:107A7000200EE80403E3EECFE4FFFBD7E65207EC69
:107A8000A1F066ECA2F0E55200EE1FF0200EE80433
:107A900003E3E5CFEDFFFBD700EE33F0140EE8046F
:107AA00003E3E5CFEDFFFBD7E5CFFBFFE5CFFAFF23
:107AB000E5CFF4FFE5CFF3FFE5CFF5FFE5CFF8FF26
:107AC000E5CFF7FFE5CFF6FFE5CFEAFFE5CFE9FF2A
:107AD000E5CFDAFFE550E5CFE0FFE5CFD8FF1000B6
:107AE0000801009B1200C0EC49F0E652D9CFE6FF36
:107AF000DACFE6FFDDECA0F0E552E552000901E146
:107B0000D0D0FF0E0601EB5D01E094D0C85103E038
:107B10007F0EC85D08E10A0EDF5CE8E00D0EDF5C59
:107B200002E10A0EDF6E0D0EDF5CE0E00AEC4BF0C6
:107B300065EC4AF003E1015001E1EA073A0EDF5C2F
:107B40001EE1060EEA5D1BE383EC4AF018E1490EE4
:107B5000015D15E1500E025D12E1440E035D0FE17F
:107B60000601EA059FEC49F0EF6A050EE66E070E86
:107B7000E66E3AEC4AF0FD0EEB6FEA6BB7D70A0EF1
:107B8000DF5CB4E10601EA07EA519FEC49F0EF6AD5
:107B9000040EEA5D48E383EC4AF045E1430E015DE3
:107BA00042E14D0E025D3FE1540E035D3CE1070EE4
:107BB000DF6EDF50DF2A9FEC49F0EF50220804E02F
:107BC0000601EA51DF5CF5E3DF049FEC49F0EF6A60
:107BD0000601D66B140EE66EE66A070EE66E070E19
:107BE000E66ED60EE66E060E12EC4AF00601E96B62
:107BF000EAC6DFFFDF50DF069FEC49F0EF502C08AC
:107C000003E0DF500008F6E3DF50016A000F006E6A
:107C1000070E0122020E6BEC4AF03AEC4AF0EA6BD6
:107C2000FE0EEB6F63D70601F9EC49F00701006B1C
:107C3000060135D0FE0EEB5D1CE10D0EDF5C03E0AE
:107C40000A0EDF5C07E1EA51EA2B9FEC49F0200EB7
:107C5000EF6E02D00AEC4BF065EC4AF003E1015004
:107C600001E1EA07EC07EC5101E040D76BEC4BF087
:107C700016D00D0EDF5C08E00AEC4BF065EC4AF024
:107C800003E1015001E1EA07EC070A0EDF5C03E1C2
:107C9000EA076BEC4BF0EC5101E028D7EA6BEB699B
:107CA00025D7E552C5EF49F070EC4BF038E1DF6ABB
:107CB00096EC49F00A080BE10D0EDF5C08E00801C4
:107CC00000B1FDD70D0EC9EC49F00FE1FBD70D0E49
:107CD000DF5C0BE196EC49F00A0807E0080100B10F
:107CE000FDD70A0EC9EC49F0FCE096EC49F028E01B
:107CF000080100B1FDD796EC49F0C9EC49F0FBE072
:107D00000901FCC9F6FFFC2BFDC9F7FF000EFD239E
:107D1000FEC9F8FFFE230800F550DF6EC9D796ECC8
:107D200049F00EE0080100B1FDD796EC49F0C9EC2E
:107D300049F0FBE00901FC2B000EFD23FE23EFD7E9
:107D4000E552C5EF49F070EC4BF035E1DF6AB8EC75
:107D500049F00A080BE10D0EDF5C08E0080100B1F4
:107D6000FDD70D0EC9EC49F00FE1FBD70D0EDF5C1E
:107D70000BE1B8EC49F00A0807E0080100B1FDD7B3
:107D80000A0EC9EC49F0FCE0B8EC49F025E0080126
:107D900000B1FDD7B8EC49F0C9EC49F0FBE0FD0EAD
:107DA000DBCFE9FFDB2AFE0EDBCFEAFF01E3DB2AB4
:107DB000EFCFDFFFCCD7B8EC49F00EE0080100B1FF
:107DC000FDD7B8EC49F0C9EC49F0FBE0FD0EDB2A29
:107DD000FE0EF1E3DB2AEFD7E552C5EF49F0C0EC28
:107DE00049F0080100B1FDD7FE0EDBCFE6FFB6EC8F
:107DF000A0F0E5520009F8E0C5EF49F0C0EC49F009
:107E0000040EE126030EFFEC49F0620EE66EDA0E78
:107E1000E66E000EE0EC49F00EE0FD0EDBCF00F068
:107E2000FE0EDBCF01F000C001F0006A0050060139
:107E3000F1130150F2135F0EE66EDA0EE66E000EDD
:107E4000E0EC49F00BE0FD0EDBCF28F0FE0EDBCFBF
:107E500029F028500601F1132950F213040EE15CB9
:107E600002E2E16AE552E16EC5EF49F0C0EC49F08B
:107E7000060EE126F3EC4AF0E66EFD0EDBCFE6FFE0
:107E8000FE0EDBCFE6FF6CEC49F069E0F3EC4AF064
:107E900076EC4BF064E0A1EC4BF061E0A1EC4BF030
:107EA0005EE08BEC4AF0EF504F0859E1010EE76EAF
:107EB0008BEC4AF0E750E926000EEA22EF502D083D
:107EC0004EE15B0EE66EDA0EE66E000EE66E020E18
:107ED000E76EDBCF00F0030EDBCF01F0E7506BEC79
:107EE0004AF0EBEC4AF0F9EC4AF039E05B0EE66E52
:107EF000DA0EE66E000EA5EC49F0D6EC49F0F35030
:107F0000A5EC4BF0040EF3CFDBFF050EF4CFDBFF47
:107F10001AEC4AF00DE1040EDBCFE9FF050EDBCFD2
:107F2000EAFFEF501CE05A0EE66EDA0EE66E12D053
:107F300092EC4AF0040EDBCFE6FF050EDBCFE6FF46
:107F400049EC98F0E552E552E552E552000907E0A8
:107F500092EC4AF0D6EC49F0F35099EC4AF0060E58
:107F6000E15C02E2E16AE552E16EC5EF49F0C0EC86
:107F700049F0020EE126FE0EDBCFC8F60601C8511D
:107F8000240A01E15FD1070A01E152D1010A01E1AE
:107F900049D1030A01E115D1010A01E1FCD0600ACF
:107FA00001E1D7D0030A01E1B9D0010A01E18FD084
:107FB000030A01E178D0530A69E0030A5CE0010A90
:107FC0004FE0160A47E0030A3CE0010A33E0070AE3
:107FD00025E0010A21E0030A11E07E0A0CE07F0A95
:107FE00001E03CD182EC4BF0F2EC49F00601010ECD
:107FF000CD6F0A0E24D183EC7DF030D10A0E21EC36
:108000004BF00601030ECD6F140ECE6FCF6B09013E
:10801000E86B06EC2EF022D1CD6B20D1F2EC49F0CA
:10802000CFEC72F00601020ECD6F22EC4AF0060191
:10803000CC6B14D1050ECD6F0A0E22EC4AF00A0E5D
:108040009ED0060ECD6F020ECE6FCF6BC96BCFECFC
:1080500072F004D1E66A36EC49F0A5EC72F0FED07D
:10806000090E21EC4BF044EC4AF0140EFC6F4D0E5F
:10807000FD6F010ED4D0080E21EC4BF044EC4AF019
:108080005B0EFC6F4D0EFD6F010EC9D0070E21EC8B
:108090004BF00601030ECD6F230ECE6FCF6BC96B75
:1080A000A0EC4AF0BCD0050EE66E94EC4BF04DEC23
:1080B0004AF006E2070EDCEC49F00601400E05D05E
:1080C000080EDCEC49F00601020ECD6F14D0050E4F
:1080D00002EC4AF0410EFC6FDA0EFD6F000E29EC47
:1080E0004AF0090EDCEC49F04DEC4AF002E2430E96
:1080F00001D0020ECD6FCAC6CEF6CBC6CFF60A0EA1
:10810000D880CE57000ECF570F0ECF03F3CFCFF648
:10811000CE03F3CFCEF6F450CF27A0D0050E21EC3E
:108120004BF006EC4AF00601020ECD6F3C0ECE6F0E
:10813000CF6B060EC96F0901E86B0AEC2EF08AECD2
:108140004BF0A7EC4AF029EC4AF00601400EC86F4C
:1081500085D0050E21EC4BF006EC4AF0FFEC49F01F
:1081600035EC4AF0EF5014E02EECA8F0000910E0D6
:108170000601020ECD6F3C0E22EC4AF0020EB3EC6B
:1081800049F009014E0EFC6FDA0EFD6F000E47D06C
:108190000601200EC86F020E21EC4BF00A015E6B47
:1081A0000601CD6BC96B0901E60507E0050EE65D2A
:1081B00004E0780E0601D26F02D00601D26BD36BB9
:1081C0004DD0060E21EC4BF08AEC4BF00601030E6D
:1081D000CD6FF00ECE6FCF6B0AEC2EF00D0EFFECD4
:1081E00049F035EC4AF0EF5007E10901C30EFC6F8E
:1081F0004D0EFD6F010E13D009011B0EFC6FDA0E40
:10820000FD6F000E29EC4AF017EC4BF09CDDE552B7
:10821000E5520901110EFC6FDA0EFD6F000E29EC1C
:108220004AF01CD00A0ECE6FCF6B400ECD6F16D029
:10823000060E21EC4BF00601240ECD6F1E0ECE6F04
:10824000CF6B0CD0CC51CC2B006E140E005C02E234
:10825000020E01D0030EE66E8ADEE552020EE15CEC
:1082600002E2E16AE552E16EC5EF49F0C0EC49F087
:10827000110EE126FE0E0601EB5D1AE10901E6058D
:1082800007E0050EE65D04E006EC4AF090EC4BF0EA
:108290000501F6BF03D005010A0EF76FAEEC4AF0F8
:1082A000D60EE66E060EE66EB2EC4AF0C2EF45F070
:1082B000FF0EEB5D10E00501F6BF03D00501140EC3
:1082C000F76FE6EC4AF0E2EC33F0E552E552BDEC34
:1082D0004AF0C2EF45F00501F6BF03D005011E0EBE
:1082E000F76F0601C8517F0A02E1BBEF45F05F0A54
:1082F00001E117D2600A01E15ED1630A01E141D1D7
:10830000020A01E1F7D0330A01E1CAD0030A68E0AA
:10831000010A2CE0110A17E0010A02E0C2EF45F061
:10832000050EEA5D02E2C2EF45F0CCEC4AF00B0E1E
:10833000E66EDA0EE66E000E29EC49F002E0C2EFBE
:1083400045F07F0EEAD1020EEA5D02E2C2EF45F08F
:1083500087EC4AF002E0C2EF45F04B0E015D02E00F
:10836000C2EF45F090EC4BF0100ED7D1040EEA5D51
:1083700023E383EC4AF020E1430E015D1DE1530E3F
:10838000025D1AE14D0E035D17E1E6EC4AF0A3EC45
:1083900098F0E552E552F3CFE9FFF4CFEAFFE906A2
:1083A000000EEA5A000EE926070EEA22EF503108C5
:1083B00001E1E8D3030E5AD00601C95101E0E2D32E
:1083C000020EEA5D01E2DED387EC4AF001E0DAD387
:1083D0004B0E015D01E0D6D390EC4BF0110E9DD118
:1083E000100EEA5D14E3380E0701005D10E1390E4E
:1083F000015D0DE1180EE66EE66AE6EC4AF0CD0E80
:10840000E66E050E12EC4AF00501E46BBBD3080ED4
:108410000601EA5D16E383EC4AF013E1430E015DC9
:1084200010E1500E025D0DE1420E035D0AE1460EC1
:10843000045D07E13A0E055D04E1E6EC4AF016DD65
:1084400095D1080E0601EA5D17E383EC4AF014E1CA
:10845000430E015D11E1500E025D0EE1490E035D18
:108460000BE1520E075D01E18DD3040EDCEC49F007
:108470000601010EC96F86D30601C95101E082D3FE
:10848000020EEA5D01E27ED387EC4AF001E07AD386
:108490004B0E015D01E076D390EC4BF0120E3DD116
:1084A000060EEA5D16E383EC4AF013E1490E015D26
:1084B00010E1500E025D0DE1520E035D0AE1390E2E
:1084C000065D07E00901FA0EFC6F4D0EFD6F010E0F
:1084D0006DD1020E0601EA5D01E254D387EC4AF049
:1084E00001E050D34B0E015D01E04CD390EC4BF01A
:1084F000210E13D1020EEA5D0BE387EC4AF008E18E
:108500004B0E015D05E1BDEC4AF0CC6B220E05D1AE
:10851000050E0601EA5D07E3450E0701005D03E174
:10852000520E015D05E044EC4BF029EC49F002E10C
:10853000230EF3D0D0EC4AF0F90EE66ED90EE66EBB
:10854000000E29EC49F001E01DD3F3EC4AF0E66E91
:10855000E6EC4AF06CEC49F001E114D3F3EC4AF09C
:1085600076EC4BF001E10ED3080EE66EE66A17ECEE
:108570004BF0EC0EE66E090E12EC4AF00901F46BBA
:1085800001D324EC4BF001E0FDD22C0E0701085D75
:1085900003E1070E091502D0070E07150901E66F62
:1085A000E80404E0050EE65D01E0ECD2BDEC4AF023
:1085B000CC6B400EB2D0020EEA5D16E3450E070109
:1085C000005D12E1520E015D0FE1020E0601C95D70
:1085D00003E0030EC95D02E1410E9FD0050EC95DA7
:1085E00001E0D0D2030E99D0020E0601EA5D06E347
:1085F00087EC4AF003E14B0E015D0BE0530E0701DF
:10860000005D03E1480E015D04E0050E0601C95D51
:108610006DE10601EA6B1E0ECE6FCF6B0901E76BB1
:108620008AEC4BF00601C92BC951080A5DE00F0A1C
:1086300048E0010A43E0030A3AE0010A31E0070A90
:1086400026E0010A0DE0030A01E09CD20901DF0ED9
:10865000FC6FD90EFD6F000E29EC4AF0050E0FD00D
:108660000901D20EFC6FD90EFD6F000E29EC4AF005
:10867000050E2CEC4BF0060E2CEC4BF0070E5DECCF
:1086800049F0DC0EFC6FD90EFD6F000E8FD0040E8A
:1086900002EC4AF0C40EFC6FD90EFD6F000E86D0BE
:1086A0000901B60EFC6FD90EFD6F000E7FD00901D7
:1086B000AC0EFC6FD90EFD6F000E78D0A7EC4AF01F
:1086C00075D0030E02EC4AF0980EFC6FD90EFD6FC8
:1086D000000E29EC4AF0040E5DEC49F08E0EFC6FA2
:1086E000D90EFD6F000E62D0200E17D0070EEA5D86
:1086F0000DE3080EE66EE66A850EE66ED90EE66EAE
:10870000000E29EC49F002E1020E07D04DEC4BF0CF
:1087100029EC49F001E036D2020EE66EB7EC3FF0EC
:1087200026D024EC4BF025E12C0E0701085D03E177
:10873000070E091502D0070E07150901E66FE804B8
:1087400003E0050EE65D05E10601D26BD36BE66A38
:108750000AD00601D251D31101E014D2780ED26FA3
:10876000D36B010EE66EE66A33ECA2F0E552E552F9
:1087700009D2CCEC4AF0730EE66ED90EE66E000E0E
:1087800029EC49F016E10901E60507E0050EE65D72
:1087900004E006EC4AF090EC4BF0010EB3EC49F02B
:1087A0000901DB0EFC6F4D0EFD6F010E29EC4AF046
:1087B000E9D1020EE66EE66A700EE66ED90EE66E3E
:1087C000000E29EC49F001E0BCD0C2EC4AF001E314
:1087D000B8D010EC4BF0020EE66E070EEFEC49F04D
:1087E00030EC49F00EE056EC4AF0020E26C0DBFFFA
:1087F000030E27C0DBFF040E28C0DBFF050E29C0D7
:10880000DBFF30EC49F005E035EC4AF00A0EEFCF23
:10881000DBFF30EC49F00EE056EC4AF0060E26C0C5
:10882000DBFF070E27C0DBFF080E28C0DBFF090EA9
:1088300029C0DBFF30EC49F005E035EC4AF00B0EC7
:10884000EFCFDBFF30EC49F005E035EC4AF00C0EE1
:10885000EFCFDBFF30EC49F030EC49F030EC49F081
:1088600008E0D6EC49F00D0EF3CFDBFF0E0EF4CF8F
:10887000DBFFF9EC4AF001E185D10C0EDB50010B76
:108880000901E06FE8505AE00A0EDB50530818E186
:10889000020EDBCF00F0030EDBCF01F0040EDBCFC6
:1088A00002F0050EB6EC4AF0020E00C0DBFF030E2C
:1088B00001C0DBFF040E02C0DBFF050E03C0DBFFBF
:1088C0000B0EDB50570818E1060EDBCF00F0070E49
:1088D000DBCF01F0080EDBCF02F0090EB6EC4AF058
:1088E000060E00C0DBFF070E01C0DBFF080E02C052
:1088F000DBFF090E03C0DBFF020EDBCFD1F9030E55
:10890000DBCFD2F9040EDBCFD3F9050EDBCFD4F9E0
:10891000060EDBCFD5F9070EDBCFD6F9080EDBCF7D
:10892000D7F9090EDBCFD8F90D0EDBCFDBF90E0E30
:10893000DBCFDCF90901780EE36F24D10901E36B89
:1089400021D1030EE66EE66A6A0EE66ED90EE66E79
:10895000000E29EC49F022E1C2EC4AF01FE210ECD3
:108960004BF0030EE66E070EEFEC49F008E0D6EC94
:1089700049F00F0EF3CFDBFF100EF4CFDBFFF9EC65
:108980004AF001E1FFD00901E05101E1FBD00F0EF7
:10899000DBCFD9F9100EDBCFDAF9F4D00A0EE66E90
:1089A000E66A5F0EE66ED90EE66E000E29EC49F01F
:1089B00004E10901E75125E119D0070EE66EE66AE8
:1089C000570EE66ED90EE66E000E29EC49F042E134
:1089D000110EE66EE66A450EE66ED90EE66E000EE4
:1089E00029EC49F012E10901E7510BE1010EE66EB5
:1089F000E66EDCEC4AF00DEC2EF0AEEC2EF02AEC3C
:108A00002EF00901010EE76FBDD0150EE66EE66A85
:108A10002F0EE66ED90EE66E000E29EC49F001E14C
:108A2000B1D0110EE66EE66A1D0EE66ED90EE66E48
:108A3000000E29EC49F055E00901E76B020EE66EE5
:108A400094EC4BF00901E60569E0050EE65D01E0F6
:108A500099D064D0CCEC4AF0170EE66ED90EE66ED3
:108A6000000E29EC49F012E12C0E0701085D09E126
:108A7000070E0715006E070E06150A0DF3500024A9
:108A800002D0070E06150901E96F7CD0070EE66ECD
:108A9000E66A0F0EE66ED90EE66E000EDADB56E0E1
:108AA0000B0EE66EE66A030EE66ED90EE66E000E5B
:108AB000D0DB03E10A015E6B65D0D0EC4AF0FC0E1E
:108AC000E66ED80EE66E000EC4DB0BE00C0EE66E12
:108AD000E66AEF0EE66ED80EE66E000ECFEC49F0B9
:108AE00004E10AEC2EF0420E34D0090EE66EE66A7E
:108AF000E50EE66ED80EE66E000EABDB0FE044EC42
:108B00004BF0CFEC49F00AE04DEC4BF098EC4BF019
:108B1000026E070EE15E0250000904E10AEC2EF03D
:108B2000410E17D0040EE66EE66AE10EE66ED80E30
:108B3000E66E000E8EDB0AE0D0EC4AF0DA0EE66E4E
:108B4000D80EE66E000ECFEC49F007E10AEC2EF0ED
:108B5000010EE66EB7EC3FF014D0D0EC4AF0D30E25
:108B6000E66ED80EE66E000E74DB0CE1E6EC4AF021
:108B700009EC37F005D0AEEC4AF055EC80F0E55248
:108B8000E552E552110EE15C02E2E16AE552E16E66
:108B9000C5EF49F0C0EC49F0080EE1260601C851C6
:108BA0007F0A01E165D15F0A43E0220A3FE0230A20
:108BB00032E0330A2AE0030A1EE0010A12E0110A39
:108BC00001E058D1050ECE5D000ECF5903E2020E32
:108BD000DCEC49F00901D70EFC6F4D0EFD6F010E64
:108BE00045D198DB01E046D10901140EFC6F4D0E12
:108BF000FD6F010E3BD18EDB01E03CD109015B0E24
:108C0000FC6F4D0EFD6F010E31D184DB01E032D1DE
:108C1000A0EC4AF02BD1140ECE5D000ECF5901E32B
:108C200029D1D0EC4AF033ECA2F0EAD0E66A23D0A6
:108C3000FF0EEB5D09E0ED0503E1ED6BEB6910D094
:108C4000ED51010801E2ED07000ED880D255000E6B
:108C5000D35508E2D207000ED35BD251D31102E103
:108C6000210E08D0D4EC4AF009E25E2B5E513C089C
:108C700005E2400EE66EB7EC3FF0C3D00901E60511
:108C800004E0050EE65D01E0F5D00A019E519F115A
:108C900006E00A015D0503E10A015E5128E0FF0ECE
:108CA0000601E1EC4AF067E20A015D0564E18DEC42
:108CB0004BF0200E0601E1EC4AF004E2F19B9EEC41
:108CC00038F0D8D0040EE1EC4AF014E2F195F351FB
:108CD00001E0D0D0060E0A019E6F9F6BA0CAE9FF8B
:108CE000A1CAEAFFEF6A0A015E5101E0C3D089EC34
:108CF00036F0C0D0080EE1EC4AF006E2F197EEA3A0
:108D0000B9D0D1EC38F0B6D0100EE1EC4AF004E264
:108D1000F199ACEC38F0AED0020EE1EC4AF00AE288
:108D2000F1938DEC4BF0020EE66E74EC2FF0E552F1
:108D300002081ED0010EE1EC4AF01DE2F19109019A
:108D4000E851000818E20A015E5115E1020EDF6EDB
:108D50008DEC4BF0DFCFE6FF76EC31F01CEC4BF006
:108D600074EC2FF0E552DF6E020EDF5C01E182D081
:108D70002AEC2EF07FD0000E0601F115006EFF0EDA
:108D800000EC4BF04DE28DEC4BF06CDB000E06017D
:108D9000F115006E200E00EC4BF005E2F29BADDA0F
:108DA0006DEC59F02DD0D8EC4AF0040E00EC4BF0ED
:108DB00012E2F295F3515EE1CE0EE66ED80EE66E4B
:108DC000000E91DB8AEC98F05FEC4BF0040E8BDB2D
:108DD00094DAC8DB4FD0ECDB080E00EC4BF007E276
:108DE000F297EEA347D089DAB6EC59F009D0E0DB70
:108DF000100E00EC4BF007E2F2997FDA82EC59F0AA
:108E0000E552E55237D0D4DB020E00EC4BF002E223
:108E1000F29306D0CDDB010EF3DB02E2F2912AD011
:108E200009019F51000816E20501ED51000812E208
:108E30000A015E510FE10901E85100080BE28AECDA
:108E40004BF0020EE66E69EC30F0E552020802E0EB
:108E50002AEC2EF09CDB02E3D7DB0CE193DB0AE289
:108E60000901360EFC6F4D0EFD6F010EF2DA02D0D5
:108E7000A3EC7DF0080EE15C02E2E16AE552E16EEE
:108E800084D20601C851200A01E012008DDB02E203
:108E90002CEF4AF0B9DB14E08AEC4BF00901E00E4C
:108EA000FC6F4D0EFD6F010EFE6F54EC3EF008019D
:108EB0004151000803E2010E56DAF9D7020E53DAE7
:108EC00012005EDA030EE1260901EA511AE133ECE1
:108ED000A8F026C000F027C001F028C002F029C089
:108EE00003F0EADA01C028F002C029F003C02AF03A
:108EF000A8EC83F01DEC85F029C0EAF90901EB6BC1
:108F00003BD0EA51026E036AEAC9E6FF03C0E6FFFE
:108F100033ECA8F0E552E7CF03F0E552E7CF02F0DB
:108F200026C004F027C005F028C006F029C007F0CD
:108F3000C3DA05C028F006C029F007C02AF0A8EC63
:108F400083F044EC85F002502824006E0350292061
:108F5000016E010E0026000E0122020E2D6E2E6AF9
:108F600000C028F001C029F02FEC84F028C000F0E8
:108F700029C001F028C0EAF909019DB907D00F0EF8
:108F80000901EB5D09E2090199AF03D00901EB6B1F
:108F90000ED00901EB2B0BD00F0EEB5D08E10901A0
:108FA0009951800B04E1EAC9EBF90701CA93090161
:108FB000EB510F0825E209019951800B21E1020EC6
:108FC0000701CA150AE10D0E0901EB5D0901D88000
:108FD000EA5503E30701CA830CD0020E0701CA1544
:108FE0000FE0070E0901EB5D0901EA5D09E30701E6
:108FF000CA93080EE66EE66AFEEC3EF0E552E552D4
:109000000601C851200A1BE1CFDA02E225DA17D0A7
:109010000901E70510E10901E85100080CE27DDBD8
:1090200045DB01E048DB0C0E24D901E070DB2BD9D5
:1090300002E02AEC2EF0010E0601C919C96F030ED9
:10904000E15C02E2E16AE552E16E9FD1120054DB7D
:109050000AE0020E945D07E00F0E945D04E097DADB
:1090600002E3000E01D0010E46DA49E1050E0901C6
:10907000A05D29E2800E0901991525E10601F05154
:109080000FE10901E7050DE10A015E510AE1060160
:10909000EEA502D0BAEC38F00601480EF06F01D010
:1090A000F0070601EF510DE1DDD90601EEA505D06F
:1090B00024D997EC59F0E552E5520601480EEF6FBE
:1090C00006D0EF0704D00601060EEF6FF06F09011E
:1090D000E70515E10901E85112E1030EDB500FE04D
:1090E00063DA02E2B9D90BD0E1DA01E0E4DA0C0E7E
:1090F000C0D801E00CDBC7D802E02AEC2EF0040E49
:10910000E15C02E2E16AE552E16E3FD1F5DA0AE0A4
:10911000020E945D07E00F0E945D04E038DA02E37E
:10912000000E01D0010EE7D918E10901E70515E1AC
:109130000901E85112E1030EDB500FE135DA02E2DA
:109140008BD90BD0B3DA01E0B6DA0C0E92D801E07D
:10915000DEDA99D802E02AEC2EF0040EE15C02E29D
:10916000E16AE552E16E11D10601F351000801E216
:10917000F307D02B000ED123CD51000810E2CEC64C
:1091800000F0CFC601F0CE07000ECF5B00500110FB
:1091900006E1CDC6E6FFB7EC3FF0E55201D0FADCC0
:1091A0003CD91E0E2D6E2E6A83D801E16ADE2CDAC0
:1091B00001E187DE32D92C0E2D6E010E2E6E78D88D
:1091C00001E144DF2AD9580E2D6E020E2E6E70D8A2
:1091D00001E13DDF22D9100E2D6E0E0E2E6E68D8E5
:1091E00006E194DF100E0601D05F0E0ED15B060182
:1091F000D407000ED55BD451D5111EE1E66A36D8EE
:10920000060180DA0501EF2BEF51E66EE66AE66AA9
:10921000E66AE66A000EE66E060EE66E07EC75F08C
:10922000006E070EE15E0050000EE66E060EE66E62
:109230001A0E7FD9A5EC72F012001200800E946E07
:109240009AECA0F00901E66BE66AB7EC3FF0E55254
:1092500012006EDA006E070EE15E00500009120087
:10926000DFD9000EE66EE66AB6D92ED25DDA90EF4F
:109270004BF0E66EF9D9010EDBCFE9FF020EDBCF32
:10928000EAFFEF501200DFCFE6FF74EC2FF0D4D9E5
:1092900069EC30F0D1D988EC30F0CED976EC31F0F1
:1092A000CBD920EC32F0E552DF6E020EDF5C12000B
:1092B000D0C628F0D1C629F0DED147DAF3CF00F0CE
:1092C000F4CF01F0F3CFE6FFF4CFE6FFA3EC3EF0DE
:1092D000E552E552090112004AECA4F0F0D92CDA6B
:1092E000F9EF4AF0E66EDFCFE6FF5AEC32F0E552D6
:1092F000E552E552E552DF6E1200010EDBCFE6FFCC
:10930000020EDBCFE6FF1200000ED8800054000EE4
:1093100001541200CEC600F0CFC601F0030E2D6E30
:109320002E6ACEC628F0CFC629F0A5D1FCC9F6FF1B
:10933000FDC9F7FFFEC9F8FF0800F5501200EA6A00
:10934000000FE96E070EEA221200E66E000EE66ECE
:10935000E66A4AECA4F0B3D9020EF3CFDBFF030EAA
:10936000F4CFDBFF1200E66EBFEC72F0E5521200A4
:10937000FD0EDBCFE9FFFE0EDBCFEAFFEF50120060
:10938000D9CFE6FFE1CFD9FF1200E552E7CFD9FFF1
:109390001200E66EB6ECA0F0E55200091200C8D942
:1093A000016E070EE15E01500009120040D9DFECAA
:1093B00089F0E552E5521200E66EE66ADCEF4AF00B
:1093C000E66E35D92FEC99F0026E050EE15E025083
:1093D000F3CF00F0F4CF01F0F350F4101200E66E7A
:1093E000FAD872D1E668A0D9E668E66AE5D85AEFFD
:1093F000A2F088D936EC41F00601EA6B1200A5D93B
:109400009CEF4BF0E66E90D9090112000601D26B79
:10941000D36B0901050EE66F1200D0C600F0D1C66D
:1094200001F01200E66E01EC99F0006E060EE15EAE
:1094300000501200D950020FE96EDACFEAFFEE5069
:10944000ED101200CE6FCF6BC96B0901E86B0AEF0C
:109450002EF0FE6F54EF3EF0050E0601D05F000EB9
:10946000D15B1200E66A34EF4BF0DECFE9FFDDCFCF
:10947000EAFF1200DFEC89F0E552E552F3CFECF69B
:1094800006013C0EED6F12000601030ECD6F5F0E5C
:10949000CE6FCF6BC96B090112000601CA07000E1F
:1094A000CB5BD880CA55000ECB551200C0D8D3EC88
:1094B00073F0E552E55212002C6A2D6A200E2E6ED2
:1094C000410E2F6E26C027F01200EA51006E016A8D
:1094D000C80E001812000026000E012200C0E6FF90
:1094E00001C0E6FF1200E66ED950030FE66E000ED3
:1094F000DA20E66E1200E76E030EE7CFDBFF06010F
:10950000C851200A12002B0E0701005D12004F0EF9
:109510000701005D1200020EDBCFE9FF030EDBCF77
:10952000EAFF1200020EDBCFE6FF030EDBCFE6FF01
:109530001200E66ECAEC9FF0E552E552E5521200C9
:109540000901760EFC6F4D0EFD6F010E1200090130
:10955000290EFC6FDA0EFD6F000E1200EAC6E6FF60
:10956000E6EF4AF027EC61F05FEF4BF0DBCF03F062
:10957000001E011E021E031E12000A0E0601CA6F03
:10958000CB6B1200010E0601EE1500081200800ED2
:109590000901991500081200050EE66EE66A120030
:1095A000060EE66EE66A12000A015E51000812001D
:1095B000000EF115006E120033ECA2F0E552E552F8
:1095C0001200F115006E016A84EF49F0000EE66E9C
:1095D000070EE66E12004AECA4F0026E050EE15E84
:1095E00002509CEF4BF05D0EE66EDA0EE66E000E5A
:1095F0001200D9CFE9FFDACFEAFFEE50ED101200EA
:10960000F215016E84EF49F008DF3C0E2D6E2E6AD4
:1096100058EF49F0EA51EA2B92DEDFCFEFFF12005C
:109620006E0EE66ED90EE66E000EE66E1200DECF0E
:10963000E6FFDDCFE6FF1200E552DF6EDFCFE6FF8B
:109640001200E66E36EF49F0A7DFF30EE66ED90E94
:10965000E66E000E29EF49F030DECE0EFC6FD90E1B
:10966000FD6F000E29EF4AF083EC9FF0E552DE52C9
:1096700063D8DD521200CEECA8F024C000F025C063
:1096800001F02450251012000A0EE66EE66A000E64
:10969000E66EDA0EE66E000E12000B0EE66EE66A5D
:1096A000790EE66ED90EE66E000E1200020EDF6E27
:1096B0000B0E39EF49F021DE010E72EF49F0006E1A
:1096C000050EE15E00501200DECF00F0DDCF01F0AC
:1096D000005001101200EA5132DEEF6AF9EF49F052
:1096E0004FDEE6527F0E0601C85D1200E66E000EE8
:1096F000E66EE66A6CEF49F043DE040EE1260901EE
:1097000094051200080ED46F070ED56F1200F5DD18
:1097100072EF49F0020EB3EF49F00A0EB3EF49F0D1
:10972000E66AE66ADCEF4AF0010EE66EDCEF4AF02C
:10973000E66E4CDF91EF97F0F3CFDEFFF4CFDDFF65
:10974000120051DF02DE1AEF4AF0E66E83EC9FF062
:04975000E5521200CC
:0C97540064EC58F0AAEC58F0EE6AEE6AE3
:10976000EE6AEE6ADDEC57F0EE6AEE6AEE6AEE6AD9
:1097700019EC55F0010EEE6E230EEE6E450EEE6EF8
:10978000670EEE6E19EC55F0040E5BEC56F0890E88
:10979000EE6EAB0EEE6ECD0EEE6EEF0EEE6E19ECC3
:1097A00055F0080E5BEC56F0FE0EEE6EDC0EEE6E23
:1097B000BA0EEE6E980EEE6E19EC55F00C0E5BECD8
:1097C00056F0760EEE6E540EEE6E320EEE6E100EFB
:1097D000EE6EE552E7CFD9FF120064EC58F0080EA8
:1097E000E126030E046EDDEC57F08FEC56F003E03B
:1097F000AFEC56F0FDE13F0E0016E9EC56F01EEC22
:1098000058F0F90EDBCF04F0FA0EDBCF05F0066A54
:10981000076A05AE02D006680768030E1F0B07E053
:10982000D8900436053606360736E806F9E1DDEC51
:1098300057F00450EF26EECF00F00550EF22EECFA8
:1098400001F00650EF22EECF02F00750EF22EECFEC
:1098500003F0F90EDBCF08F0FA0EDBCF09F00A6A4D
:109860000B6A09AE02D00A680B68030E1F0B03E0F7
:10987000C0EC56F0FDE10850005C095001580A5058
:1098800002580B50035806E2AAEC58F0EE2AEE22DA
:10989000EE22EE22C7EC56F0026A036A01AE02D055
:1098A000026803681D0EAFEC56F0FDE1AAEC58F01B
:1098B00057EC58F0400E046E056A066A076AD9CF65
:1098C000E9FF95EC56F0EE500758060E00C0DBFF9E
:1098D000070E01C0DBFFC7EC56F081EC58F00150D9
:1098E0000318E8AE02D0033404D00250005C0350E9
:1098F00001586AE3060EDBCFE6FF070EDBCFE6FF7B
:1099000083EC56F060EC58F0E9CF02F0EACF03F0B8
:10991000DB50E924006E010EDB50EA20DFEC56F04C
:10992000B0EC97F0046E060EE15E045060EC58F067
:109930007AEC56F019EC55F0E9CF02F0EACF03F0DB
:109940009EEC56F0060EDBCF28F0070EDBCF29F099
:10995000040E28C0DBFF050E29C0DBFF3F0EE76EBB
:1099600047EC58F0E7500026000E012240EC58F07A
:1099700001500318E8AE02D0033404D00250005C5A
:10998000035001581EE2040EDBCF02F0050EDBCFC0
:1099900003F0FB0EDB500224006EFC0EDB500320B4
:1099A000DFEC56F019EC55F0E9CF04F0EACF05F002
:1099B0009EEC56F09DEC58F0400EEE26000EED2287
:1099C000CDD788EC58F004D0040EDB6A050EDB6AB4
:1099D00040EC58F0040EDB50025C006E050EDB50CC
:1099E0000358DFEC56F0B6EC56F0046EFC0EDB507C
:1099F0000720056E04C0E6FFE66E60EC58F0E9CF84
:109A00000AF0EACF0BF0DB50E924086E010EDB50C0
:109A1000EA20096E08C0E6FFE66EB0EC97F00C6E27
:109A2000060EE15E0C50080EE15C02E2E16AE552CE
:109A30008AEF56F0D4EC56F0080EA9EC56F0100E52
:109A40005BEC56F07AEC56F0D9CFE6FFDACFE6FFC2
:109A5000CEEC56F0030E046E8FEC58F0100E5BEC5B
:109A600056F08FEC56F003E0AFEC56F0FDE13F0E00
:109A70000016E9EC56F0CDEC57F0380EEE5C000E17
:109A8000EE58000EEE58000EEE580DE2380E046E41
:109A9000056A066A076AA6EC58F095EC56F0026E65
:109AA000EE50075813D0780E086E096A0A6A0B6ADE
:109AB000A6EC58F0EEEC58F0085C006EEE50095839
:109AC000016EEE500A58026EEE500B58036EEAEC2F
:109AD00057F00C0EDBCFE6FF0D0EDBCFE6FF000EDE
:109AE000E66E0B0EE66E83EC56F0D8EC56F0080EE0
:109AF000E66EE66AD9CFE6FFDACFE6FF83EC56F0F2
:109B0000D8EC56F0100EA9EC56F07AEC56F0FD0E9B
:109B1000DBCFE6FFFE0EDBCFE6FFCEEC56F0100EFD
:109B2000E15C02E2E16AE5528AEF56F0D4EC56F0CD
:109B300019EC55F0EECFDFFF010EEECFDBFF020E8A
:109B4000EECFDBFF030EEECFDBFF040EBFEC57F0D2
:109B5000040EEECFDBFF050EEECFDBFF060EEECFE1
:109B6000DBFF070EEECFDBFF080EBFEC57F0080E51
:109B7000EECFDBFF090EEECFDBFF0A0EEECFDBFFF1
:109B80000B0EEECFDBFF0C0EBFEC57F00C0EEECF42
:109B9000DBFF0D0EEECFDBFF0E0EEECFDBFF0F0E69
:109BA000EECFDBFF400EE66EE66AE66AE66A83EC1D
:109BB00056F0A20EE66E0A0EE66E8FEC53F0006EC3
:109BC000080EE15E005033EC57F07AEC55F0780E59
:109BD0000026A40E01226A0E0222D70E69EC58F06C
:109BE00003E0BFEC54F0FDE191EC54F0190EAEEC43
:109BF00054F0FDE1EDEC56F087EC55F0560E0026E2
:109C0000B70E0122C70E0222E80EDBEC58F003E08B
:109C1000BFEC54F0FDE1A1EC54F0140EAEEC54F0A6
:109C2000FDE108EC57F094EC55F0DB0E0026700EC9
:109C30000122200E0222240EAEEC58F003E0BFEC0D
:109C400054F0FDE184EC54F00F0EAEEC54F0FDE165
:109C500020EC57F0A1EC55F0EE0E0026CE0E0122BE
:109C6000BD0E0222C10EDFEC58F003E0BFEC54F051
:109C7000FDE194EC54F00A0EAEEC54F0FDE1E3EC9F
:109C800058F0AEEC55F0AF0E00260F0E01227C0E00
:109C90000222F50E69EC58F003E0BFEC54F0FDE150
:109CA00091EC54F0190EAEEC54F0FDE1EDEC56F0F1
:109CB000BBEC55F02A0E0026C60E0122870E0222AA
:109CC000470EDBEC58F003E0BFEC54F0FDE1A1ECF3
:109CD00054F0140EAEEC54F0FDE108EC57F0C8EC73
:109CE00055F0130E0026460E0122300E0222A80E59
:109CF000AEEC58F003E0BFEC54F0FDE184EC54F01E
:109D00000F0EAEEC54F0FDE120EC57F0D5EC55F021
:109D1000002A950E0122460E7BEC58F0160E1F0B02
:109D200003E0BFEC54F0FDE194EC54F00A0EAEEC0D
:109D300054F0FDE1E3EC58F0E2EC55F0D80E0026CB
:109D4000980E0122800E0222690E69EC58F003E0A1
:109D5000BFEC54F0FDE191EC54F0190EAEEC54F070
:109D6000FDE1EDEC56F0EFEC55F0AF0E0026F70EEE
:109D70000122440E02228B0EDBEC58F003E0BFEC14
:109D800054F0FDE1A1EC54F0140EAEEC54F0FDE102
:109D900008EC57F0FCEC55F0B10E00265B0E0122EA
:109DA000FF0E0222AEEC58F003E0BFEC54F0FDE1F0
:109DB00084EC54F00F0EAEEC54F0FDE120EC57F0C3
:109DC00009EC56F0BE0E0026D70E01225C0E0222D0
:109DD000890EDFEC58F003E0BFEC54F0FDE194ECA9
:109DE00054F00A0EAEEC54F0FDE1E3EC58F016EC42
:109DF00056F0220E0026110E0122900E02226B0E4A
:109E000069EC58F003E0BFEC54F0FDE191EC54F044
:109E1000190EAEEC54F0FDE1EDEC56F023EC56F0EB
:109E2000930E0026710E0122980EE4EC56F00C0FF2
:109E30005EEC54F0E0EC54F00C0E1F0B03E0BFECB2
:109E400054F0FDE1A1EC54F0140EAEEC54F0FDE141
:109E500008EC57F030EC56F08E0E0026430E01222F
:109E6000790E0222A60EAEEC58F003E0BFEC54F0DF
:109E7000FDE184EC54F00F0EAEEC54F0FDE120EC6B
:109E800057F03DEC56F0210E0026080E0122B40ECC
:109E90000222490EDFEC58F003E0BFEC54F0FDE184
:109EA00094EC54F00A0EAEEC54F0FDE154EC57F093
:109EB00087EC55F0620E0026250E01221E0E0222AE
:109EC000F60E6DEC58F003E0BFEC54F0FDE191ECC0
:109ED00054F01B0EAEEC54F0FDE170EC57F0C8EC02
:109EE00055F0400E0026B30E0122400E0222C00E95
:109EF000B2EC58F003E0BFEC54F0FDE1A1EC54F0FB
:109F0000170EAEEC54F0FDE147EC57F009EC56F0BB
:109F1000510E00265A0E01225E0E0222260EB6ECCB
:109F200058F003E0BFEC54F0FDE184EC54F0120E65
:109F3000AEEC54F0FDE15CEC57F07AEC55F0AA0E73
:109F40000026C70E0122B60E0222E90EBAEC58F026
:109F500003E0BFEC54F0FDE194EC54F00C0EAEECD9
:109F600054F0FDE154EC57F0BBEC55F05D0E0026CB
:109F7000100E01222F0E0222D60E6DEC58F003E0D7
:109F8000BFEC54F0FDE191EC54F01B0EAEEC54F03C
:109F9000FDE170EC57F0FCEC55F0530E0026140E6A
:109FA0000122440E0222020EB2EC58F003E0BFEC94
:109FB00054F0FDE1A1EC54F0170EAEEC54F0FDE1CD
:109FC00047EC57F03DEC56F0810E0026E60E0122DC
:109FD000A10E0222D80EB6EC58F003E0BFEC54F00C
:109FE000FDE184EC54F0120EAEEC54F0FDE15CECBB
:109FF00057F0AEEC55F0C80E0026FB0E0122D30E32
:10A000000222E70EBAEC58F003E0BFEC54F0FDE199
:10A0100094EC54F00C0EAEEC54F0FDE154EC57F01F
:10A02000EFEC55F0E60E0026CD0E0122E10E0222E5
:10A03000210E6DEC58F003E0BFEC54F0FDE191EC23
:10A0400054F01B0EAEEC54F0FDE170EC57F030EC28
:10A0500056F0D60E0026070E0122370E0222C30E3E
:10A06000B2EC58F003E0BFEC54F0FDE1A1EC54F089
:10A07000170EAEEC54F0FDE147EC57F0A1EC55F0B3
:10A08000870E00260D0E0122D50E0222F40EB6EC2C
:10A0900058F003E0BFEC54F0FDE184EC54F0120EF4
:10A0A000AEEC54F0FDE15CEC57F0E2EC55F0ED0E57
:10A0B0000026140E01225A0E0222450EBAEC58F068
:10A0C00003E0BFEC54F0FDE194EC54F00C0EAEEC68
:10A0D00054F0FDE154EC57F023EC56F0050E002649
:10A0E000E90E0122E30E0222A90E6DEC58F003E006
:10A0F000BFEC54F0FDE191EC54F01B0EAEEC54F0CB
:10A10000FDE170EC57F094EC55F0F80E0026A30E2C
:10A110000122EF0E0222FC0EB2EC58F003E0BFEC7D
:10A1200054F0FDE1A1EC54F0170EAEEC54F0FDE15B
:10A1300047EC57F0D5EC55F0D90E0026020E01225F
:10A140006F0E0222670EB6EC58F003E0BFEC54F03D
:10A15000FDE1DADB120EAEEC54F0FDE15CEC57F001
:10A1600016EC56F08A0E00264C0E01222A0E022210
:10A170008D0EBAEC58F003E0BFEC54F0FDE1D4DBF7
:10A180000C0EECDBFEE18BEC57F0BBEC55F0420E15
:10A190000026390E0122FA0E0222FF0E71EC58F051
:10A1A00002E0EDDBFEE1BDDB1C0ED8DBFEE1A3EC43
:10A1B00057F0E2EC55F0810E0026F60E0122710EEA
:10A1C0000222870EBEEC58F002E0D9DBFEE1B9DBDB
:10A1D000150EC4DBFEE192EC57F009EC56F0220EAE
:10A1E0000026610E01229D0E02226D0EC2EC58F077
:10A1F00002E0C5DBFEE188DB100EB0DBFEE1ABEC7C
:10A2000057F030EC56F00C0E0026380E0122E50E09
:10A210007BEC58F0170E1F0B02E0B1DBFEE184DB94
:10A22000090E9CDBFEE18BEC57F087EC55F0440EF9
:10A230000026EA0E0122BE0E0222A40E71EC58F096
:10A2400002E09DDBFEE16DDB1C0E88DBFEE1A3EC92
:10A2500057F0AEEC55F0A90E0026CF0E0122DE0E0F
:10A2600002224B0EBEEC58F002E089DBFEE169DB16
:10A27000150E74DBFEE192EC57F0D5EC55F0600E54
:10A2800000264B0E0122BB0E0222F60EC2EC58F045
:10A2900002E075DBFEE138DB100E60DBFEE1ABECCB
:10A2A00057F0FCEC55F0700E0026BC0E0122BF0EDC
:10A2B0000222BE0EE7EC58F002E061DBFEE134DB87
:10A2C000090E4CDBFEE18BEC57F023EC56F0C60E8A
:10A2D00000267E0E01229B0E0222280E71EC58F001
:10A2E00002E04DDBFEE11DDB1C0E38DBFEE1A3ECE2
:10A2F00057F07AEC55F0FA0E0026270E0122A10E37
:10A300000222EA0EBEEC58F002E039DBFEE119DB76
:10A31000150E24DBFEE192EC57F0A1EC55F0850E12
:10A320000026300E0122EF0E0222D40EC2EC58F0AD
:10A3300002E025DBFEE1E8DA100E10DBFEE1ABEC1B
:10A3400057F0C8EC55F0050E00261D0E0122880EB0
:10A350000222040EE7EC58F002E011DBFEE1E4DA41
:10A36000090EFCDAFEE18BEC57F0EFEC55F0390EFC
:10A370000026D00E0122D40E0222D90E71EC58F024
:10A3800002E0FDDAFEE1CDDA1C0EE8DAFEE1A3EC34
:10A3900057F016EC56F0E50E0026990E0122DB0E62
:10A3A0000222E60EBEEC58F002E0E9DAFEE1C9DA7C
:10A3B000150ED4DAFEE192EC57F03DEC56F0F80EB3
:10A3C00000267C0E0122A20E02221F0EC2EC58F0C3
:10A3D00002E0D5DAFEE198DA100EC0DAFEE1ABEC6D
:10A3E00057F0A2DB650E0026560E0122AC0E0222AB
:10A3F000C40EE7EC58F002E0C2DAFEE195DA090E8D
:10A40000ADDAFEE179EC57F075DB440E0026220E42
:10A410000122290E0222F40E76EC58F002E0AFDAA7
:10A42000FEE17FDA1A0E9ADAFEE164EC57F0BDDB4A
:10A43000970E0026FF0E01222A0E0222430EC6ECC2
:10A4400058F002E09CDAFEE17CDA160E87DAFEE1D3
:10A4500099EC57F030EC56F0A70E0026230E01229F
:10A46000940E0222AB0ECAEC58F002E088DAFEE14C
:10A470004BDA110E73DAFEE182EC57F07CDB390E19
:10A480000026A00E0122930E0222FC0ECEEC58F004
:10A4900002E075DAFEE148DA0B0E60DAFEE179ECF3
:10A4A00057F0C4DBC30E0026590E01225B0E0222B8
:10A4B000650E76EC58F002E062DAFEE132DA1A0E4E
:10A4C0004DDAFEE164EC57F03CDB920E0026CC0E38
:10A4D00001220C0E02228F0EC6EC58F002E04FDA79
:10A4E000FEE12FDA160E3ADAFEE199EC57F084DB42
:10A4F0007D0E0026F40E0122EF0E0222FF0ECAECA2
:10A5000058F002E03CDAFEE1FFD9110E27DAFEE155
:10A5100082EC57F0FCDAD10E00265D0E0122840E8B
:10A520000222850ECEEC58F002E029DAFEE1FCD9D9
:10A530000B0E14DAFEE179EC57F044DB4F0E0026E7
:10A540007E0E0122A80E02226F0E76EC58F002E079
:10A5500016DAFEE1E6D91A0E01DAFEE164EC57F0F4
:10A560008CDBE00E0026E60E01222C0E0222FE0EEF
:10A57000C6EC58F002E003DAFEE1E3D9160EEED99C
:10A58000FEE199EC57F004DB140E0026430E012285
:10A59000010E0222A30ECAEC58F002E0F0D9FEE14F
:10A5A000B3D9110EDBD9FEE182EC57F04CDBA10EE2
:10A5B0000026110E0122080E02224E0ECEEC58F09B
:10A5C00002E0DDD9FEE1B0D90B0EC8D9FEE179EC8D
:10A5D00057F0C4DA820E00267E0E0122530E0222AC
:10A5E000F70E76EC58F002E0CAD9FEE19AD91A0EBD
:10A5F000B5D9FEE164EC57F00CDB350E0026F20E07
:10A6000001223A0E0222BD0EC6EC58F002E0B7D984
:10A61000FEE197D9160EA2D9FEE199EC57F084DA43
:10A62000BB0E0026D20E0122D70E02222A0ECAEC41
:10A6300058F002E0A4D9FEE167D9110E8FD9FEE1EE
:10A6400082EC57F0CCDA910E0026D30E0122860E52
:10A650000222EB0ECEEC58F002E091D9FEE164D973
:10A660000B0E7CD9FEE10BD9E4D92AEC58F0040E8C
:10A67000BFEC57F011EC58F0080EBFEC57F004ECAB
:10A6800058F00C0EBFEC57F0F7EC57F0100EE15CF1
:10A6900002E2E16AE5523ED312DBFCDA3AE2DFCFB6
:10A6A00006F0010EDBCF07F0D89006360736D890BB
:10A6B00006360736FB0EDB5006247DEC58F00720EB
:10A6C000EA6EEECF02F00250E66E47EC58F0B8D9D1
:10A6D000080E44D9FEE10450E66E010EB3EC57F0CB
:10A6E000AFD9100E3BD9FEE10450E66E020EB3EC7A
:10A6F00057F0A6D9180E32D9FEE10450E66E030ECB
:10A70000B3EC57F0E1EC57F0E552E750EF6EE4DAC6
:10A71000C4D7080EE15C02E2E16AE552FBD2CFDA6F
:10A72000B9DA01E3A2D022DB7DEC58F00720EA6E13
:10A73000EFCF02F0036A046A056A010E0C6E0D6A1F
:10A740000E6A0F6A9DEC58F0EE500C26EE500D226A
:10A75000EE500E22EE500F22FB0EDB500C247DEC4F
:10A7600058F00D20EA6EEFCF08F0096A0A6A0B6A0A
:10A77000080E1F0B02E004DBFEE108500212095034
:10A7800003120A5004120B500512020E146E156AC1
:10A79000166A176A9DEC58F0EE501426EE501522FA
:10A7A000EE501622EE501722FB0EDB5014247DECE7
:10A7B00058F01520EA6EEFCF10F0116A126A136A92
:10A7C000100E1F0B07E0D8901036113612361336D4
:10A7D000E806F9E11050021211500312125004124F
:10A7E00013500512030E1C6E1D6A1E6A1F6A9DEC33
:10A7F00058F0EE501C26EE501D22EE501E22EE5058
:10A800001F22FB0EDB501C247DEC58F01D20EA6E4D
:10A81000EFCF18F0196A1A6A1B6A180E1F0B07E0AF
:10A82000D890183619361A361B36E806F9E1185052
:10A830000212195003121A5004121B500512DFCFD6
:10A8400000F0010EDBCF01F0D89000360136D89031
:10A8500000360136B6DB02C0EEFF03C0EEFF04C0D7
:10A86000EEFF05C0EEFF38DA5BD7080EE15C02E2CE
:10A87000E16AE5524FD288DB90DBF7EF57F084DBDB
:10A88000040E00C0DBFF050E01C0DBFF060E02C098
:10A89000DBFF070E03C0DBFF9DEC58F004EF58F020
:10A8A00073DB98DBD2EC58F0DACFEAFF2AEF58F0EE
:10A8B0006BDBC4DBA1EC58F011EF58F0E96EDACF96
:10A8C000EAFF57EF58F0DACFEAFF0C50EE14086EAB
:10A8D0000D50EE14096E0E50EE140A6E0F50EE1469
:10A8E0000B6EC4D303220050DE260150DE2202503C
:10A8F000DE220350DD22DD52DD52A1EC58F096EC51
:10A9000058F0EFCF03F01200080EDBCF04F0090E71
:10A91000DBCF05F00A0EDBCF06F00B0EDBCF07F026
:10A920001200A1EC58F0BAD3040EDBCF04F0050EF0
:10A93000DBCF05F0060EDBCF06F0070EDBCF07F00E
:10A9400012000C0EDBCF04F00D0EDBCF05F00E0E67
:10A95000DBCF06F00F0EDBCF07F01200D8900732E6
:10A96000063205320432E8061200EEEC58F0081602
:10A97000EE500916EE500A16EE500B1677D3D8900B
:10A980000036013602360336E8061200EEEC58F0C7
:10A990000416EE500516EE500616EE50071612007D
:10A9A000DACFEAFF0850EE18046E0950EE18056E73
:10A9B0000A50EE18066E0B50EE18076E0450120087
:10A9C0000C0EDBCF00F00D0EDBCF01F00E0EDBCF57
:10A9D00002F00F0EDBCF03F01200080EDBCF00F009
:10A9E000090EDBCF01F00A0EDBCF02F00B0EDBCF3E
:10A9F00003F012004CDB81EF58F0F0DB041AEE504C
:10AA0000051AEE50061AEE50071A04501200E6DB43
:10AA1000081AEE50091AEE500A1AEE500B1A1200DC
:10AA2000DDDB0412EE500512EE500612EE50071256
:10AA30001200FD0EDBCFE9FFFE0EDBCFEAFF1200B6
:10AA4000C0DAE552E750EF6EDFCF08F0010EDBCF42
:10AA500009F0D89008360936D89008360936FB0E2A
:10AA6000DB5008244ADB0920EA6E18D30C0EDBCF3A
:10AA700008F00D0EDBCF09F00E0EDBCF0AF00F0E43
:10AA8000DBCF0BF01200080EDBCF08F0090EDBCF96
:10AA900009F00A0EDBCF0AF00B0EDBCF0BF0120031
:10AAA000040EDBCF08F0050EDBCF09F0060EDBCF7E
:10AAB0000AF0070EDBCF0BF0120043DBEECF08F0FD
:10AAC000EECF09F0EECF0AF0EFCF0BF01200DBCFA4
:10AAD0000FF00C1E0D1E0E1E0F1E1200081E091E6A
:10AAE0000A1E0B1ED9501200041E051E061E071E4C
:10AAF000D95012000A01A225006E0550A321016E53
:10AB00000650A421026E0750A521036E12000A010F
:10AB1000A625006E0550A721016E0650A821026EE1
:10AB20000750A921036E12000A01AA25006E0550E4
:10AB3000AB21016E0650AC21026E0750AD21036EB1
:10AB400012000A01AE25006E0550AF21016E0650BD
:10AB5000B021026E0750B121036E12000A01B22526
:10AB6000006E0550B321016E0650B421026E0750ED
:10AB7000B521036E12000A01B625006E0550B721FB
:10AB8000016E0650B821026E0750B921036E120003
:10AB90000A01BA25006E0550BB21016E0650BC218A
:10ABA000026E0750BD21036E12000A01BE25006E21
:10ABB0000550BF21016E0650C021026E0750C12111
:10ABC000036E12000A01C225006E0550C321016EFA
:10ABD0000650C421026E0750C521036E12000A01FF
:10ABE000C625006E0550C721016E0650C821026EB1
:10ABF0000750C921036E12000A01CA25006E0550D4
:10AC0000CB21016E0650CC21026E0750CD21036E80
:10AC100012000A01CE25006E0550CF21016E0650AC
:10AC2000D021026E0750D121036E12000A01D225F5
:10AC3000006E0550D321016E0650D421026E0750DC
:10AC4000D521036E12000A01D625006E0550D721CA
:10AC5000016E0650D821026E0750D921036E1200F2
:10AC60000A01DA25006E0550DB21016E0650DC2159
:10AC7000026E0750DD21036E12000A01DE25006E10
:10AC80000550DF21016E0650E021026E0750E121E0
:10AC9000036E1200F70EDBCF00F0F80EDBCF01F0F1
:10ACA000EFD94BDA0050EE5C0150EE580250EE58EE
:10ACB0000350EE581200E926000EEA22120004DAD0
:10ACC000080EE12625DA040EDB6A050EDB6A060EA5
:10ACD000DB6A070EDB6A120034DAEE2A000EEE227F
:10ACE000EE22EE222ADA040EEE26000EEE22EE22EC
:10ACF000EE221200E9CF00F0EACF01F0E9CFE6FF43
:10AD0000EACFE6FF1200FB0EDBCFE6FFFC0EDBCF47
:10AD1000E6FF1200E16EE552E7CFD9FF12000450C2
:10AD20001F0B04DAEECF03F0120058DA045C006E59
:10AD3000EE500558016EEE5006581200E9CFE6FFBE
:10AD4000EACFE6FF96EC4DF0E552E552E552E552CA
:10AD50001200E66EE66AE66AE66A8FEF58F0D8906F
:10AD60000332023201320032E8061200040EDBCF59
:10AD700006F0050EDBCF07F0FB0EDB5006241200B9
:10AD8000D890083609360A360B36E8061200F90E56
:10AD9000DBCF00F0FA0EDBCF01F012007DDC026E9B
:10ADA000080EE15E025012008FD9100EE12612004B
:10ADB000EDEC4BF0006E060EE15E00501200016EED
:10ADC00000C0E6FFE66E12000222FD0E0322D950FB
:10ADD0001200016A026A036A12006ADDA5DDD9CF9A
:10ADE000E9FFD4DDAED9EECF0CF0EECF0DF0EECF13
:10ADF0000EF0EFCF0FF00C1E0D1E0E1E0F1EA6D96B
:10AE000063EF54F00322D950080F58DDEDEF54F0F2
:10AE100047DD87DDC7D9BADD0C0EDBCF0CF00D0E98
:10AE2000DBCF0DF00E0EDBCF0EF00F0E50DEDAD9B9
:10AE300063EF54F00322D9500C0F40DDE0EF54F0E3
:10AE40001ADD7FDD83D9A2DD080EDBCF0CF0090E01
:10AE5000DBCF0DF00A0EDBCF0EF00B0E38DED9CFB4
:10AE6000E9FF63EF54F050DDBDD990DD040EDBCF78
:10AE70000CF0050EDBCF0DF0060EDBCF0EF0070E4B
:10AE800026DE90D963EF54F00322D9508FD108DD2C
:10AE90004BDD88D97BDD04DE081E091E0A1E0B1E51
:10AEA000D9CFE9FFB5EF54F0EADC4BDD9BD96EDD7D
:10AEB000DDDD14DE080F8FD1DEDC33DD47D966DD42
:10AEC000FCDD0CDE0C0F87D1F3DC1EDD041E051E3D
:10AED000061E071ED9CFE9FFA3DD84D9FDEF54F08C
:10AEE000E7DC12DDD9CFE9FF51DDCDDDF7DD040F61
:10AEF00072D1C5DC26DDF8DD040FE96E91DD26D9BF
:10AF0000FDEF54F0B8DC0DDDEFDD080FE96E88DDF4
:10AF100049D9FDEF54F0B3DCB6DD64D978DD42D910
:10AF2000D0EF54F0BDDCC9DD3DD971DD5BD9D0EF88
:10AF300054F0B6DCF9DCD8DD0C0FE96E71DDD9CF49
:10AF4000E9FFFDEF54F0B4DCABDDD9CFE9FF5FDD05
:10AF5000FDD8D0EF54F08FDC89DDF8D858DDD9CF9B
:10AF6000E9FFD0EF54F0006E34DFE7D8EE50002652
:10AF7000EE500122EE500222EE5003221200E76E44
:10AF800058DDE7505BEF56F00450001205500112F7
:10AF900006500212075003121200080E00C0DBFF19
:10AFA000090E01C0DBFF0A0E02C0DBFF0B0E03C05F
:10AFB000DBFFCCD8DACFEAFF12003BDD100E5BEFEF
:10AFC00056F0FD0EDB500024E96EFE0EDB50012032
:10AFD000EA6E12000C0E00C0DBFF0D0E01C0DBFF9D
:10AFE0000E0E02C0DBFF0F0E03C0DBFF12000C0EC3
:10AFF000DB50EE260D0EDB50EE220E0EDB50EE2265
:10B000000F0EDB50EE221200080EDB50EE26090E6A
:10B01000DB50EE220A0EDB50EE220B0EDB50EE224E
:10B020001200040EDB50EE26050EDB50EE22060E5B
:10B03000DB50EE22070EDB50EE22120000C0DFFFD5
:10B04000010E01C0DBFF020E02C0DBFF030E03C0D6
:10B05000DBFF1200DF50EE26010EDB50EE22020E67
:10B06000DB50EE22030EDB50EE22120008500412D9
:10B07000095005120A5006120B5007120450120014
:10B08000F90EDBCF02F0FA0EDBCF03F01200040E54
:10B09000DBCF00F0050EDBCF01F01200EECF04F0A5
:10B0A000EECF05F0EECF06F0EFCF07F01200005024
:10B0B000EE260150EE220250EE220350EE22120044
:10B0C000B8DC180E5BEF56F0D9CFE6FFE1CFD9FF21
:10B0D000120008DC070E1F0B120004DC050E1F0B0C
:10B0E000120072EC54F0040E1F0B120072EC54F0BC
:10B0F000060E1F0B120068DE59D0E96EFC0EDB5005
:10B100001200060EDBCF02F0070EDBCF03F01200B9
:10B11000DE6ADE6ADE6ADD6ADD52DD521200FB0E97
:10B12000DBCFE9FFFC0EDBCFEAFF1200EECF00F031
:10B13000EECF01F0EECF02F0120054D8DACFEAFFE2
:10B140001200D9CFE9FFDACFEAFF1200D950080F79
:10B15000E96E120032DF040E5BEF56F053DE110E83
:10B160001F0B120067DE090E1F0B12004BDE0E0EC6
:10B170001F0B120089DE140E1F0B12005BDE0B0E7C
:10B180001F0B12003FDE100E1F0B120053DE0A0EC3
:10B190001F0B120037DE0F0E1F0B120075DE150E8F
:10B1A0001F0B1200D9500C0FE96E1200040F5EEC59
:10B1B00054F0FAEF54F03EDE0C0E1F0B120064DE6A
:10B1C000160E1F0B12003FEC54F033EF57F05CDE0D
:10B1D000170E1F0B1200E96EB5EF54F0DACFEAFF3D
:0CB1E000EE501200D950040FE96E12006E
:04B1EC00F9EC62F028
:10B1F000B8EC64F009E10901080EFC6FE00EFD6F88
:10B20000000E56EC63F017D00901FE0EFC6FDF0E46
:10B21000FD6F000E56EC63F020EC64F09EEC64F0E1
:10B220000901FA0EFC6FDF0EFD6F000E56EC63F0A5
:10B23000020E6FEC63F0FEEF62F0B8EC64F003E135
:10B2400004EC64F006D00901F50EFC6FDF0EFD6F13
:10B25000000E56EF63F0F9EC62F00501F3B50BD088
:10B26000E3EC62F0FBCAFCF9FCCAFDF9FDCAFEF989
:10B2700054EC3EF0E2DFFEEF62F0F9EC62F0050123
:10B28000F3B509D0E3EC62F0FECAE6FFFFCAE6FFC1
:10B290009EEC64F0D2DFFEEF62F048EC64F0F3A5C0
:10B2A00002D0000E11D00CEC65F0EAEC64F087ECF3
:10B2B00037F0E552E552EAEC64F0C6EC74F0E55282
:10B2C000E55202EC63F0010E9AEC63F002E2E16AEF
:10B2D000E552E16E0050FEEF62F048EC64F0F3B529
:10B2E00009D02EEC65F09B0EFC6F340EFD6F010E45
:10B2F000DBEC64F0020EE15C02E2E16AE552E16E31
:10B30000FEEF62F048EC64F0F3B509D02EEC65F086
:10B31000B60EFC6F340EFD6F010EDBEC64F0020E16
:10B32000E15C02E2E16AE552E16EFEEF62F04EECB2
:10B3300064F00A0E0CEC65F00901A051E66EE66AB5
:10B34000CC0EE66EDF0EE66E000E58EC64F029ECD3
:10B3500063F0C50EE66EDF0EE66E000E5BEC64F089
:10B3600002E2E16AE552E16EFEEF62F04EEC64F05B
:10B370000A0E0CEC65F00701CAA308D038EC63F0A4
:10B380009E0EE66EDF0EE66E000E07D038EC63F020
:10B39000860EE66EDF0EE66E000E34EC65F004EC11
:10B3A00065F085EC63F07E0EE66EDF0EE66E000E55
:10B3B00043EC63F07B0EE66EDF0EE66E000E5BEC98
:10B3C00064F002E2E16AE552E16EFEEF62F04EECFB
:10B3D00064F0E66A66EC63F090EC63F0FD0EDBCFA0
:10B3E000E6FFFE0EB2EC63F002E1010E06D00501AD
:10B3F000F3B302D074EC63F0000E9AEC63F002E257
:10B40000E16AE552E16E0050FEEF62F01BEC65F080
:10B41000D950FB0FEFEC64F00BE090EC63F0FB0E07
:10B42000DBCFE6FFFC0EB2EC63F002E1010E06D0CA
:10B430000501F3B302D074EC63F0000E9AEC63F0F4
:10B4400002E2E16AE552E16E0050FEEF62F0F9ECD3
:10B4500062F0D8EC63F021E0BFEC64F0DEEC64F065
:10B4600020EC64F0A3EC98F017EC65F0E7CF01F066
:10B47000E552E7CF00F00050F3240A01F96F0150C4
:10B48000F420FA6FF9CA00F0016EFD0EDB500018CF
:10B4900007E1FE0EDB50011803E1F36AF46A16D0EF
:10B4A000FD0E10EC64F0BCEC64F008E02CEC63F0F2
:10B4B00005E0DF2A010EF7E3DB2AF5D7BCEC64F0E8
:10B4C00003E189EC64F0EF6ADEEC63F0020EE15C0C
:10B4D00002E2E16AE552E16EFEEF62F0F9EC62F041
:10B4E000D8EC63F016E0FD0E10EC64F02CEC63F089
:10B4F00005E0DF2A010EFAE3DB2AF8D7DECF00F001
:10B50000DDCF01F00A01F951001806E1FA510118E6
:10B5100003E1F36AF46A21D0DF2A010E01E3DB2A9A
:10B52000D9CFE9FFDACFEAFFFD0EEECFDBFFFE0E4B
:10B53000EDCFDBFFBCEC64F008E02CEC63F005E041
:10B54000DF2A010EF7E3DB2AF5D7BCEC64F003E158
:10B5500089EC64F0EF6ADEEC63F0020EE15C02E27B
:10B56000E16AE552E16EFEEF62F04EEC64F0E66AED
:10B5700066EC63F00501F3A502D0000E0BD0E3ECFE
:10B5800062F027EC64F0670EE66EDF0EE66E000EEA
:10B590002CEC64F09AEC63F002E2E16AE552E16EB1
:10B5A0000050FEEF62F0F9EC62F020EC64F0E66A25
:10B5B0000BEC64F0F3A502D0000E0AD04BEC64F063
:10B5C0005E0EFC6F330EFD6F010E56EC63F0010E44
:10B5D000FEEF62F01BEC65F00501F3A502D0000E52
:10B5E0000BD0E3EC62F027EC64F0550EE66EDF0E54
:10B5F000E66E000E2CEC64F09AEC63F002E2E16A75
:10B60000E552E16E0050FEEF62F0F9EC62F015ECED
:10B6100064F0010EE66E0BEC64F0F3A502D0000EB0
:10B620000AD04BEC64F08B0EFC6F330EFD6F010EF5
:10B6300056EC63F0010EFEEF62F048EC64F0F3A507
:10B6400002D0000E27D00CEC65F0D1C9E6FFD2C9BC
:10B65000E6FFD3C9E6FFD4C9E6FFDA0EE66E340E84
:10B66000E66E010E34EC65F0E4EC63F0D5C9E6FF5C
:10B67000D6C9E6FFD7C9E6FFD8C9E6FF530EE66E86
:10B68000DF0EE66E000E31EC65F0E4EC63F002ECE8
:10B6900063F0010E9AEC63F002E2E16AE552E16EBA
:10B6A0000050FEEF62F0F9EC62F020EC64F0F5DDA2
:10B6B000E552E552FEEF62F0F9EC62F0070EE1268A
:10B6C0000501F3A502D0000E70D04BEC64F0A3ECA2
:10B6D00064F0070EF36E020EF3CFDBFFDF6A200E7D
:10B6E000DF5C62E2DFCFE6FF83EC9FF0E552030E02
:10B6F000F3CFDBFF040EF4CFDBFF030EDBCFE9FF5C
:10B70000040EDBCFEAFFEF504DE0DFCFE6FFE66A45
:10B71000490EE66EDF0EE66E000E58EC64F0ECECBF
:10B7200063F0030EDBCFE6FF040EDBCFE6FF470E30
:10B73000E66EDF0EE66E000EE66E050EDBCFE6FF70
:10B74000060EDBCFE6FF01EC75F0ECEC63F0050EC6
:10B75000DBCF00F0060EDBCF01F0000E005E060E20
:10B76000015A010E00C0DBFFDBCFE6FF020EDB500B
:10B77000E552E724006E016A013412E20050A0088D
:10B78000000E01540DE259DD140E2EEC65F0A3EC11
:10B7900064F0010EDB50070FE76E020EE7CFDBFF10
:10B7A00002EC63F0DF2A9BD7010E006E070EE15C0E
:10B7B00002E2E16AE552E16E0050FEEF62F0F9EC60
:10B7C00062F0E652020EDF6E200EDF5C11E21CEC2E
:10B7D00064F00EE06BEC63F006E12FEC63F003E144
:10B7E00010EC63F002D015EC64F059EC63F0ECD788
:10B7F0004BEC64F0AD0EFC6F330EFD6F010EDBEC15
:10B8000064F007EC93F0B8EC64F002E0ACEC63F0A9
:10B81000000EE552FEEF62F0E3EC64F0DF6A010E29
:10B82000E66E83EC9FF0E55200EC65F0200EDF5CE5
:10B8300011E21CEC64F00EE06BEC63F006E12FEC1F
:10B8400063F003E110EC63F002D015EC64F059EC06
:10B8500063F0ECD7B8EC64F004E0E66AB7EC3FF0D4
:10B86000E552000E006E030EE15C02E2E16AE55271
:10B87000E16E0050FEEF62F048EC64F0F3A502D0F8
:10B88000000E34D0E3EC62F03F0EE66EDF0EE66EA3
:10B89000000E1EEC63F0080EF5EC62F0310EE66E61
:10B8A000DF0EE66E000EF1EC62F00E0EF5EC62F0CB
:10B8B000210EE66EDF0EE66E000EF1EC62F0020E77
:10B8C000F5EC62F0170EE66EDF0EE66E000EF1ECA0
:10B8D00062F0030EF5EC62F0050EE66EDF0EE66E2A
:10B8E000000EF1EC62F002EC63F0010E9AEC63F0F2
:10B8F00002E2E16AE552E16E0050FEEF62F0E7EC31
:10B9000064F0080EE9EC62F011E015EC64F0020E50
:10B91000E9EC62F00BE015EC64F0030EE9EC62F088
:10B9200005E015EC64F00E0E3EEC64F00CEC63F0F8
:10B93000A3DF006E060EE15E0050DF6E07EC93F0B1
:10B94000B8EC64F002E0ACEC63F0DF50E552FEEFDF
:10B9500062F048EC64F0F3A502D0000E56D0E3ECA0
:10B9600062F0FF0EE66EDE0EE66E000E1EEC63F079
:10B97000050EF5EC62F0F70EE66EDE0EE66E000EDA
:10B98000F1EC62F0060EF5EC62F0EE0EE66EDE0E05
:10B99000E66E000EF1EC62F0070E8EEC64F0EC0E39
:10B9A000E66E090EE66ED90EE66EDE0EE66E000E4F
:10B9B00031EC65F001EC75F029EC63F00A015D51A2
:10B9C00006E0B60EE66EDE0EE66E000E19D0200E14
:10B9D0000601C85D06E1930EE66EDE0EE66E000E11
:10B9E0000FD0C851E66EE66A740EE66EDE0EE66EA5
:10B9F000000E12EC65F0720EE66EDE0EE66E000EC4
:10BA0000EDEC62F002EC63F0010E9AEC63F002E2FE
:10BA1000E16AE552E16E0050FEEF62F0E7EC64F09F
:10BA2000050EE9EC62F01DE06BEC63F006E12FEC33
:10BA300063F003E110EC63F002D015EC64F0060E45
:10BA4000E9EC62F00EE06BEC63F006E12FEC63F0E2
:10BA500003E110EC63F002D015EC64F0070E3EEC4D
:10BA600064F00CEC63F075DF9EEC63F002E0ACEC8C
:10BA700063F0DF50E552FEEF62F048EC64F0F3A5AE
:10BA800002D0000E2AD04BEC64F0680EFC6FDE0E84
:10BA9000FD6F000E56EC63F00D0EE66E66EC63F083
:10BAA0002CEC63F007E109015F0EFC6FDE0EFD6F09
:10BAB000000E06D027EC64F09EEC64F004EC64F019
:10BAC00056EC63F0EC0EE66E090EE66E550EE66E71
:10BAD000DE0EE66E000E2CEC64F09AEC63F002E2EF
:10BAE000E16AE552E16E0050FEEF62F04EEC64F068
:10BAF0001CEC64F009E1010EDB6AD950010FE66E1F
:10BB0000000EDA20E66E02D015EC64F00D0E3EEC6D
:10BB100064F00CEC63F0B1DF9EEC63F002E0ACEC9F
:10BB200063F0DF509AEC63F002E2E16AE552E16E05
:10BB30000050FEEF62F048EC64F0F3A502D0000E76
:10BB400023D0E3EC62F04D0EE66EDE0EE66E000EE4
:10BB50001EEC63F0040EF5EC62F0460EE66EDE0EAF
:10BB6000E66E000EF1EC62F0090E8EEC64F00A0E47
:10BB7000F5EC62F0390EE66EDE0EE66E000EF1ECCC
:10BB800062F002EC63F0010E9AEC63F002E2E16A0B
:10BB9000E552E16E0050FEEF62F0E7EC64F0040E57
:10BBA000E9EC62F00BE015EC64F0090EE9EC62F0F0
:10BBB00005E015EC64F00A0E3EEC64F00CEC63F06A
:10BBC000BADF9EEC63F002E0ACEC63F0DF50E552CC
:10BBD000FEEF62F048EC64F0F3A502D0000E9ED0B8
:10BBE000E3EC62F0330EE66EDE0EE66E000E1EEC47
:10BBF00063F00901F751E66EE66A280EE66EDE0E86
:10BC0000E66E000EF6EC64F00901F851E66EE66AA5
:10BC10001D0EE66EDE0EE66E000EF6EC64F006011A
:10BC2000C851E66EE66A0E0EE66EDE0EE66E000E99
:10BC300012EC65F00901EA51000812E238EC63F0F9
:10BC4000020EE66EDE0EE66E000E43EC63F085EC4F
:10BC500063F0FC0EE66EDD0EE66E000E43EC63F064
:10BC60000501F551E66EE66AF10EE66EDD0EE66E52
:10BC7000000EF6EC64F00501F6514DE0E70EE66EBD
:10BC8000DD0EE66E000EEDEC62F00501F6A107D0C8
:10BC9000E20EE66EDD0EE66E000EEDEC62F00501E2
:10BCA000F6A307D0DD0EE66EDD0EE66E000EEDECBF
:10BCB00062F00501F6A507D0D90EE66EDD0EE66E40
:10BCC000000EEDEC62F00501F6A707D0D50EE66E8A
:10BCD000DD0EE66E000EEDEC62F00501F6A907D070
:10BCE000D10EE66EDD0EE66E000EEDEC62F00501A3
:10BCF000F6AB07D0C90EE66EDD0EE66E000EEDEC7B
:10BD000062F00501F6AD07D0C10EE66EDD0EE66EFF
:10BD1000000EEDEC62F002EC63F0010E9AEC63F0C1
:10BD200002E2E16AE552E16E0050FEEF62F0E3EC00
:10BD300064F00501F3A502D0000E2CD04BEC64F0AA
:10BD4000B70EFC6FDD0EFD6F000E56EC63F0DF6A80
:10BD5000100EDF5C1EE2EFEC63F0EF5018E0DFCF77
:10BD6000E6FFE66AB30EE66EDD0EE66E000E81ECCF
:10BD700063F0EFEC63F0EF50E66EE66A470EE66EB6
:10BD8000DF0EE66E000E05EC63F002EC63F0DF2AD6
:10BD9000DFD7010E006E030EE15C02E2E16AE552BC
:10BDA000E16E0050FEEF62F0F9EC62F0E6521CEC3E
:10BDB00064F002E1000E31D0C0EC63F0DF6E0FECF6
:10BDC00065F0000EDF5C28E3100EDF5C25E21CEC62
:10BDD00064F022E0C0EC63F0E66EEFEC63F0E55255
:10BDE000E750EF6E080EDF5C07E315EC64F0080E19
:10BDF000DF5C180F3EEC64F00F0EDF5C02E107EC35
:10BE000093F04BEC64F0C70EFC6F330EFD6F010E28
:10BE100056EC63F0010E01D0000EE552EFD352EC68
:10BE200064F017E0F90EDBCFE6FFFA0EDBCFE6FF9A
:10BE3000180EE66EE66AE66A07D04BCBFBFF4ACBEC
:10BE4000FAFF0B014951F96EF8DF006E050EE15E55
:10BE500000504BEC64F0DD0EFC6F330EFD6F010EF5
:10BE600055EF64F052EC64F017E0F90EDBCFE6FF1B
:10BE7000FA0EDBCFE6FF140EE66EE66AE66A07D03E
:10BE80004BCBFBFF4ACBFAFF0B014951F96EF8DFB0
:10BE9000006E050EE15E00504BEC64F0F00EFC6F9E
:10BEA000330EFD6F010E55EF64F052EC64F017E0B5
:10BEB000F90EDBCFE6FFFA0EDBCFE6FF160EE66EDD
:10BEC000E66AE66A07D04BCBFBFF4ACBFAFF0B01D1
:10BED0004951F96EF8DF006E050EE15E00504BEC43
:10BEE00064F0070EFC6F340EFD6F010E55EF64F029
:10BEF00052EC64F017E0F90EDBCFE6FFFA0EDBCF71
:10BF0000E6FF150EE66EE66AE66A07D04BCBFBFF4E
:10BF10004ACBFAFF0B014951F96EF8DF006E050EAE
:10BF2000E15E00504BEC64F0200EFC6F340EFD6FB0
:10BF3000010E55EF64F052EC64F017E0F90EDBCF20
:10BF4000E6FFFA0EDBCFE6FF170EE66EE66AE66A5C
:10BF500007D04BCBFBFF4ACBFAFF0B014951F96EDF
:10BF6000F8DF006E050EE15E00504BEC64F0350E1C
:10BF7000FC6F340EFD6F010E55EF64F03ADBE150BB
:10BF8000F90FEFEC64F001E18BD015EC64F091EC6B
:10BF900099F0E552E552C9DB01E190D0030EE66E5F
:10BFA000E66AAF0EE66EDD0EE66E000E4BDB12E1CA
:10BFB000AD0EE66EDD0EE66E0A0EE66EE66AE66A27
:10BFC00007D04BCBFBFF4ACBFAFF0B014951F96E6F
:10BFD000F8DF53D0030EE66EE66AA90EE66EDD0EBC
:10BFE000E66E000E2FDB12E1A70EE66EDD0EE66EAA
:10BFF0000A0EE66EE66AE66A07D04BCBFBFF4ACB39
:10C00000FAFF0B014951F96EF8DF37D0030EE66EE7
:10C01000E66AA30EE66EDD0EE66E000E13DB12E19D
:10C02000A10EE66EDD0EE66E0A0EE66EE66AE66AC2
:10C0300007D04BCBFBFF4ACBFAFF0B014951F96EFE
:10C04000F8DF1BD0030EE66EE66A9D0EE66EDD0E8F
:10C05000E66E000EF7DA24E19B0EE66EDD0EE66E6C
:10C060000A0EE66EE66AE66A07D04BCBFBFF4ACBC8
:10C07000FAFF0B014951F96EF8DF006E050EE15E23
:10C0800000500FEC65F0D8DB19E0F90EDBCFE6FFCE
:10C09000FA0EDBCFE6FF0F0EE66EE66AE66A09D01F
:10C0A000000E14D04BCBFBFF4ACBFAFF0B014951DA
:10C0B000F96EF8DF006E050EE15E0050ECDB510E0C
:10C0C000FC6F340EFD6F010EF1DA010E97D2EADB40
:10C0D00014E0000EE66EE66A0B0EE66EE66AE66AAD
:10C0E00007D04BCBFBFF4ACBFAFF0B014951F96E4E
:10C0F000F8DF006E050EE15E00500601F36BCBDB4E
:10C100006E0EFC6F340EFD6F010ECFD3CBDB14E04F
:10C11000000EE66EE66A0C0EE66EE66AE66A07D088
:10C120004BCBFBFF4ACBFAFF0B014951F96EF8DF0D
:10C13000006E050EE15E005006011E0EF36FABDBD4
:10C14000850EFC6F340EFD6F010EAFD3E3EC64F08F
:10C15000010EDF6E020EDF6E0E0EF66E000EF76E33
:10C16000000E44DB830EE66EDD0EE66E000EC9DACD
:10C170000F0EF66E000EF76E000ED8DB100EF66E88
:10C18000000EF76E000ED2DB0E0E2FDA7F0EE66E7B
:10C19000DD0EE66E000EE66EA7DBC6EC64F000EC8A
:10C1A00065F00701CC51CD11CE110AE0CCC7E6FFF6
:10C1B000CDC7E6FFCEC7E6FF97DB9DDB00EC65F061
:10C1C000DFCFE6FFE66A7C0EE66EDD0EE66E000E61
:10C1D0001CDAF9D917DA010E006E030EE15C02E2F7
:10C1E000E16AE552E16E005009D258DB030EE66EBB
:10C1F000B7EC3FF0E552000E9DDA02E2E16AE5524B
:10C20000E16E0050FBD1F5D9FE0EDB50330A0AE097
:10C21000010A05E0030A19E151DA08E009D0B7DAAA
:10C2200014E104D0B4DA11E149DA02E1000E0ED0D3
:10C230004BDB6EEC5AF0E552E552F4CF01F020EC06
:10C2400065F0F3CFEEFF01C0EDFF010ED7D1D1D9DC
:10C25000070EE126FB0EE4DAFFD917E08DDB15E0CF
:10C26000FBD960080DE255DBEFCF00F07B0E005CE0
:10C2700007E2F2D9E00FE66E4CDBE552E750EF6ED5
:10C28000DF2A010EE9E3DB2AE7D776DB04E1DF2AC8
:10C29000010E01E3DB2A020EDB6A030EDB6A55DACC
:10C2A000ABDA04BE0568040E79DAFEE1EFD901E1EC
:10C2B00019D1090E066E350E076E010E086E020EBC
:10C2C000DBCF09F0030EDBCF0AF00B6A0ABE0B6866
:10C2D000040ED89009360A360B36E806FAE1065005
:10C2E0000924036E07500A20046E08500B20056EC7
:10C2F00003C0E6FF04C0E6FFE66EB1EC98F097DB02
:10C3000027C000F028C001F029C002F00006000E8E
:10C31000015A025A53DB090E0F6E350E106E010ED4
:10C32000116E020EDBCF12F0030EDBCF13F0146A96
:10C3300013BE1468040ED890123613361436E8066D
:10C34000FAE10F5012240C6E105013200D6E115094
:10C3500014200E6E0C2A000E0D220E220CC0E6FFD9
:10C360000DC0E6FF0EC0E6FFCDDA91EC97F0156E3A
:10C37000070EE15E1550000901E0ADD0040EDB6A46
:10C3800066DA27EC5AF0E552E55207DBD950050F83
:10C39000E66E000EDA20E66E53DAD7D92DDA04BE47
:10C3A0000568040EFBD9FEE171D9E66E2CDF066E3E
:10C3B000050EE15E0650000901E1BED00B014C51B3
:10C3C0004D114E1124E0050EDBCFE6FF060EDBCF4C
:10C3D000E6FFFB0EDBCFE6FFFC0EDBCFE6FFFD0E3C
:10C3E000DBCFE6FFFE0EDBCFE6FF010EE66E07D0E9
:10C3F0004ECBFBFF4DCBFAFF0B014C51F96EF8DF32
:10C40000006E070EE15E0050000901E095D0020EBB
:10C41000DBCFE9FF030EDBCFEAFFEA02F3CFEAFF4F
:10C42000E902F3CFE9FFF450EA26000EE9260A0EEE
:10C43000EA22EECF00F0EECF01F0EFCF02F0050ED2
:10C44000DBCFE6FF060EDBCFE6FFFB0EDBCFE6FF22
:10C45000FC0EDBCFE6FFFD0EDBCFE6FFFE0EDBCFF3
:10C46000E6FF06D002C0FBFF01C0FAFF0050F96EE4
:10C47000F9DF036E060EE15E0350E76E040EE7CFB0
:10C48000DBFFDB5059E00B014C514D114E1120E008
:10C49000050EDBCFE6FF060EDBCFE6FFFB0EDBCFA4
:10C4A000E6FFFC0EDBCFE6FFFD0EDBCFE6FFFE0E68
:10C4B000DBCFE6FFE66A07D04ECBFBFF4DCBFAFFA2
:10C4C0000B014C51F96EF8DF006E070EE15E005073
:10C4D0001DEC59F031D0020EDB2A030E01E2DFD64B
:10C4E000DB2ADDD60B014F51501151111FE0DECF79
:10C4F000E6FFDDCFE6FFFB0EDBCFE6FFFC0EDBCF7A
:10C50000E6FFFD0EDBCFE6FFFE0EDBCFE6FF07D03A
:10C5100051CBFBFF50CBFAFF0B014F51F96EF8DF07
:10C52000006E060EE15E0050000906E1EBD988D9E5
:10C53000D8EC36F07CDAE552070EE15C02E2E16A03
:10C54000E552E16E5BD0A4D9F3A502D0000E34D041
:10C55000A2D9720EFC6FDD0EFD6F000EA7D8DE6A49
:10C56000DD6AF8D904BE0568040E18D9FEE18ED83C
:10C5700022E00901700EFC6FDD0EFD6F000E96D8F3
:10C58000E9D904BE0568040E09D9FEE10050032470
:10C590000901FC6F01500420FD6F02500520FE6F61
:10C5A000FC2B000EFD23FE2354EC3EF0DF2A010E8F
:10C5B000D8E3DB2AD6D7010EBDD802E2E16AE55204
:10C5C000E16E00501BD03CD9F6EC58F0E552E55234
:10C5D000120054D924DA1CEF64F043DA8CD943EF0B
:10C5E00064F03FDAD3D943EF64F0E66E83EC9FF05A
:10C5F00071D1D9CFE6FFE1CFD9FF1200E552E7CFE5
:10C60000D9FF1200E7D99EEF64F0E66E6DD907EC12
:10C6100075F0F1D900EF65F008D974D920EF64F016
:10C62000010EE76EF90EDBCF00F0FA0EDBCF01F062
:10C63000E7500026000E0122DEEF64F015DA5BD928
:10C6400043EF64F0E66EF1D891EC97F0D4D900098D
:10C650001200D1D943EF64F05CD9EF501200010E03
:10C66000E76EA2D9E750E926000EEA22EF50120049
:10C67000010EE66EE66AEAC900F0016A026A036A20
:10C68000EAC9E6FF6ED1EDD904EF65F0005003244E
:10C69000F36E01500420F46E02500520F86EF4CFC2
:10C6A000F7FFF3CFF6FF0800F5501200FE6F54EFCE
:10C6B0003EF0DF50DF2AE2D80FEF65F005D9C7D989
:10C6C00006EC5AF0B4D9E5520009120083EC9FF051
:10C6D000E55243EF64F068D9EF502D081200E66E82
:10C6E000BFEC72F0E55212000A014C0EFB6F330EE4
:10C6F000FC6F010EFD6FA4D82BEC59F0E552E5520A
:10C700001200D6D878D900EF65F0010EE66EE66A21
:10C71000EBC900F0016A026A036AEBC9E6FF21D1A6
:10C7200096D8A3EC98F0E552D5D00B0149514A11A7
:10C730004B111200006E020EE15C1200006E060E3C
:10C74000E15E0050DF6EB8EF64F0090E006E350E4A
:10C75000016E010E026E1200400EE66EB7EC3FF065
:10C76000E5521200DBCFE6FF72D8D6EC98F0026EED
:10C77000060EE15E025000091200E65215EF64F069
:10C7800054D8DFEC89F0E552E552F35012005FD93E
:10C79000E7EC59F0E552E55200091200D890033653
:10C7A00004360536E8061200020EE12605011200E5
:10C7B000020EE126D950FD0FEFEF64F0E0D800C083
:10C7C000F3FF01C0F4FF120060EC76F0006E090E7A
:10C7D000E15E005043EF64F00ED9CDEF64F0DF501E
:10C7E000EA6AE50FE96E050EEA221200F86E08000B
:10C7F000F550E66EE66A1200020EDBCF03F0030E80
:10C80000DBCF04F0056A12000901F70EFC6FDF0EA2
:10C81000FD6F000E1200CAEC9FF009D9050112004D
:10C82000DBCFDEFFDBCFDDFF1200F90EDBCFE6FF53
:10C83000FA0EDBCFE6FF1200D950F90FEFEF64F0EC
:10C84000FD0EDBCFE6FFFE0EDBCFE6FF1200DECFF4
:10C85000E6FFDDCFE6FF120007D901EC75F0CBD87B
:10C86000D1DE010E12006EEC5AF0E552E552F90EDF
:10C87000F3CFDBFFFA0EF4CFDBFF1200E66ECAEC5B
:10C880009FF017EF65F0F3CFDEFFF4CFDDFF12006E
:10C89000B0DED4EF63F097DE09011200AADE020ECB
:10C8A000E1261200A6DE95EF63F000DF010EA6D6AA
:10C8B000DBD807EF75F091DEA5DE1DEC59F0050E13
:10C8C0000EDF020EE15C1200BBD8EECFE6FFEFCF29
:10C8D000E6FF1200E552F3CF00F0F4CF01F0F3CF02
:10C8E000E6FFF4CFE6FF1200010EDBCFE6FF020EFB
:10C8F000DBCFE6FF1200D8EC74F0006E050EE15EAF
:10C9000000501200FB0EDBCFE6FFFC0EDBCFE6FF94
:10C910001200DECFE9FFDDCFEAFF120066DEE10E96
:10C92000E66EDE0EE66E000EF1EF62F05FDF810E66
:10C93000E66EDD0EE66E000E05EF63F0A3EC3EF052
:10C94000E552E55212004B0EFC6FDF0EFD6F000E3C
:10C9500056EF63F0FADEDECF03F0DDCF04F0056AB8
:10C96000120001C0E6FF02C0E6FF03C0E6FF1200AE
:10C970007F0E0601C85D12006FDE20081200FD0E5A
:10C98000DBCF00F0FE0EDBCF01F0120001EC75F002
:10C99000026E070EE15E02501200050EF3CFDBFFC0
:10C9A000060EF4CFDBFF1200F90EDBCFE9FFFA0E23
:10C9B000DBCFEAFF12007ADE1DEF59F000C0E6FF80
:10C9C00001C0E6FF120015DE030EE126120011DEA3
:10C9D000BDEF63F0000EE66E060EE66E1200E96E25
:10C9E000FF0EDA20EA6EEE50ED1012003AD807EC96
:10C9F00075F029EF63F0006E070EE15E0050120043
:10CA0000DE5241DFDD521200F9EC75F0046E0B0EC0
:10CA1000E15E045043EF64F062DEE3EF62F005DFB5
:10CA200033EF64F01ED867EC75F029EF63F0E55240
:10CA3000E552E552120032DF010EE66E66EF63F05A
:10CA4000FA0EDBCFE9FFFB0EDBCFEAFF1200FC0E94
:10CA5000DBCFE6FFFD0EDBCFE6FF120040DE4BEF43
:0ECA600064F0E66E27EF64F0E66EEAEF64F035
:02CA6E00E4ECF6
:10CA70006BF0020EE126E00E6214DF6E0F0E6514FD
:10CA80000B01406F66CF41FB67CF42FB68CF43FB92
:10CA900069CF44FB6ACF45FB6BCF46FB6CCF47FBAE
:10CAA0006DCF48FB609EDF5001E067D20B01415122
:10CAB000A60A01E15BD2030A01E12FD2010A01E1DA
:10CAC00022D2070A01E115D23D0A01E1F7D1080A95
:10CAD00001E178D1030A01E136D11C0A01E1FAD063
:10CAE000010A01E1E8D00D0A01E1B4D0010A01E137
:10CAF00091D0070A6FE0010A67E0030A45E0010AE6
:10CB000018E0860A01E046D21B0E425D03E145CBE8
:10CB1000DDF90BD01A0E425D01E03CD24551000E0A
:10CB2000F35046250901DE6FDF6B0901010EE56F49
:10CB300031D242CBA0F944CB01F0006A4351090144
:10CB40000024A16F000E0120A26F48CB01F0006A03
:10CB50000B01475109010024A36F000E0120A46FAF
:10CB60000901700ED880A155170EA25502E2A16BE3
:10CB7000A26B0901700ED880A355170EA45501E3CE
:10CB800009D2A36BA46B06D2C3EC6BF003E0EFEC0D
:10CB90006BF0FDE18BEC6BF003E0F6EC6BF0FDE18C
:10CBA00094EC6BF003E014EC6CF0FDE100500C240D
:10CBB0000901A56F01500D20A66F02500E20A76F2E
:10CBC00003500F20A86FE6D142CBADF90901780ED2
:10CBD000E16FE0D1C3EC6BF003E0EFEC6BF0FDE153
:10CBE0008BEC6BF003E0F6EC6BF0FDE194EC6BF09A
:10CBF00003E014EC6CF0FDE100500C240901D16F4E
:10CC000001500D20D26F02500E20D36F03500F2021
:10CC1000D46FC0D1C3EC6BF003E0EFEC6BF0FDE13F
:10CC20008BEC6BF003E0F6EC6BF0FDE194EC6BF059
:10CC300003E014EC6CF0FDE100500C240901D56F09
:10CC400001500D20D66F02500E20D76F03500F20D9
:10CC5000D86FA0D142CBE0F90901E05129E044CBE3
:10CC600001F0006A0B01435109010024D96F000E45
:10CC70000120DA6F680ED91905E1010EDA1902E117
:10CC8000D96BDA6BF00E0B01461504E00901DB6B82
:10CC9000DC6B0AD046CB01F0006A45510901002443
:10CCA000DB6F000E0120DC6F0901780EE36F72D19B
:10CCB0000901E36B6FD142CB90F947CB91F944CB9B
:10CCC00001F0006A435109010024926F000E012017
:10CCD000936F60D14D0E0701CB5D03E142CB9FF90D
:10CCE00026D042CB26F0276A286A296A490E2B6E85
:10CCF000060E2C6E2D6A2E6AF0ECA7F022C026F0EC
:10CD000023C027F024C028F025C029F0F40E2626E1
:10CD1000010E2722000E28222922E80E2B6E030E78
:10CD20002C6E2D6A2E6A59ECA8F026C09FF944CBD0
:10CD300001F0006A0B014351090100248E6F000EBF
:10CD400001208F6F27D1090194510B01425D0EE044
:10CD500009019451020803E20F0E945D07E1040EED
:10CD60000B01425D03E0040EA4EC6BF00901945149
:10CD70000B01425D05E1090195510B01435D0CE09A
:10CD8000020EA4EC6BF00B01420506E123EC6CF003
:10CD900003E20901010E096F42CB94F943CB95F9E7
:10CDA0000501F3A104D00F0E0B01451504D00B01B2
:10CDB00046390F0B0F0B0901966F44CB97F948CBFF
:10CDC00098F9E8D00F0E0901945D02E10B01428948
:10CDD0000B0142510901995D0FE10B01435109011A
:10CDE0009A5D0AE10B01445109019B5D05E10B01CC
:10CDF000455109019C5D03E0010EA4EC6BF0800E2F
:10CE000009019A150AE1800E0B01431506E0100E88
:10CE1000431503E0100EA4EC6BF0020E09019C1503
:10CE200007E1020E0B01451503E0200EA4EC6BF0A8
:10CE300042CB99F943CB9AF944CB9BF945CB9CF96A
:10CE400039EC6CF021E10901A951AA11AB11AC1127
:10CE50001BE10901A551A611A711A81115E023ECAA
:10CE60006CF003E20901010E096FA5C9A9F9A6C971
:10CE7000AAF9A7C9ABF9A8C9ACF90901A907000E1D
:10CE8000AA5BAB5BAC5B16D039EC6CF001E182D0F5
:10CE90000901A951AA11AB11AC1101E17BD023EC1E
:10CEA0006CF003E20901010E096F0901A96BAA6B7D
:10CEB000AB6BAC6B010EA4EC6BF06CD04351640D0A
:10CEC0005DEC6CF0800E0026000E0122080E0F0BA8
:10CED00005E0D89001320032E806FBE10B01445135
:10CEE000640DF35000240901F56FF4500120F66F32
:10CEF00051D042CBC0F943CBC1F947CBC2F90901AC
:10CF0000780EE26F47D0010EDB6A1BEC6CF042E258
:10CF1000FDEC6BF009EC6CF0F8D7010EDB6A1BEC52
:10CF20006CF006E2FDEC6BF0070F09EC6CF0F7D744
:10CF3000410E0B01445D03E0420E445D03E1050137
:10CF4000320E02D00501310ECA6F380E0B01445D5E
:10CF500002E10501F381330E0B01425D03E105019E
:10CF6000530E02D005014E0ECB6F14D042CBBCF94C
:10CF700043CBBDF944CBBEF90DD00B0141510E0A94
:10CF800009E1425109019E5D03E0010EA4EC6BF042
:10CF900042CB9EF9010E006E020EE15C02E2E16AF4
:10CFA000E552E16E0050DDEF6BF0E4EC6BF0E65221
:10CFB0000F0E0F0155150B01406F56CF41FB57CF98
:10CFC00042FB58CF43FB59CF44FB5ACF45FB5BCFC5
:10CFD00046FB5CCF47FB5DCF48FB50CFDFFF0F0127
:10CFE000509F070EDF14040832E1020E0B01415D71
:10CFF00001E089D00501E551000801E384D039EC56
:10D000006CF001E180D00B01435109019F5D01E10A
:10D010007AD023EC6CF001E376D041CB00F942CB1F
:10D0200001F99FC902F9F00E0B0144150901036FC4
:10D0300045CB04F946CB05F947CB06F948CB07F9B0
:10D040000F0140B7FDD787DBE5C508F95CD0070EB7
:10D05000DF14020821E10B014451000804E243CB34
:10D06000C7F944CBC3F94851000804E247CBC8F9DB
:10D0700048CBC4F94251000804E241CBC9F942CB84
:10D08000C5F94651000804E245CBCAF946CBC6F9BA
:10D090000901780EE46F37D00B014151FA0A33E1F0
:10D0A00044CB00F0016A026A036A45CB04F0056ACA
:10D0B000066A076A080E1F0B02E091DBFEE13DECF9
:10D0C0006CF046CB08F0096A0A6A0B6A100E1F0B57
:10D0D00002E08CDBFEE1005008240901CD6F015015
:10D0E0000920CE6F02500A20CF6F03500B20D06F63
:10D0F00048CB01F0006A0B01475109010024CB6FB6
:10D10000000E0120CC6F010EE55257D309010851E2
:10D1100002E1E5C508F9000C0901095114E0096BA9
:10D120000F0140B7FDD7F1DA060E466FD00E476FFC
:10D13000070E486F496B4A6B4B6B4C6B400E4D6F43
:10D14000080E456F406F0901085101E1000C020E05
:10D15000005D11E10501E55100080DE28ADB0BE0FD
:10D1600072DB09E2010EE66EE4ECA8F0E5520F0175
:10D1700040B7FDD7F0DA09010807000C0F0140B7EE
:10D18000FDD7C3DA0A0E466F010E456F080E406FD9
:10D1900040B7FED712000F0140B7FDD7B6DA060E32
:10D1A000466F2C0E476F010E486F496B4A6B090E94
:10D1B0004B6F100E4C6F86DB40B7FED7120004DBBE
:10D1C0000F0140B7FDD775DB190E95DA40B7FED7D2
:10D1D000D5DFF3D2F9DA0F0140B7FDD76ADB020ED3
:10D1E0008ADA40B7FED7CADFE8D2EEDA0F0140B7DD
:10D1F000FDD75FDB030E7FDA40B7FED7BFDFDDD29E
:10D20000E3DA040EE12647DB54EC8AF0E552E552FE
:10D2100026C0DEFF27C0DEFF28C0DEFF29C0DDFFFD
:10D22000DD52DD52FE0EDB50020802E122DB4EE150
:10D230000F0140B7FDD769DA0B0E466FFE0EDBCF4C
:10D2400047FF486B496BACDA00504A6FA9DA080E09
:10D25000FEDAFEE100500F014B6FA2DA100EF7DA92
:10D26000FEE100500F014C6F16DBA3EC98F0F6DAEC
:10D27000040ED89000360136E804FBE1026A036A26
:10D28000180E086ED9CFE9FFDACFEAFFE8501F0B7E
:10D29000EECF04F0EECF05F0EECF06F0EECF07F0C4
:10D2A00007E0D8900732063205320432E806F9E189
:10D2B0000F0E0416056A066A076ADFDA00C04DFF22
:10D2C0000F01080E456F406F40B7FED7040EE15CBA
:10D2D00002E2E16AE552E16E70D276DA0F0140B700
:10D2E000FDD7E7DA1B0E07DA40B7FED7FE0EDB04E8
:10D2F0001AE1DFDA1A0E476F486B496BFD0EDBCF80
:10D3000001F001C000F001504A6FFF0EE76EFC0E05
:10D31000DBCF00F0E7500016016A00C04BFF4C6BFA
:10D32000D1DA40B7FED72ADF48D24EDA0F0140B734
:10D33000FDD7EBD9090E466F476BFE0EDBCF48FFDA
:10D34000030E456F080E406F40B7FED717DF35D28A
:10D350003BDA030EE126020EDB6AFC0EDBCF28F07F
:10D36000FD0EDBCF29F0180E281801E1295001E14C
:10D3700010D1170E281801E1295001E1EED0160E48
:10D38000281801E1295001E1E2D0150E281801E129
:10D39000295001E1D6D0140E281801E1295001E1ED
:10D3A000CAD0130E281801E1295001E1BFD0120E96
:10D3B000281801E1295001E1B4D0110E281801E12B
:10D3C000295001E180D0100E281801E1295058E0C1
:10D3D0000F0E281801E129504DE00C0E281801E12C
:10D3E000295034E00B0E281801E1295016E00A0EEE
:10D3F000281801E1295002E0000EECD00501F4519B
:10D4000001E1CAD0FA0EDBCFE6FFFB0EDBCFE6FF71
:10D4100049DAD5DEE552B2DEC8D00501F45101E1AA
:10D42000BBD0040E090199150BE0070E0901955DAB
:10D4300007E0010EE66ED9DEE5520601F36BB5D0CA
:10D44000570EE66E4E0EE66E010EB4D00501F45195
:10D4500001E1A2D0090199A907D0E66AC6DEE5522A
:10D4600006011E0EF36FA1D07D0EE66E4E0EE66E27
:10D47000010EA0D00501F45101E18ED007DA20D0D1
:10D480000501F45101E188D0A0CADEFFA1CADDFF89
:10D49000A0D908E09ED92C0805E0DF2A010EF8E3A8
:10D4A000DB2AF6D796D92C0836E1DCD901E3DB2A52
:10D4B000EF6A87D984DEE552DECFE6FFDDCFE6FFF7
:10D4C000F1D988DE71D00501F45166E0A0CADEFF13
:10D4D000A1CADDFF7ED908E07CD92C0805E0DF2A4F
:10D4E000010EF8E3DB2AF6D774D92C0814E1BAD977
:10D4F00001E3DB2AEF6ADECFE6FFDDCFE6FFDFECFC
:10D5000089F0ACD9F3CFE6FFF4CFE6FF5AD9E5DED8
:10D51000E552E55249D0110EE66E4E0EE66E010E52
:10D5200049D00501F45138E029DE03D00501F4515A
:10D5300033E031DE3AD00501F45112E0A7D9020EF2
:10D5400017D00501F4510CE0A1D9E66A12D005010B
:10D55000F45106E09BD9030E0BD00501F45106E10E
:10D56000230EE66E4E0EE66E010E0CD08FD9010E24
:10D57000E66E46DEE552E552E5520E0EE66E4E0EC2
:10D58000E66E010E9AD8010EF36E020EF3CFDBFFAA
:10D5900012D00501F45106E1230EE66E4E0EE66E42
:10D5A000010E08D00ED9C1DEE5520E0EE66E4E0E0B
:10D5B000E66E010E82D8FE0EDB500BE03AEC2EF048
:10D5C000020EE66EBFEC72F0E552E66A76EC31F0E0
:10D5D000E552010E006E030EE15C02E2E16AE552E3
:10D5E000E16E0050EAD0D9CFE6FF020EE126050138
:10D5F000540EC86F520EC96FCA6BCB6BCC6B900EBA
:10D600006F6E6EAEFED7606A0F01A00E196F1869BB
:10D61000016B200E006F506BE00E1D6F1C69800EB9
:10D62000096F680E086F400E0D6F800E0C6F116B46
:10D63000106F706AD20E716E020E726E200E736ED3
:10D6400002D902E26F6A02D0600E6F6E0901006BB0
:10D65000086B096B0601EE850701760ECF6F520E3F
:10D66000D06F010ED16F07016E0ED56FCA0ED66F47
:10D67000000ED76F0701AA0ED86FCF0ED96F000E1C
:10D68000DA6F07010C0EED6FD10EEE6F000EEF6F2B
:10D690000701180EF06FD10EF16F000EF26F0B0143
:10D6A000500E496FD30E4A6F000E4B6F020EE15CB5
:10D6B00002E2E16AE552E16E80D0E66EECD8070E38
:10D6C000E66E4E0EE66E010EE66E000EE66E060E7D
:10D6D000E66E07EC75F0026E070EE15E0250EDD8C3
:10D6E000F3CFE6FFF4CFE6FFD8EC74F0036E050E3F
:10D6F000E15E03501200476F486B496BFE0EDBCFB3
:10D700004AFF4B6B4C6B62EF6CF0406B400E426F0C
:10D71000200E416F1200B1D847CB08F0096A0A6A9F
:10D720000B6A100E1F0B1200085000260950012230
:10D730000A5002220B50032248CB0CF00D6A0E6AED
:10D740000F6A180E1F0B1200E66EE66AFEEC3EF042
:10D75000E552E5521200406B426B800E416F00C9EA
:10D7600046FF01C947FF02C948FF03C949FF04C971
:10D770004AFF05C94BFF06C94CFF07C94DFF080EFC
:10D78000456F406F120045CB00F0016A026A036AE0
:10D7900046CB04F0056A066A076A080E1F0B1200E2
:10D7A000D9CFE9FFDACFEAFFEECF00F0EECF01F0FC
:10D7B000EECF02F0EFCF03F01200E552E7CFD9FF32
:10D7C000120064D852EF6CF0D9CFE6FFE1CFD9FF59
:10D7D0001200DECFE9FFDDCFEAFFEF501200D89054
:10D7E0000436053606360736E8061200D8900836A5
:10D7F00009360A360B36E8061200010EDB28EA6A03
:10D80000410FE96E0B0EEA22EF50E66E010EDB507F
:10D810001200EA6AAE0FE96E090EEA22E552E750FD
:10D82000EF6E010EDB2A1200D8900C360D360E3644
:10D830000F36E8061200070EF36E010EDBCFF4FF81
:10D84000F350F45C12000501F45100081200D89066
:10D850000332023201320032E8061200E552E5528C
:10D860005DEF6CF0DFCFE9FFDF2A010EDBCFEAFFCF
:10D870001200800E0901991512000450002605506F
:10D88000012206500222075003221200A0CAE6FF1E
:10D89000A1CAE6FF1200FC0EDBCFE6FFFD0EDBCFD8
:10D8A000E6FF1200DFEC89F0E552E552F350E66E38
:10D8B00012002BDF050E466F1200F3CF00F0F4CFFD
:0ED8C00001F012004D6B080E456F406F120014
:02D8CE005354B1
:10D8D0004154002B435553443A002B4346554E3A8E
:10D8E000005244590053454E44204641494C0043A0
:10D8F0004F4E4E454354204641494C00434C4F53F4
:10D900004544004441544120414343455054005351
:10D91000454E44204F4B002B4353513A0053544142
:10D9200054453A2054435020434C4F5345440053F0
:10D93000544154453A2054435020434F4E4E4543A2
:10D9400054494E470053544154453A20434F4E4E9C
:10D95000454354204F4B0053544154453A20004313
:10D960004F4E4E454354204F4B0036342C002C0074
:10D97000322C002B434C4950002B5044503A204449
:10D9800045414354002B435245473A203000222C56
:10D990002236383637220D0041542B434950535418
:10D9A0004152543D22544350222C220041542B43D7
:10D9B000494653520D0041542B4349504845414478
:10D9C0003D310D0041542B43494943520D00222C57
:10D9D000220041542B435354543D2200220D004158
:10D9E000542B434744434F4E543D312C224950223F
:10D9F0002C22002B43524547002B434F50533A00F3
:10DA00002B434D45204552524F52005345545550DB
:10DA100000223B2B434F50533F0D0041542B434FAB
:10DA200050533D312C312C220041542B434C504F4C
:10DA300052543D22544350222C2236383637220D80
:10DA40000041542B434950434C4F53450D00415422
:10DA50002B434950534855540D00002D00220049D6
:10DA60005000534D5300562900562C207265663DD8
:10DA7000004D502D302050413132562042415454F7
:10DA8000455259204F4B2028004D502D30205041F9
:10DA9000414C4552542121212031325620424154DB
:10DAA0005445525920435249544943414C2028007F
:10DAB0002520534F4329004D502D30205041414CDB
:10DAC00045525421212120435249544943414C207D
:10DAD000534F43204C4556454C20415050524F41E6
:10DAE000434845442028004D502D30205041547269
:10DAF000756E6B20686173206265656E206F70655E
:10DB00006E6564202876616C6574206D6F6465298C
:10DB10002E004D502D3020504156656869636C656C
:10DB200020616C61726D20697320736F756E64691A
:10DB30006E6721000D204341433A20000D204F44E1
:10DB40004F3A200025000D20534F433A2000206B10
:10DB50006D00206D6900202D20000D2052616E6740
:10DB6000653A20004E6F74206368617267696E6762
:10DB7000004368617267696E672053746F707065E7
:10DB800064004368617267696E672C204865617440
:10DB9000696E6700507265706172696E67004368F4
:10DBA000617267696E6720446F6E650043686172D9
:10DBB00067696E672C20546F7070696E67206F669E
:10DBC00066004368617267696E6700506572666FD0
:10DBD000726D616E6365202D200052616E67652055
:10DBE0002D200053746F72616765202D20005374DF
:10DBF000616E64617264202D20002C312C496E7698
:10DC0000616C6964205553534420726573756C745C
:10DC1000002C302C00202D204D53473A2000534D2E
:10DC2000532046524F4D3A20004D502D3020504148
:10DC3000000D00222C31350D0041542B4355534427
:10DC40003D312C22004D502D302063332C302C00E0
:10DC50004D502D302063312C302C004D502D302074
:10DC600061004D502D3020004D502D5320302000AC
:10DC70004D502D3020482A2D4F564D2D446562754C
:10DC80006743726173682C302C3235393230303052
:10DC90002C004D502D30204554004D502D30206724
:10DCA0000043312D362C4334302D34312C4334395C
:10DCB000004D502D302056004D502D302044002F67
:10DCC00056002F002E004D502D30204600302C30B5
:10DCD0002C004D502D302057004D502D30204C0041
:10DCE0002C706572666F726D616E6365002C726177
:10DCF0006E6765002C73746F72616765002C7374B6
:10DD0000616E64617264002C73746F70706564007E
:10DD10002C68656174696E67002C70726570617241
:10DD200065002C646F6E65002C746F706F66660002
:10DD30002C6368617267696E67002C004D502D304E
:10DD400020530020004D502D43203020004D502DF9
:10DD50003020454D001A000D0A0041542B43495014
:10DD600053454E440D002320004D502D30206300BC
:10DD70002000436F6D6D616E64733A002F56002F63
:10DD8000002E004F564D53204669726D77617265C3
:10DD90002076657273696F6E3A20003400504552E8
:10DDA00000330052414E00310053544F00300053B5
:10DDB0005441000D0A200046656174757265733A1E
:10DDC000002053544B554E46002053544B46554C5F
:10DDD000002052490020544F002050440020504F52
:10DDE000520020424F52000A202E2E6C6173743A6A
:10DDF000000A20437261736865733A002072656699
:10DE00003D000A20313256204C696E653A000A20E6
:10DE10004E45542053746174653A3078000A2047A7
:10DE2000524E204C65643A000A20524544204C650D
:10DE3000643A00444941473A000D0A20506172613A
:10DE40006E6F69643A000D0A2049503A00536572BA
:10DE50007665723A0043757272656E743A200028D6
:10DE60006E6F6E65290D0A0047534D4C4F434B3A78
:10DE7000200029000D0A2047534D2F475052533A96
:10DE8000204E6F7420636F6E6E6563746564202826
:10DE90003078000D0A2047534D3A204F4B0D0A2091
:10DEA0005365727665723A204E6F7420636F6E6EA2
:10DEB0006563746564000D0A20475052533A204F41
:10DEC0004B0D0A205365727665723A20436F6E6E71
:10DED0006563746564204F4B000D0A2047534D3A2B
:10DEE000000D0A2050617373776F72643A000D0A57
:10DEF00020557365723A000D0A2041504E3A004792
:10DF00005052533A000D0A204E6F7469666963617E
:10DF100074696F6E733A000D0A20556E6974733A16
:10DF2000000D0A2056656869636C65547970653A1E
:10DF3000000D0A2056656869636C6549443A004DD6
:10DF40006F64756C653A003A000A00506172616D49
:10DF5000733A002C004D6F64756C652070617373AB
:10DF6000776F72643A2000526567697374657265F1
:10DF700064206E756D6265723A2000562900562C39
:10DF8000207265663D004D502D3020504131325693
:10DF90002042415454455259204F4B2028004D50A7
:10DFA0002D30205041414C45525421212120313205
:10DFB00056204241545445525920435249544943F2
:10DFC000414C2028002520534F432900414C455205
:10DFD0005421212120435249544943414C20534F5D
:10DFE00043204C4556454C20415050524F414348E8
:10DFF00045442028001A000D0A00220D0A00415451
:10E000002B434D47533D220023200030313233341F
:10E01000353637383941424344454600232053744E
:10E020006F707065642043414E2073696D0D0A0066
:10E0300023205374617274696E672043414E2073CC
:10E04000696D0D0A0041542B4353510D0041542B6F
:10E050004350494E3F0D0041542B434F50533F0D09
:10E06000000A0023202053696D2054783A200020B4
:10E07000657374206D696C6573290D0A00206964ED
:10E0800065616C2C200025202800232020534F435D
:10E090003A20202020202000290D0A0020280023DB
:10E0A000202056494E3A202020202020000D0A0A28
:10E0B000002320205369676E616C3A2020200020E5
:10E0C000560D0A00232020313256204C696E653AE5
:10E0D00020002320205357495443483A2020200051
:10E0E0002F56002F002E0023204669726D77617233
:10E0F000653A20000D0A2320444941470D0A0A00D1
:10E1000023204C656176696E6720446961676E6F94
:10E110007374696373204D6F64650D0A00232027B3
:10E120004D2720434F4D4D414E44533A0D0A202078
:10E1300000232027532720434F4D4D414E44533A4F
:10E140000D0A2020002320434F4D4D414E44533AA9
:10E150002048454C50203F204449414720524553D8
:10E160004554206F722053202E2E2E0D0A000D0ACA
:10E17000004F564D5344494147000D0A23204E4F4E
:10E180005449465920414C41524D20414C4552542E
:10E190000D0A000D0A23204E4F544946592054526F
:10E1A000554E4B20414C4552540D0A000D0A232078
:10E1B0004E4F544946592043484152474520414C0F
:10E1C0004552540D0A001B5B324A1B5B30313B3019
:10E1D00031480D23204F564D5320444941474E4F5F
:10E1E0005354494353204D4F44450D0A0A00200023
:10E1F000200D0A5477697A7920436F6D6D616E64E2
:10E20000733A0056200043292000432E2E0043205D
:10E210002800503A0042617474657279206D6F6E07
:10E2200069746F722072657365742E0052542D509C
:10E2300057522D4261747443656C6C2C0052542DFE
:10E240005057522D426174745061636B2C004D50D5
:10E250002D302048004D0043200054656D70733A06
:10E2600020003A003A2B0043002E2E2E004F4B2068
:10E27000006D56200053443A003F002100566F6C59
:10E2800074733A20000A2046756C6C2063686172D2
:10E2900067653A20000A2054696D653A2000206FB6
:10E2A0007220004F46460043686172676520416CEA
:10E2B0006572743A2000554E534554004D617820E4
:10E2C000696465616C2072616E67653A20000D209B
:10E2D0004F444F3A2000252900252E2E00252028C6
:10E2E000000D20534F433A2000206B6D00206D69D4
:10E2F00000202D20000D2052616E67653A20000D30
:10E300002046756C6C206368617267653A20004E28
:10E310006F74206368617267696E6700206D696E53
:10E320002E000D2046756C6C3A20000D20434847A6
:10E330003A20004368617267696E672053746F709A
:10E34000706564004368617267696E6720446F6E30
:10E3500065004368617267696E672C20546F707046
:10E36000696E67206F6666004368617267696E67F1
:10E37000002073733D00206C74613D002074613D8A
:10E38000002074773D00206C76613D002076613D71
:10E39000000A232076773D00204449523D00204169
:10E3A0004C543D00204C4F4E3D00204C41543D000C
:10E3B0000A23204649583D002053513D00206472F5
:10E3C0003D002064693D00204F444F3D00205354E0
:10E3D000533D002C302C0063004D502D3020004D5B
:10E3E000502D30205041002C30004D502D302063F6
:10E3F000004D502D30204852542D5057522D5573FA
:10E4000061676553746174732C302C383634303046
:10E41000000D20446F776E20006D20000D20557098
:10E4200020000D20446563656C20000D204163636E
:10E43000656C20002520000D20436F6E7374200052
:10E4400025002057682F6B6D20523D004566666998
:10E450006369656E63792000456666696369656E08
:10E46000637920756E6B6E6F776E2C206E6F2070E7
:10E470006F7765722F64697374616E636520646180
:10E48000746120617661696C61626C652E00205751
:10E4900068002057680D20446F776E20006D202D96
:10E4A000002057680D20557020002057680D20442B
:10E4B0006563656C20002057680D20416363656CBF
:10E4C000200025202D00206B6D0D20436F6E73748E
:10E4D00020002057682000202B00506F77657220A5
:10E4E0002D00495000534D53000A00232073696DDD
:10E4F0002064617461206C696E6520002C002C38EA
:10E50000363430302C004D502D30204852542D4799
:10E5100050532D4C6F672C002C002C302C006300C6
:10E520004D502D302000545A004E4C005443004FA3
:10E5300032005254005641005452002C002C302C12
:09E540000063004D502D30200055
:06E54A00FF0012003AEC94
:10E5500078F0060EDF5C05E29EA2FED79E92DF2ACF
:10E56000F8D763EF77F03AEC78F07A0EDF5C05E2EB
:10E570009EA2FED79E92DF2AF8D763EF77F0F5ECE4
:10E5800077F0FE0EDB50000804E2EDDFFE0EDB0646
:10E59000F8D713EF78F0D7EF77F0D7EF77F081B0B7
:10E5A00005D08180050EE66EEADFE5528190140EFB
:10E5B000E66EE5DFE55281801200F5EC77F00E0E95
:10E5C000C4EC77F054EC8AF067EC77F02E0EE66E30
:10E5D000EEEC77F035EC98F0EAEC77F00C0EF3CF38
:10E5E000DBFF0D0EF4CFDBFFF3CF00F0F4CF01F033
:10E5F000F350F41001E1C6D0040EDB6A050EDB6AAD
:10E60000060EDB6A070EDB6A010EF36E080EF3CF0F
:10E61000DBFF090EDB6A0A0EDB6A0B0EDB6A0C0EEF
:10E62000DB2ADBCFE9FF0D0E01E3DB2ADBCFEAFFBC
:10E63000EF5057E0040EDBCF00F0050EDBCF01F00A
:10E64000060EDBCF02F0070EDBCF03F0B9EC77F05C
:10E6500000C026F001C027F002C028F003C029F056
:10E66000F0ECA7F095EC77F00C0EDBCFE9FF0D0E88
:10E67000DBCFEAFFEF50D00F046E056A066A076A27
:10E68000E8500026055001220650022207500322BE
:10E69000040E00C0DBFF050E01C0DBFF060E02C04A
:10E6A000DBFF070E03C0DBFF080EDBCF26F0090EF1
:10E6B000DBCF27F00A0EDBCF28F00B0EDBCF29F0E3
:10E6C000B9EC77F0F0ECA7F0080E22C0DBFF090EE2
:10E6D00023C0DBFF0A0E24C0DBFF0B0E25C0DBFFCF
:10E6E0009ED729EC78F0EECF08F0EECF09F0EECF10
:10E6F0000AF0EFCF0BF09CDB040EDBCF14F0050E1D
:10E70000DBCF15F0060EDBCF16F0070EDBCF17F0D0
:10E7100014C026F015C027F016C028F017C029F045
:10E72000A5EC82F027C010F028C011F029C012F02B
:10E730002AC013F0080EDBCF1CF0090EDBCF1DF052
:10E740000A0EDBCF1EF00B0EDBCF1FF01CC026F035
:10E750001DC027F01EC028F01FC029F0A5EC82F0D4
:10E7600027C018F028C019F029C01AF02AC01BF0E1
:10E770004DDBE4DB55EC83F0EADB48DB9BDBBFECF5
:10E7800082F002D039DBB6DB4ADB27C026F028C096
:10E7900027F029C028F02AC029F00E0EE15C02E221
:10E7A000E16AE55260D3F5EC77F0080EEDDB05DFAA
:10E7B0008EDB29EC78F0EECF00F0EECF01F0EECF5B
:10E7C00002F0EFCF03F02C6A2D6AC80E2E6E420EB7
:10E7D0002F6EC6DB55EC83F073EC85F0040E26C07B
:10E7E000DBFF050E27C0DBFF060E28C0DBFF070E90
:10E7F00029C0DBFF040EDBCF04F0050EDBCF05F0F4
:10E80000060EDBCF06F0070EDBCF07F073DB07DB6E
:10E8100029EC78F0EECF10F0EECF11F0EECF12F041
:10E82000EFCF13F0040EDBCF18F0050EDBCF19F09D
:10E83000060EDBCF1AF0070EDBCF1BF0640E2B6E3B
:10E840002C6A2D6A2E6A18C026F019C027F01AC04B
:10E8500028F01BC029F0F0ECA7F022C018F023C06C
:10E8600019F024C01AF025C01BF022C026F023C0E6
:10E8700027F024C028F025C029F0A5EC82F027C09D
:10E8800014F028C015F029C016F02AC017F0BEDA1F
:10E8900055DBBEEC82F05BDB2C6A2D6A700E2E6EAF
:10E8A000420E2F6E55EC83F027C008F028C009F007
:10E8B00029C00AF02AC00BF0A9DA52DBBFEC82F0C3
:10E8C0001CDB9ADA77DBF6DAA8EC83F0A8DA2C6A9C
:10E8D0002D6A2E6A450E2F6EA8EC83F073EC85F03E
:10E8E000080EE15C02E2E16AE552BDD27EDB040E75
:10E8F000E126DE68DD68FB0EDBCF00F0FC0EDBCF2F
:10E9000001F0013435E200500008000E015430E2FD
:10E91000A2DA01E3DB2AEF50DF1AFB0EDB06FC0E66
:10E9200001E2DB06020EDB6A030EDB6A020EDBCFBE
:10E9300000F0030EDBCF01F0D890015004E6080E82
:10E94000005C000E0158D7E2DF50010B06E01FDB30
:10E95000010E001AA00E011A01D019DB00C0DEFF63
:10E9600001C0DDFF020EDB2A030EE0E3DB2ADED767
:10E97000DECF00F0DDCF01F000C0F3FF01C0F4FFF7
:10E98000040EE15C02E2E16AE5526DD22EDB19DB96
:10E99000EE50ED100CE06BDB0AE069DB0D0803E1E3
:10E9A0000BDA0A0EEF6EBDDAF2E3DB2AF0D73BD3C7
:10E9B0001CDBD950FA0F72DBEFCFF6FFEE2AEFCF58
:10E9C000F7FF000EEE22EFCFF8FFEE220800F55021
:10E9D00058DB04E0A6DAEDE3DB2AEBD7E6D105DB72
:10E9E000FB0EDBCFE9FFDB2AFC0EDBCFEAFF01E306
:10E9F000DB2AEF5046DB04E094DAF2E3DB2AF0D7BF
:10EA0000D4D1D5D901E0C9D942DB58DB5CD2CFD90A
:10EA100001E0C3D969DAFFEC8AF0DCDAE55227DBE2
:10EA200004E07FDAFCE3DB2AFAD7BFD1C0D901E0EA
:10EA3000B4D9BFD999EC8BF0A2DA19DB04E071DA12
:10EA4000FCE3DB2AFAD7B1D1B2D901E0A6D9B1D91A
:10EA50008CEC8CF094DA0BDB04E063DAFCE3DB2A69
:10EA6000FAD7A3D144DA54DA040EEE26000EED22D2
:10EA7000FB0EDBCFE9FFFC0EDBCFEAFFEF6A040EF3
:10EA8000DF6EDF5023E08BDAE76EFD0EDBCF03F0A5
:10EA9000FE0EE7500316046A056AE7D9FB0EDB0693
:10EAA000DBCFE9FFFC0E01E2DB06DBCFEAFFE5523C
:10EAB000E750EF6E86DA040E0F0B06E0EC52D890AA
:10EAC000ED32EF32E806FAE1DF06DBD7FCD16FD991
:10EAD00001E063D909DAC6DF7DDAE552C8DA04E07D
:10EAE00020DAFCE3DB2AFAD760D101DAD950F90F3A
:10EAF000D5DA080EEE26000EED22F90EDBCFE9FF87
:10EB0000FA0EDBCFEAFFEF6A080EDF6EDF502AE075
:10EB100046DA036E046A056A066AFAD9EE500316ED
:10EB2000EE500416EE500516EE5006169ED9F90E5C
:10EB3000DB06DBCFE9FFFA0E01E2DB06DBCFEAFF03
:10EB4000E552E750EF6EE4D9040EE76ED890030E5D
:10EB5000EB32020EEB32010EEB32EF32E706F6E15A
:10EB6000DF06D4D7B0D123D901E017D922D9BDDF30
:10EB700006DA7DDA04E0D5D9FCE3DB2AFAD715D131
:10EB800034DA0C0EA2D901E008D91FDA33DA8CECA2
:10EB90008CF0F5D91ADAA3EC98F0E552E5520B0E99
:10EBA000F3CFDBFFDB50006E016AF40EDBCF02F027
:10EBB000F50EDBCF03F001500318E8AE02D00334AA
:10EBC00004D00250005C0350015809E244D901E32B
:10EBD000DB2AF30EDBCFEFFF0B0EDB2AE3D7F5D9F1
:10EBE0006DDAE55253D90C0EE15C02E2E16AE552BE
:10EBF0003AD1FBD9050EE126010EDE6EDE6ADE6A31
:10EC0000DD6ADD52DD52F40EDB50E76E040EE7CF15
:10EC1000DBFFDB50000817E21CDAABD9EECF26F0A1
:10EC2000EECF27F0EECF28F0EFCF29F0F0ECA7F0F1
:10EC300025C0EDFF24C0EDFF23C0EDFF22C0EFFF94
:10EC4000040EDB06E6D7BFD855EC84F022D92BDAC8
:10EC5000EDDE086E090EE15E0850F4D9FCD801E340
:10EC6000DB2A2E0EEF6E300EE66EF40EDBCFE6FFE3
:10EC7000F50EDBCFE6FFA7D82EC0F5FF55EC84F0EC
:10EC8000F5AE08D0000E226C231E2322241E24225F
:10EC9000251E25224AD922C0E6FF23C0E6FF24C054
:10ECA000E6FF25C0E6FF38D96BDF086E0C0EE15E8B
:10ECB0000850ECD8050EE15C02E2E16AE552D3D0DF
:10ECC00094D9040E02D901E068D8D950F60FE6D9DC
:10ECD000D890030EEB50000A08E6000EEE5C000E22
:10ECE000EE58000EEE58000EEE5821E2B4D801E3C3
:10ECF000DB2A2D0EEF6EF60EDBCF00F0F70EDBCF2A
:10ED000001F0F80EDBCF02F0F90EDBCF03F0001EAE
:10ED1000011E021E031EF60E00C0DBFFF70E01C02F
:10ED2000DBFFF80E02C0DBFFF90E03C0DBFFF60EBF
:10ED3000DBCF08F0F70EDBCF09F0F80EDBCF0AF0DF
:10ED4000F90EDBCF0BF074D82C6A2D6A2E6A450EB3
:10ED50002F6E55EC83F063D82DD955EC83F0CDD8C8
:10ED6000060EE66EE66A48D82C6A240E2D6E740EE6
:10ED70002E6E490E2F6E9ED8A8EC83F073EC85F0B2
:10ED800088D8CAD836DF086E0B0EE15E0850040E34
:10ED9000E15C02E2E16AE55266D085D909DE006EE7
:10EDA000050EE15E005022EF78F041D93CD11DD92B
:10EDB0002DD114D9FAEF77F0FD0EDBCFE9FFFE0E6F
:10EDC000DBCFEAFF1200F60EDBCF04F0F70EDBCF4D
:10EDD00005F0F80EDBCF06F0F90EDBCF07F03ED9D9
:10EDE000DFCF2BF0010EDBCF2CF0020EDBCF2DF0AE
:10EDF000030EDBCF2EF012002CD9EECF04F0EECFB5
:10EE000005F0EECF06F0EFCF07F0120027C02CF090
:10EE100028C02DF029C02EF02AC02FF0120027C0E4
:10EE200000F028C001F029C002F02AC003F012004F
:10EE300008C026F009C027F00AC028F00BC029F04E
:10EE4000A5EC82F027C004F028C005F029C006F028
:10EE50002AC007F01200FD0EDBCFE9FFDB2AFE0E11
:10EE6000DBCFEAFF1200E16EDED000500324F36E28
:10EE700001500420F46E02500520F86EF4CFF7FF25
:10EE8000F3CFF6FF0800F550E66E1200DBD817EF5F
:10EE900078F026C000F027C001F028C002F029C099
:10EEA00003F026C0E6FF27C0E6FF28C0E6FF29C022
:10EEB000E6FF120004C027F005C028F006C029F0C4
:10EEC00007C02AF01200E552AED0E1269FD0E552ED
:10EED000E55226C0DEFF27C0DEFF28C0DEFF29C0C6
:10EEE000DDFFDD52DD52120079D847EF78F07DD892
:10EEF000E6521200B3D8A5EF82F027C0DEFF28C08B
:10EF0000DEFF29C0DEFF2AC0DDFFDD52DD52120028
:10EF1000D950FB0F4EEF78F0E66AE66AE66AEEEF4C
:10EF200077F0FD0EDB2AFE0E120022C000F023C097
:10EF300001F024C002F025C003F0120010C027F039
:10EF400011C028F012C029F013C02AF0120027C007
:10EF50000CF028C00DF029C00EF02AC00FF01200EE
:10EF600000C027F001C028F002C029F003C02AF039
:10EF700012000A0E2B6E2C6A2D6A2E6A1200006E89
:10EF8000060EE15E00501200E126EEEF77F0DECFD4
:10EF900000F0DDCF01F0D8900132003212000B0EEC
:10EFA000006EE00E016E000E026E0F0E1200D9CF41
:10EFB000E6FF39D02C6A2D6A610E2E6E450E2F6E3B
:10EFC0001200D950FD0F4EEF78F0D9CFE6FFDACF1F
:10EFD000E6FF1200E552E552E5521200FD0EDBCFCE
:10EFE000E6FFFE0EDBCFE6FF1200D9CFE6FFE1CF52
:10EFF000D9FF1200D950F60F51D8EECFE6FFEECF71
:10F00000E6FFEECFE6FFEFCFE6FF1200FA0EDBCF12
:10F0100000F0FB0EDBCF01F0FC0EDBCF02F0005066
:10F02000011002101200E552E7CFD9FF1200FD0EC9
:10F03000DBCF00F0FE0EDBCF01F000C0F3FF01C01C
:10F04000F4FF1200FD0EF3CFDBFFFE0EF4CFDBFF6B
:10F050001200D9CFE9FFDACFEAFF120004C026F090
:10F0600005C027F006C028F007C029F01200A4DE72
:10F07000EF5012003CDFDF6A7C0ECA6ECC6ACB68B0
:10F080001200E66E99DEE552E750EF6E1200F80EC0
:10F09000DBCFE6FFF90EDBCFE6FF1200E96EFF0ED5
:10F0A000DA20EA6E1200FA0EDBCFE6FFFB0EDBCFB2
:10F0B000E6FFFC0EDBCFE6FFEEEF77F08FDF8FDCB5
:04F0C000EAEF77F00C
:0CF0C40045EC7DF0030EE126020EDB6A35
:10F0D000000E0901E76EE119E8AE02D0E13503D078
:10F0E000E750D880E15501E2E107000E0901E76E23
:10F0F000E219E8AE02D0E23503D0E750D880E255FD
:10F1000001E2E20709010A51000807E20A0703E1E8
:10F1100009019B9102D009019B810901A52B000ED9
:10F12000A623A723A8230901905157E009018E5176
:10F130008F1153E0090199B715D00C0E99130901ED
:10F14000966B0901976B0901010E946F0901030E7B
:10F15000956F0901100E916F0901926B936B090174
:10F16000986B5FD00901052B3C0E055D63E3056BD1
:10F170000901922B000E932309019051026E036A3C
:10F1800090C928F003C029F08EC92DF08FC92EF048
:10F19000B6EC84F026C000F027C001F00001265034
:10F1A000090106270001275009010723000E082343
:10F1B0000923600E065DEA0E0759000E0859000E7D
:10F1C000095938E30901982B600E0901065FEA0E20
:10F1D000075B000E085B095B2DD0090190512AE105
:10F1E00009018E518F1126E1090199A723D0F30E51
:10F1F00099170901966B0901976B5F0E0901A05DD4
:10F200000AE20901150E946F09010E0E956F040EA6
:10F2100034EC7DF006D00901040E946F0901030E51
:10F22000956F0901056B066B076B086B096B020E86
:10F2300034EC7DF009010F5119E0010EE66EBFECD0
:10F2400072F0E5520DEC2EF0100EE66E090EE66E31
:10F25000000EE66E060EE66E69EC98F0E552E55299
:10F26000E552E5523AEC2EF009010F6B045108E12A
:10F270000901905105E109018E518F1101E192D0F0
:10F280000501F45101E18ED0DE6ADD6A9ADB06BE2B
:10F29000076880EC7DF00050011001E181D06E0E16
:10F2A000046E510E056E010E066EDECF07F0DDCF47
:10F2B00008F0096A08BE0968050E2C6E2D6A2E6AD0
:10F2C00007C027F008C028F009C029F0D4EC84F06A
:10F2D00024C007F025C008F026C009F004502424FB
:10F2E000F36E05502520F46E065072EC7DF0020E90
:10F2F000E0DB0800F550026E036AC8C728F0C9C7F2
:10F3000029F02D6E03C02EF0CEECA8F024C000F042
:10F3100025C001F0245025103DE1020EDB5002E033
:10F32000B3EC72F00F0140B7FDD7406B4ADB06BE6D
:10F330000768E6DB070E0016000E0116050ED890D2
:10F3400000360136E804FBE100C042FF3ADB06BEAE
:10F350000768D6DB030ED89001320032E804FBE1E7
:10F3600000C041FF0F01030E466F220E476F29DBDD
:10F3700006BE0768B2DB01C000F0016A00C048FFAA
:10F3800020DB06BE0768A9DB005052DBF36E020EDD
:10F39000F3CFDBFFDF2A010E01E278D7DB2A76D735
:10F3A0000901046B000E006E030EE15C02E2E16AEB
:10F3B000E55238D36ADB080EE1266250026E036A1A
:10F3C000050ED89003320232E804FBE16150046E6E
:10F3D000056A030ED89004360536E804FBE10250B6
:10F3E0000424006E03500520016E060E00C0DBFFF2
:10F3F000070E01C0DBFF0F0E65140B01406F66CFD7
:10F4000041FB67CF42FB68CF43FB69CF44FB6ACF28
:10F4100045FB6BCF46FB6CCF47FB6DCF48FB609E37
:10F4200009013C0E0A6F43CB03F0026A0B01445101
:10F430000224006E000E032000C0DEFFDD6E020E0F
:10F4400045CBDBFFDECF00F0DDCF01F009010D5130
:10F45000001854E10E51011851E1060EDBCF02F005
:10F46000070EDBCF03F00B51021848E10C510318D3
:10F4700045E10F5143E1200EE66EE50EE66E000E0B
:10F48000E66E100EE66E090EE66ED8EC74F0006EB5
:10F49000050E1ADB2E0EE66EE66A1E0EE66EE50E11
:10F4A000E66E000E81DA060EDBCFE6FF070EDBCF3D
:10F4B000E6FF1A0EE66EE50EE66E000E75DADECF9A
:10F4C000E6FFDDCFE6FFFADA6FDA030EDB6A080E3D
:10F4D000F36E030EDBCFF4FFF350F45C08E2030E8F
:10F4E00098DAE66AEBDA60DA030EDB2AF0D7090174
:10F4F000010E0F6F0B6B0C6B0D6B0E6B620E0B0125
:10F50000425D02E0010EDED0D950060FE96EDACF7F
:10F51000EAFFEC0EEE1801E091D0070EED1801E0C5
:10F520008DD0000EDFCF28F0010EDBCF29F0340E96
:10F53000281802E1830E291859E0430E281802E129
:10F540001C0E29184FE04F0E281802E1430E29180F
:10F5500045E01E0E281802E1800E29183BE01F0E20
:10F56000281802E1800E291827E0680E281802E109
:10F57000430E291818E0690E281801E0A2D0430EA6
:10F58000291801E09ED0020EDB50006E016A050EC4
:10F590002D6E2E6A00C028F001C029F0CEECA8F034
:10F5A00028C090F98ED0020EDB5009018E6F8F6B50
:10F5B000D8908E378F3785D009013C0EE16F020E4F
:10F5C000DB50E8307F0B006E280E005E000E00C09E
:10F5D000ADF977D009013C0EE26F73D04CDA00C070
:10F5E000C2F96FD048DA00C0C0F96BD009013C0EF7
:10F5F000E26F020EDB50270DF3CF00F0F4CF01F0E5
:10F60000630E50DA2FEC84F028C000F029C001F01E
:10F6100028C0A0F909012850250DF3CFA1F9F4CF96
:10F62000A2F9640E3FDACEECA8F028C0A1F929C0F7
:10F63000A2F928C0A3F929C0A4F943D0D950060FD4
:10F64000E96EDACFEAFFE80EEE183BE1070EED189F
:10F6500038E1D9CFE9FFDACFEAFF0D0EEE1831E13C
:10F66000EE502FE14B0E0701CB5D04E1020EDBCF24
:10F670009FF927D0020EDBCF26F0276A286A296A75
:10F68000E80E2B6E030E2C6E2D6A2E6AF0ECA7F09E
:10F6900022C026F023C027F024C028F025C029F07E
:10F6A000F40E2626010E2722000E28222922490EBA
:10F6B0002B6E060E2C6E2D6A2E6A59ECA8F026C011
:10F6C0009FF9010E006E080EE15C02E2E16AE5526C
:10F6D000A9D1DBD9020EE1260F0E0F0155150B0142
:10F6E000406F56CF41FB57CF42FB58CF43FB59CF1A
:10F6F00044FB5ACF45FB5BCF46FB5CCF47FB5DCF5E
:10F7000048FB50CFDFFF0F01509F0901010E046F2E
:10F710003C0E0A6F070EDF14020850E0070EDF14DC
:10F7200003080EE1010EDB6AB5D907E2010E71D9BB
:10F73000010EDB50090F87D9F7D70901BF6B3ED007
:10F74000070EDF1404080DE10901310EAE6F010E42
:10F75000DB6AA0D933E2010E5CD9010EDB2873D934
:10F76000F8D7070EDF14050829E10B01415117E115
:10F770000901998D999F0901A951AA11AB11AC11E9
:10F780001DE1A5C9A9F9A6C9AAF9A7C9ABF9A8C9D4
:10F79000ACF9A907000EAA5BAB5BAC5B0DD009010D
:10F7A000999D998F0901A951AA11AB11AC1106E0DD
:10F7B000A96BAA6BAB6BAC6B010E56D9010E006E38
:10F7C000020EE15C02E2E16AE5522CD15ED9FC0E48
:10F7D000DBCF28F0FD0EDBCF29F02E0E28184CE1F0
:10F7E00029504AE16BD9E66E84D9F7D80CE036D9B6
:10F7F000F3CF0BF9F4CF0CF961D9E66E000EE66E8B
:10F80000E66AEBD802E1000E38D028D9F3CF0DF923
:10F81000F4CF0EF909010F6BB3EC72F00F0140B792
:10F82000FDD7406B070E09010B15006E016A050E2E
:10F83000D89000360136E804FBE100C042FF0BC956
:10F8400000F00CC901F0030ED89001320032E80438
:10F85000FBE100C041FF080E09010B27000E0C233D
:10F860000F01030E466F220E476F016A0EC948FF53
:10F8700009010D51DDD801D0000EE552E7CFD9FFC7
:10F880001200D9CFE6FF020EE1260501560EC86F21
:10F89000410EC96FCA6BCB6BCC6B0901DC0E006FDC
:10F8A000DA0E016FD40E026F340E036F046B056B1A
:10F8B000066B076B086B096B0A6B0B6B0C6B0D6BA4
:10F8C0000E6B0F6B0901E5690901A56BA66BA76BB0
:10F8D000A86B900E6F6E6EAEFED7606A0F01196B4B
:10F8E0001869016BFD0E006F506BE00E1D6F1C69F7
:10F8F000C00E096F400E086F200E0D6F9C0E0C6F2E
:10F90000800E116FA20E106FA00E156F260E146FD1
:10F91000010E706ED20E716E020E726E200E736E3C
:10F920000501F451000802E26F6A02D0600E6F6EAA
:10F930000701B40ED56FF30ED66F000ED76F070117
:10F94000D20ED86FF60ED96F000EDA6F0701C40E13
:10F95000DB6FF00EDC6F000EDD6F0B01CC0E496F1C
:10F96000F70E4A6F000E4B6F0601EE81EE83010E1B
:10F97000006E020EE15C02E2E16AE55253D0050E30
:10F980002C6E2D6A2E6A05C027F006C028F007C02D
:10F9900029F0D4EC84F002502424F36E0350252087
:10F9A000F46E045072EF7DF0E66E040EDBCFE6FFDE
:10F9B000050EDBCFE6FF07EC75F0006E070E64EF77
:10F9C0007DF06E0E026E510E036E010E046EDECFE0
:10F9D00005F0DDCF06F0076A12004AECA4F0006ED5
:10F9E000050EE15E0050FA0EF3CFDBFFFB0EF4CF05
:10F9F000DBFFD950FA0FE96EFF0EDA20EA6EEE5007
:10FA0000ED1012000900F5CF00F00800F5CF01F06D
:10FA10001200DB50EA6A410FE96E0B0EEA22EF504A
:10FA2000E66E1200E16E0050E552E7CFD9FF1200FA
:10FA30000F01496F4A6B4B6B4C6B4D6B080E456F5A
:10FA4000406F010E1200EA6AAE0FE96E090EEA225B
:10FA5000E552E750EF6E010EDB2A12004AD8DFECC8
:10FA600089F0E552E5521200E66EE66AFEEC3EF0E1
:10FA7000E552E552120009013C0EE26F020EDB5026
:10FA8000006E280E005E000E1200D9CFE6FFE1CF17
:10FA9000D9FF1200080EF36E010EDBCFF4FFF35016
:10FAA000F45C12002D6E2E6AF3CF28F0F4CF29F00B
:10FAB0001200F626000EF722F8221200180EE66E4B
:10FAC000E50EE66E000E1200E15E0050040EF3CF6C
:10FAD000DBFF050EF4CFDBFF120051DF030EE9DF81
:10FAE00002EF7DF02620F86EF4CFF7FFF3CFF6FF9C
:10FAF0001200FA0EDBCFE6FFFB0EDBCFE6FF1200B3
:06FB00003EDF02EF7DF084
:0AFB06000A0EE66E010EE66EF4EC46
:10FB100081F00A0EE66EE66AF4EC81F05AECA2F08F
:10FB20000601CE6BCF6B0601CD6B0901C60EFC6FD3
:10FB3000E10EFD6F000E39EC82F0F4C5E7F8080124
:10FB4000E869E9691200CCEC81F0030EE1260801B6
:10FB5000800EE91501E0A5D0E20E006E450E016EA3
:10FB6000010E026EEA0E066E450E076E010E086E5D
:10FB7000E8C809F0E9C80AF0090E0A02F3CF0AF052
:10FB80000902F3CF09F0F4500A260B6A0ABE0B688B
:10FB900006500924F36E07500A20F46E08500B201B
:10FBA00044EC82F00800F5CF03F0046A056AD890AF
:10FBB000033604360536BFDB0900F5CFDEFF0A0049
:10FBC000F5CFDDFF0F01406B04EC82F0070E00164D
:10FBD000000E0116050ED89000360136E804FBE150
:10FBE00000C042FF04EC82F0030ED89001320032D4
:10FBF000E804FBE100C041FF010EF36E020EF3CFFB
:10FC0000DBFF6DDB04BE056841EC82F0F5CF46FFFB
:10FC100066DB04BE056841EC82F0F5CF47FF5FDB91
:10FC200004BE056841EC82F0F5CF48FF58DB04BE06
:10FC3000056841EC82F0F5CF49FF51DB04BE056851
:10FC400041EC82F0F5CF4AFF4ADB04BE056841EC87
:10FC500082F0F5CF4BFF43DB04BE056841EC82F038
:10FC6000F5CF4CFF3CDB04BE056841EC82F0F5CFDC
:10FC70004DFF0F01080E456F4087010E0801E82572
:10FC8000E86F000EE921E96F110E2D6E2E6AE8C8AB
:10FC900028F0E9C829F02FEC84F024C0E8F825C04A
:10FCA000E9F8040E0601F115006E040EB2DB09E05E
:10FCB0000901AC0EFC6FE10EFD6F000EAFDBF1959C
:10FCC000F295100EF115006E100EA3DB09E009018C
:10FCD000930EFC6FE10EFD6F000EA0DBF199F2991F
:10FCE000200EF115006E200E94DB09E009017A0E5A
:10FCF000FC6FE10EFD6F000E91DBF19BF29B030E9A
:10FD0000E15C02E2E16AE552E16E4BD345DB020EB3
:10FD1000E126E66A83EC9FF0E552F3CFDEFFF4CFF5
:10FD2000DDFF43DB0FE0140EE66EE66ADECFE6FF92
:10FD3000DDCFE6FF76DB01EC99F0006E060EE15EAA
:10FD4000005008D0710EE66EE10EE66E6ADB69ECDB
:10FD500098F06CDBFADA31DBA3EC98F0E552E5526F
:10FD6000F350E66E2ADB5DDB27EC61F098DB020ED8
:10FD7000E15C02E2E16AE552E16E13D30DDBE5DA04
:10FD80001CDBB6EC34F0E552E5520A019E519F119E
:10FD900005E00A015E5102E189EC36F002D3FCDA9B
:10FDA000D4DA27DB450EFC6FE10EFD6F000E61DB40
:10FDB0000901310EFC6FE10EFD6F000E5ADB52DBC4
:10FDC00051DBA4DF33DB09011D0EFC6FE10EFD6F7B
:10FDD000000E4FDBE66A20EC32F0E552E2D2DCDACC
:10FDE000E66A010EE66E00DBE66AE66AFDDA5AECC8
:10FDF000A2F0ABDAFEDA000EFC6FE10EFD6F000E32
:10FE000038DB0A0E39DBA5EC72F0CBD2C5DA050E71
:10FE1000E126010EF36E020EF3CFDBFFF36EDB6E15
:10FE20000901F40EFC6FE00EFD6F000E22DB0E0EDA
:10FE3000F66E000EF76E000ED1DAE70EE66EE00EFB
:10FE4000E66E000E3EDB0F0EF66E000EF76E000E35
:10FE500030DB100EF66E000EF76E000E2ADB0E0E73
:10FE6000E66E83EC9FF0E552F3CF00F0F4CF01F0A3
:10FE7000F3CFE6FFF4CFE6FFA7DA01EC75F0026EF0
:10FE8000070EE15E0250DFDA0701CC51CD11CE1131
:10FE900008E0CCC7E6FFCDC7E6FFCEC7E6FF1FDB15
:10FEA00019DB020EDBCFE6FFE66AE00EE66EE00E3F
:10FEB000E66E000EC5DACEDA2EECA8F0E66EE66A43
:10FEC000D20EE66EE00EE66E000E60DAC3DA33ECB8
:10FED000A8F026C000F027C001F028C002F029C019
:10FEE00003F02C6A2D6A200E2E6E410E2F6E26C056
:10FEF00027F001C028F002C029F003C02AF0A8ECC6
:10FF000083F044EC85F028C0DEFF29C0DDFF010E40
:10FF1000E66EE66A79DA026A036A00C0E6FF01C0AB
:10FF2000E6FF02C0E6FF03C0E6FFC40EE66EE00E89
:10FF3000E66E000E2BDAF9EC75F0046E0B0EE15E46
:10FF4000045081DABF0EE66EE00EE66E000EE5D9D3
:10FF50000901E951E66EE66AB10EE66EE00EE66E64
:10FF6000000EAFDAAD0EE66EE00EE66E000ED5D9ED
:10FF7000AE0EE66E090EE66E9F0EE66EE00EE66EC3
:10FF8000000E04DA28DAC80EE66E050EE66E9C0E48
:10FF9000E66EE00EE66E000E53DA1DDA980EE66E9F
:10FFA000E00EE66E000EB9D90901A051E66EE66AD0
:10FFB0008A0EE66EE00EE66E000E83DAA1C9E6FF59
:10FFC000A2C9E6FF860EE66EE00EE66E000E92DA3D
:10FFD000A3C9E6FFA4C9E6FF7D0EE66EE00EE66E5D
:10FFE000000E88DA6F0EE66EE00EE66E000E95D912
:10FFF0000801800EE9150FE1E8C8E6FFE9C8E6FF51
:020000040001F9
:10000000630EE66EE00EE66E000E5BDA110EE66E33
:10001000E66ADAD91FDA0901610EFC6FE00EFD6FA6
:10002000000EC6D9570EFC6FE00EFD6F000EC0D952
:100030004D0EFC6FE00EFD6F000EBAD9450EFC6F41
:10004000E00EFD6F000E15DA050EE15C02E2E16ADA
:10005000E552E16EA6D1A0D9B0D9DFEC89F0E55226
:10006000E552F3CFE9F99DD197D9F4C5E7F8050139
:10007000010EF46F07EC93F00801E86BE96B0901DE
:10008000300EFC6FE00EFD6F000E30D285D9E7C850
:10009000F4F507EC93F00801E869E96909011C0E21
:1000A000FC6FE00EFD6F000E21D276D9040EE12622
:1000B00066D9EF5001E10CD162D9EF50230801E17C
:1000C00007D1FD0EDBCFDEFFDBCFDDFF6ED918E001
:1000D0006CD9200815E069D960080DE2E5D9EFCFA9
:1000E00000F07B0E005C07E260D9E00FE66EDCD921
:1000F000E552E750EF6EDF2A010EE8E3DB2AE6D790
:1001000054D9200804E1DF2A010E01E3DB2A020EA4
:10011000DB6A030EDB6A830E006E460E016E010E73
:10012000026E020EDBCF03F0030EDBCF04F0056A94
:1001300004BE056880D903C027F004C028F005C0BC
:1001400029F0D4EC84F024C003F025C004F026C0CC
:1001500005F000502424F36E01502520F46E025067
:10016000262092D90800F55001E1A0D0830E056E3B
:10017000460E066E010E076E020EDBCF08F0030E70
:10018000DBCF09F00A6A09BE0A6855D908C027F012
:1001900009C028F00AC029F0D4EC84F024C008F08B
:1001A00025C009F026C00AF005502424026E06502E
:1001B0002520036E07502620046E02C0E6FF03C010
:1001C000E6FFE66EB1EC98F0E552E552E55227C045
:1001D00000F028C001F027C0E6FF28C0E6FF830E2C
:1001E0000E6E460E0F6E010E106E020EDBCF11F07A
:1001F000030EDBCF12F0136A12BE13681CD911C0B4
:1002000027F012C028F013C029F0D4EC84F024C0E9
:1002100011F025C012F026C013F00E5024240B6EEE
:100220000F5025200C6E105026200D6E0BC0E6FFDF
:100230000CC0E6FFE66E16D991EC97F0146E070E2F
:10024000E15E145000092BE1020EDBCFE9FF030E43
:10025000DBCFEAFFEA02F3CFEAFFE902F3CFE9FFDF
:10026000F450EA26EA0EE926080EEA22EECF00F064
:10027000EECF01F0EFCF02F0DECFE6FFDDCFE6FFFD
:10028000FD0EDBCFE6FFFE0EDBCFE6FF06D002C0A1
:10029000FBFF01C0FAFF0050F96EF9DF18D0020E23
:1002A000DB2A030E01E237D7DB2A35D768D8EF50B7
:1002B000530805E1EFD803E150D828DD08D05FD816
:1002C000EF504D0805E1E6D803E147D857DDAED839
:1002D000040EE15C02E2E16AE552E16E62D0EA0EF0
:1002E000006E450E016E010E026E020EDBCFF3FFB3
:1002F000DB2AF350066E076A090E286E296AE8C8E1
:100300002DF0E9C82EF089EC84F026500624036E07
:1003100027500720046E056A120092D8DBD8000E21
:10032000E66E060EE66EA3EC3EF0E552E5521200D4
:1003300007EC75F0C9D000500324F36E015004207F
:10034000F46E0250052044EF82F009016E0EFC6F3E
:10035000E10EFD6F000E39EF82F0020EE76EFD0E2A
:10036000DBCF00F0FE0EDBCF01F0E7500026000EE1
:10037000012200C0E6FF01C0E6FF32EF82F0FD0E71
:10038000DBCFE9FFFE0EDBCFEAFF1200E66E000EC8
:10039000E66E060EE66E1200D9CFE6FFE1CFD9FF7A
:1003A0001200E552E7CFD9FF12007ED8EF501200BD
:1003B00060D8050E61D809011200FB0EDBCFE6FF05
:1003C000FC0EDBCFE6FF1200E30EE66EE00EE66EFB
:1003D000000E20EF82F001EC75F076D0F86E080088
:1003E000F550E66EE66A120033ECA2F0E552E552F3
:1003F0001200010E41D809011200E750E926000E53
:10040000EA22EF5020081200DECF00F0DDCF01F02D
:100410001200F215016E0050011012002AD80601D8
:100420001200D60EE66E060EE66E1200E552E5529A
:10043000E552E55212001B0E2C6E2D6A2E6A120038
:10044000E66E6FEF82F0030EF3CFDBFF040EF4CF06
:10045000DBFF12006DDF6E0EE66EE10EE66E000E43
:100460008DEF81F0FD0EDBCFE6FFFE0EDBCFE6FF6A
:100470001200FE6F54EF3EF0E66EBFEC72F0E552F4
:10048000120059DF08001200F86EF4CFF7FFF3CF27
:10049000F6FF1200010EE76E72DFFDEF81F0006ED5
:1004A000050EE15E00501200DECFE9FFDDCFEAFF6E
:1004B000120094DFE50EE66EE00EE66E000E7AEFB7
:1004C00082F064DF98EF81F0006E070EE15E00506D
:1004D00023EF82F0D8EC74F0E2DF23EF82F0030E1A
:1004E000DBCFE6FF040EDBCFE6FF1200C2DF020E19
:0A04F000C3DF57D7A5DF98EF81F0B6
:0604FA00219E05D0219EA9
:1005000029AE02D0296C218E29C023F0226A336AD9
:10051000326A860E246E256A24EF86F0219E08D06A
:10052000219E29AE05D0286C291EE86A2922218E39
:1005300029C023F028C022F0336A326A8E0E246E5E
:10054000256A24EF86F0219E0CD0219E29AE09D089
:10055000266C271E281E291EE86A27222822292207
:10056000218E29C023F028C022F027C033F026C0F6
:1005700032F09E0E246E256A24EF86F02F7E216ACB
:1005800060EC86F078EC86F021B608EF86F021A2C8
:100590000AD021AA03D021BE08EF86F021A414EFCF
:1005A00086F011EF86F021AA05D021AC14EF86F079
:1005B00011EF86F021A00AD021A808D021BE04D0D6
:1005C00021A402D01DEF86F021EF86F0326A256A61
:1005D0002F502A5C316E10E327C033F028C022F080
:1005E00029C023F02AC030F02CC027F02DC028F0FD
:1005F0002EC029F0213A09D02CC033F02DC022F0B2
:100600002EC023F02FC030F0316C219E21BC218EF2
:1006100030C024F021B050EF86F01A0E316050EF58
:1006200086F0246A2A6A21A408D0276C281E291E75
:100630002A1EE86A282229222A2221AC08D0336CFB
:10064000221E231E241EE86A222223222422266A36
:10065000315207E02A342932283227322632312E0D
:10066000F9D72750332628502222295023222A50F6
:10067000242226C032F0219E24AE0BD0326C331ED1
:10068000221E231E241EE86A332222222322242231
:10069000218E24A006D0D880233222323332323247
:1006A000302A30C024F024EF86F0216A60EC86F016
:1006B00078EC86F021B608EF86F021A205D021BAA9
:1006C00008EF86F00FEF86F021BA1BEF86F021A02D
:1006D00005D021B808EF86F01BEF86F021B80FEFA8
:1006E00086F0256A7F0E2A24246EE86A25222F5080
:1006F000245EE86A255A1A0E306E2A6A326A336A14
:10070000226A236A2C50275E2D50285A2E50295ACF
:10071000000E2A5A09E72C5027262D5028222E5049
:100720002922000E2A2201D0328AD8902736283674
:1007300029362A36D8903236333622362336302EB2
:10074000E1D7295028102710D8A4328A24EF86F048
:10075000216A60EC86F078EC86F021B608EF86F02E
:1007600021A205D021B808EF86F00FEF86F021AA6C
:1007700005D021B008EF86F00FEF86F021B002D04F
:1007800021A802D01BEF86F0256A2F502A24246E60
:10079000E86A25227E0E245EE86A255A326A336AA8
:1007A000226A236A2E502902F4CF23F0F3CF22F0DD
:1007B0002D502902F3503326F4502222000E23221A
:1007C0002E502802F3503326F4502222000E23220A
:1007D0002C502902F3503226F4503322000E2222EC
:1007E00023222D502802F3503226F4503322000EDB
:1007F000222223222E502702F3503226F450332295
:10080000000E222223222C502802F4503226000E01
:100810003322222223222D502702F4503226000EAA
:1008200033222222232224EF86F0206A2EAE1BEFF1
:1008300084F02E6C201E29AE20EF84F0296C201E3F
:1008400021ECA9F029BE2AEF84F020AE000C296C1F
:10085000256C000C20BE27EF84F02188FF0C206A55
:100860002EAE38EF84F02D6C2E1EE86A2E22201E4C
:1008700029AE40EF84F0286C291EE86A2922201E48
:10088000CEECA8F029BE50EF84F020AE000C286C0E
:10089000291EE86A2922246C251EE86A2522000CFC
:1008A00020BE47EF84F02188FF0C206AE86A2EAE54
:1008B00062EF84F02B6C2C1E2D1E2E1E2C222D225E
:1008C0002E22201E29AE6DEF84F0266C271E281ED6
:1008D000291E272228222922201E59ECA8F029BEF1
:1008E00084EF84F020AE000C266C271E281E291EE3
:1008F000E86A272228222922226C231E241E251E74
:10090000232224222522000C20BE74EF84F02188AB
:10091000FF0C29C033F028C032F028502D02F4CF4C
:1009200027F0F3CF26F029502E02F4CF29F0F3CF91
:1009300028F02D02F3502726F4502822E86A2922B5
:1009400032502E02F3502726F4502822E86A29223A
:100950002EAEAFEF84F03250285E3350295A33AEBA
:10096000000C2D50285E2E50295A000C28C032F061
:1009700028502D02F4CF27F0F3CF26F029502E0275
:10098000F4CF29F0F3CF28F02D02F3502726F450AE
:100990002822E86A292232502E02F3502726F450EA
:1009A0002822E86A2922000C29C033F028C032F03E
:1009B00027C031F027502C02F4CF25F0F3CF24F0DC
:1009C00028502D02F4CF27F0F3CF26F02C02F3505D
:1009D0002526F4502622E86A272231502D02F350B2
:1009E0002526F4502622E86A272229502C02F350AB
:1009F0002626F450272229502D02286AE86A282248
:100A0000F3502726F450282231502E02F350262688
:100A1000F4502722296AE86A2822292232502E021D
:100A2000F3502726F4502822E86A292233502E0258
:100A3000F3502826F4502922000C216A60EC86F03D
:100A400021B627EF85F021A20AD021B403D07F0E72
:100A5000296E19D0800E296E16D0296A14D021B0C3
:100A6000FCD7870E2A60F1D77E0E2A64F6D7860E51
:100A70002A5C04E0D89029322A2AF9D721A403D08D
:100A8000296C29AEEAD71200216A60EC86F021B603
:100A90004EEF85F021A20ED021B405D07F0E296E35
:100AA000FF0E286E1FD0800E296E286A1BD0296A7F
:100AB000286A18D021B0FBD78F0E2A60EDD77E0EA2
:100AC0002A64F5D78E0E2A5C05E0D89029322832A8
:100AD0002A2AF8D721A406D0286C291EE86A2922E0
:100AE00029AEE5D71200216A60EC86F021B67DEFD1
:100AF00085F021A20FD021B407D07F0E296EFF0E02
:100B0000286E276E266E25D0800E296E01D0296AA8
:100B1000000EF6D721B0FBD7266A9F0E2A60EBD7CE
:100B20007E0E2A64F4D79E0E2A5C07E0D890293204
:100B30002832273226322A2AF6D721A40AD0266C58
:100B4000271E281E291EE86A27222822292229AECC
:100B5000DED71200B3EC85F021B6000C21B0000CFA
:100B600021A4000C010C216A60EC86F078EC86F080
:100B700021B6120021AE08D021A004D021A802D0B5
:100B800021801200219012002F502A5C0BE12E5080
:100B9000295C08E12D50285C05E12C50275C02E11E
:100BA00021801200D8A002D0218E10D02A502FC050
:100BB0002AF02F6E29502EC029F02E6E28502DC0FD
:100BC00028F02D6E27502CC027F02C6E2F502A5C59
:100BD00010E0FF0F09E0219021B403D021AE218461
:100BE000120021AE219412002F2AD8902E322D32DD
:100BF0002C322C50275E2D50285A2E50295A29BEAF
:100C0000EAD7D8902736283629362A2EF8D7C8D7DB
:100C10007F0E2A6EFF0E296E286E276E12007F0E41
:100C200021BEFF0E2A6E02D07F0E2A6E800E296E24
:100C3000286A276AF3D721AE04D0800E2A6E296A6B
:100C4000F7D72A6A296AF4D72350221033103210BA
:100C5000F8E025BEF0D723BE0CD024502510EBE0E1
:100C6000D89032363336223623362406D8A02506CD
:100C7000F2D72550D4E12428D2E032AE11D07F0E35
:100C8000321402E133A00CD0332AE86A2222232254
:100C900007E3D880233222323332242A2428BFE0CB
:100CA0002450C9E033C027F022C028F02334296E35
:100CB00024302A6E29322A9E21BE2A8E0EEF86F01B
:100CC00029362A3602E32184217E06E121802A6A20
:100CD000296A286A276A12002A2803E0D880293264
:100CE0001200D890293202E12182120021861200DE
:100CF0002E362F3602E3218C217E06E121882F6AD1
:100D00002E6A2D6A2C6A12002F2803E0D8802E321A
:0C0D10001200D8902E32EAE1218A120075
:040D1C0011DB030ED6
:100D2000E126020EDB6A000E0901E76EE119E8AE6A
:100D300002D0E13503D0E750D880E15501E2E10768
:100D4000000E0901E76EE219E8AE02D0E23503D0E9
:100D5000E750D880E25501E2E2070901015100089D
:100D600007E2010703E109019B9102D009019B8180
:100D70000901A52B000EA623A723A82309010351CF
:100D800019E0010EE66EBFEC72F0E5520DEC2EF0AC
:100D9000040EE66E090EE66E000EE66E060EE66EB8
:100DA00069EC98F0E552E552E552E5523AEC2EF046
:100DB0000901036B005171E00501F4516EE0DE6A38
:100DC000DD6A8BDA04BE0568C0DA24C003F0D5DA28
:100DD000ABDA61E05E0E046E520E056E010E066E19
:100DE000DECF07F0DDCF08F0096A08BE0968E2DA55
:100DF00007C027F008C028F009C029F0D4EC84F01F
:100E000024C007F025C008F026C009F004502424AF
:100E1000F36E05502520F46E065086DA026E036AE2
:100E2000C8C728F0C9C729F02D6E03C02EF0CEEC3C
:100E3000A8F024C000F025C001F02450251026E1C0
:100E4000020EDB5002E0B3EC72F00F0140B7FDD7A9
:100E50006FDA43DA04BE056827DAF62A000EF722B5
:100E6000F8220800F5CF47FF38DA04BE05681CDA1F
:100E7000020EF626000EF722F8220800F5CF48FFF2
:100E80000F0148DAF36E020EF3CFDBFFDF2A010E0B
:100E900098E3DB2A96D70901006B000E006E030E63
:100EA000E15C02E2E16AE55229D24ADA0A0EE12661
:100EB0006250026E036A050ED89003320232E804D3
:100EC000FBE16150046E056A030ED89004360536C6
:100ED000E804FBE102500424006E03500520016E7B
:100EE000080E00C0DBFF090E01C0DBFF0F0E65140A
:100EF0000B01406F66CF41FB67CF42FB68CF43FBDE
:100F000069CF44FB6ACF45FB6BCF46FB6CCF47FBF9
:100F10006DCF48FB609E0901010E006F3C0E016F12
:100F20000B014351DE6EDD6A030E44CBDBFF4451FF
:100F3000026E036A080E452544CB00F003C001F0A1
:100F4000000A05E0D89000360136E804FBE1040E03
:100F500000C0DBFF050E01C0DBFF09010251006E7E
:100F6000016A0050DF184DE10150DE52DD1849E101
:100F7000035147E1430EE66EE50EE66E000EE66EA7
:100F8000040EE66E090EE66ED8EC74F0006E050EE7
:100F9000EBD92D0EE66EE66A410EE66EE50EE66EC4
:100FA000000E75D9080EDBCFE6FF090EDBCFE6FF9A
:100FB0003D0EE66EE50EE66E000E69D9DECFE6FF69
:100FC000DDCFE6FFCBD963D9020EDB6A080EF36EE4
:100FD000020EDBCFF4FFF350F45C0FE2020EDB50A5
:100FE000EA6A410FE96E0B0EEA22EF50E66EE66AFE
:100FF000B5D94DD9020EDB2AE9D70901010E036FDD
:10100000026B400E0B01425D03E342514A0802E2CB
:10101000010EA9D0410E425D01E0A4D0000EDFCF49
:1010200028F0010EDBCF29F00C0E281801E1295021
:1010300066E02F0E281801E129505BE00D0E2818FC
:1010400001E1295029E0460E281801E129501DE050
:101050005C0E281801E1295014E00F0E281801E158
:1010600029500BE0050E281801E07CD0295001E042
:1010700079D03FD900C0C2F975D03BD900C0C0F9C2
:1010800071D037D900C0C1F96DD009013C0EE16FB4
:101090007CD900C0ADF966D04B0E0701CB5D04E1F1
:1010A000030EDBCF9FF95ED0030EDBCF26F0276A5D
:1010B000286A296AE80E2B6E7DD9F0ECA7F022C0D1
:1010C00026F023C027F024C028F025C029F0F40E14
:1010D0002626010E2722000E28222922490E2B6ED9
:1010E000060E2C6E2D6A2E6A59ECA8F026C09FF9C8
:1010F00039D0030EDB50640DF4CFA0F933D0D950B2
:10110000040FE96EDACFEAFFEE50ED1017E10901A6
:10111000998D999F0901A951AA11AB11AC1122E136
:10112000A5C9A9F9A6C9AAF9A7C9ABF9A8C9ACF973
:10113000A907000EAA5BAB5BAC5B0DD00901999DC2
:10114000998F0901A951AA11AB11AC110BE0A96B40
:10115000AA6BAB6BAC6B010EE66EE66AFEEC3EF082
:10116000E552E552010E006E0A0EE15C02E2E16A10
:10117000E552C4D0E5D8020EE126FC0EDBCF28F004
:10118000FD0EDBCF29F02D0E281826E1295024E191
:10119000E5D8E66E01D98CD80CE0B6D8F3CFDEFFE7
:1011A000F4CFDDFFDBD8E66E000EE66EE66A80D88F
:1011B00002E1000E12D0A8D8F3CF02F90901036BA7
:1011C000B3EC72F00F0140B7FDD7B2D8DFCF47FFC5
:1011D00002C948FF9FD801D0000E006E020EE15CEC
:1011E00002E2E16AE5528AD0D9CFE6FF020EE1269B
:1011F00005014F0EC86F320EC96FCA6BCB6BCC6B3B
:101200000901006B016B026B036B0901E5690901C0
:10121000A56BA66BA76BA86B900E6F6E6EAEFED71C
:10122000606A0F01196B1869016BFD0E006F010EEA
:10123000706ED20E716E020E726E200E736E05010C
:10124000F451000802E26F6A02D0600E6F6E07016F
:10125000AA0ED56F0E0ED66F010ED76F07011C0EAA
:10126000DB6F0D0EDC6F010EDD6F0B01740E496F2D
:10127000110E4A6F010E4B6F0601EE81EE83010ED7
:10128000006E020EE15C02E2E16AE55237D0E66EE2
:10129000060EDBCFE6FF070EDBCFE6FF07EC75F0AF
:1012A000006E070EB4EF89F050D867D8D3EF89F0FD
:1012B0004AECA4F0006E050EE15E0050FA0EF3CF8A
:1012C000DBFFFB0EF4CFDBFFD950FA0FE96EFF0E08
:1012D000DA20EA6EEE50ED1012005E0E006E520E35
:1012E000016E010E026EDECF03F0DDCF04F0056A61
:1012F000120009013C0EE26FC5EF89F0E16E00506B
:10130000E552E7CFD9FF120047D8DFEC89F0E5526C
:10131000E5521200496B4A6B4B6B4C6B4D6B080EE0
:10132000456F406F010E12003ED80800F5501200C4
:10133000406BE00E426FFB0E416F020E466F1200D3
:10134000D9CFE6FFE1CFD9FF120034D803C027F090
:1013500004C028F005C029F0D4EF84F03B0EE66EFF
:10136000E50EE66E000E1200E15E0050060EF3CFB1
:10137000DBFF070EF4CFDBFF120000502424F36ED6
:1013800001502520F46E02501200030EDB50006E57
:10139000280E005E000E1200FA0EDBCFE6FFFB0EF9
:1013A000DBCFE6FF12002620F86EF4CFF7FFF3CF75
:0E13B000F6FF1200030E2C6E2D6A2E6A12003C
:0213BE00FF0E20
:1013C000E3CFEAFFE552FF0EE3CFE9FFE552E66A1D
:1013D000E66AD9CFE6FFDACFE6FFFC0EE124D96E4C
:1013E000FF0EE220DA6EE66AE66AE66A200EEF5C3D
:1013F00006E0090EEF5C03E0EF6603D03FD0EE504D
:10140000F5D72D0EEF5C03E1FF0EE32A03D02B0E80
:10141000EF5C01E1EE502F0EEF6424D03A0EEF6046
:1014200021D0D890F90EE336FA0EE336FD0EDECF6A
:10143000E3FFFE0EDDCFE3FFD890F90EE336FA0EA0
:10144000E336D890F90EE336FA0EE336FD0EE3509C
:10145000DE26FE0EE350DD22300EEE5CDE26000EB0
:10146000DD22D9D7FF0EE3CFE8FFE85207E0F90EFF
:10147000E31EE32AFA0ED8B4E306E31EE552E55272
:10148000E552FF0EE3CFDAFFE552FF0EE3CFD9FFBF
:10149000E552E1CFE9FFE2CFEAFFED52ED52EECFA8
:1014A000F3FFEFCFF4FF1200FF0EE3CFEAFFE552A8
:1014B000FF0EE3CFE9FFE552E66AE66AE66AE66A0E
:1014C000D9CFE6FFDACFE6FFFA0EE124D96EFF0EA0
:1014D000E220DA6EE66AE66AE66AE66AE66A200E04
:1014E000EF5C06E0090EEF5C03E0EF6603D06BD023
:1014F000EE50F5D72D0EEF5C03E1FF0EE32A03D08B
:101500002B0EEF5C01E1EE502F0EEF6444D03A0E4B
:10151000EF6041D0D890F50EE336F60EE336F70EC5
:10152000E336F80EE336FB0EDECFE3FFFC0EDECF34
:10153000E3FFFD0EDECFE3FFFE0EDDCFE3FFDD5266
:10154000DD52D890F50EE336F60EE336F70EE336AD
:10155000F80EE336D890F50EE336F60EE336F70EC6
:10156000E336F80EE336FB0EE350DE26FC0EE350C6
:10157000DE22FD0EE350DE22FE0EE350DD22DD52C0
:10158000DD52300EEE5CDE26000EDE22DE22DD2293
:10159000DD52DD52B9D7FF0EE3CFE8FFE85213E08A
:1015A000F50EE31EF60EE31EF70EE31EF80EE31E25
:1015B000F50EE32A08E1F60EE32A05E1F70EE32A29
:1015C00002E1F80EE32AE552E552E552E552E55212
:1015D000D9CFE9FFDACFEAFFEECF26F0EECF27F042
:1015E000EECF28F0EFCF29F0FF0EE3CFDAFFE55280
:1015F000FF0EE3CFD9FFE552E552E5521200D9CFF5
:10160000E6FFDACFE6FFFA0EE3CFD9FFFB0EE3CF1A
:10161000DAFFFD0EE35209E72D0EDE6EFC0EE31E2F
:10162000E32AFD0ED8B4E306E31EE652E652E65284
:10163000FD0EE124E76EFF0EE220E46EE652F70EA7
:10164000E3CFE6FFF70EE3CFE6FF6FEC8BF0F90E8A
:10165000E124E96EFF0EE220EA6E5FEC8BF00AE116
:101660005CEC8BF009E15FEC8BF008E15CEC8BF05B
:1016700007E108D06AEC8BF065EC8BF06AEC8BF03C
:1016800065EC8BF06AEC8BF0DE6AF90EE126FF0E5A
:10169000E222FF0EE3CFDAFFE552FF0EE3CFD9FFE0
:1016A000E552FC0EE124E96EFF0EE220EA6EEECF79
:1016B000F3FFEFCFF4FF1200EF380F0B1200EF50E3
:1016C0000F0B02E1EE52D8841200EF380F0B300FEF
:1016D000DE6E1200EE500F0B300FDE6E1200FC0EAD
:1016E000E3CFE9FFFD0EE3CFEAFF100EE66EEE6AF0
:1016F000EE6AEF6AD890FD0EE336FE0EE336ED3665
:10170000ED36EF36FF0EE30609E090EC8BF0EE527B
:1017100090EC8BF0EE5290EC8BF0EDD7E56E120072
:10172000030EEF24E8B6EF6E300EEF24E8BEEF6E46
:10173000000CD9CFE6FFDACFE6FFF80EE3CFD9FFF2
:10174000F90EE3CFDAFFFD0EE35215E72D0EDE6E44
:10175000FA0EE31EFB0EE31EFC0EE31EFD0EE31E5F
:10176000FA0EE32A08E1FB0EE32A05E1FC0EE32A68
:1017700002E1FD0EE32AE652E652E652E652E65256
:10178000FB0EE124E76EFF0EE220E46EE652F30E5C
:10179000E3CFE6FFF30EE3CFE6FFF30EE3CFE6FF82
:1017A000F30EE3CFE6FF36EC8CF0F50EE124E96EA4
:1017B000FF0EE220EA6E23EC8CF019E126EC8CF0AF
:1017C00018E123EC8CF017E126EC8CF016E123EC09
:1017D0008CF015E126EC8CF014E123EC8CF013E195
:1017E00026EC8CF012E123EC8CF011E112D02CEC01
:1017F0008CF031EC8CF02CEC8CF031EC8CF02CEC8F
:101800008CF031EC8CF02CEC8CF031EC8CF02CEC7E
:101810008CF031EC8CF0DE6AF50EE126FF0EE22250
:10182000FF0EE3CFDAFFE552FF0EE3CFD9FFE5521B
:10183000FA0EE124E96EFF0EE220EA6EEECFF3FF2E
:10184000EFCFF4FF1200EF380F0B1200EF500F0B29
:1018500002E1EE52D8841200EF380F0B300FDE6E2B
:101860001200EE500F0B300FDE6E1200FA0EE3CFB7
:10187000E9FFFB0EE3CFEAFF200EE66EEE6AEE6AAA
:10188000EE6AEE6AEF6AD890FB0EE336FC0EE336A2
:10189000FD0EE336FE0EE336ED36ED36ED36ED3673
:1018A000EF36FF0EE3060FE065EC8CF0EE5265ECD0
:1018B0008CF0EE5265EC8CF0EE5265EC8CF0EE5252
:1018C00065EC8CF0E1D7E56E1200030EEF24E8B66C
:1018D000EF6E300EEF24E8BEEF6E000CFE0EE3CF8D
:1018E000FEF4FF0EE3CFFFF41200FFC429F0FEC4A4
:1018F00028F0350E2D6E450E2E6EB6EC84F0262A9D
:10190000E86A2722279E27C0FFF426C0FEF4FEC403
:10191000F3FFFFC4F4FF1200D9CFE6FFDACFE6FFF2
:10192000F80EE3CFD9FFF90EE3CFDAFFE652E65225
:10193000E652E652E652FB0EE124E76EFF0EE2208D
:10194000E46EE652F30EE3CFE6FFF30EE3CFE6FFDD
:10195000F30EE3CFE6FFF30EE3CFE6FF36EC8CF0B9
:10196000F50EE124E96EFF0EE220EA6EFEEC8CF04B
:1019700019E101EC8DF018E1FEEC8CF017E101ECBF
:101980008DF016E1FEEC8CF015E101EC8DF014E128
:10199000FEEC8CF013E101EC8DF012E1FEEC8CF02A
:1019A00011E112D007EC8DF00CEC8DF007EC8DF00E
:1019B0000CEC8DF007EC8DF00CEC8DF007EC8DF05D
:1019C0000CEC8DF007EC8DF00CEC8DF0DE6AF50E72
:1019D000E126FF0EE222FF0EE3CFDAFFE552FF0E13
:1019E000E3CFD9FFE552FA0EE124E96EFF0EE220C3
:1019F000EA6EEECFF3FFEFCFF4FF1200EF380F0BDC
:101A00001200EF500F0B02E1EE52D8841200EF38B3
:101A10000F0B300FDE6E1200EE500F0B300FDE6E2C
:021A20001200B2
:0E1A22000ADB030EE126020EDB6A000E09014C
:101A3000E76EE119E8AE02D0E13503D0E750D88077
:101A4000E15501E2E107000E0901E76EE219E8AE97
:101A500002D0E23503D0E750D880E25501E2E20738
:101A600009010051000807E2000703E109019B9109
:101A700002D009019B810901A52B000EA623A723F3
:101A8000A8230901905141E009018E518F113DE0D9
:101A9000090199A73AD00901012B3C0E015D35E3FC
:101AA000016B0901922B000E932309019051026EE4
:101AB000036A90C928F003C029F08EC92DF08FC9A0
:101AC0002EF0B6EC84F026C000F027C001F0000133
:101AD0002650090102270001275009010323000EA7
:101AE00004230523600E025DEA0E0359000E04591B
:101AF000000E05590AE30901982B600E0901025FE7
:101B0000EA0E035B000E045B055B0901065101E16F
:101B10009AD00501F45101E196D0DE6ADD6A64DAFB
:101B200006BE07689FDA0050011001E18AD0080E56
:101B3000046E520E056E010E066EDECF07F0DDCF8D
:101B400008F0096A08BE0968050E2C6E2D6A2E6A17
:101B500007C027F008C028F009C029F0D4EC84F0B1
:101B600024C007F025C008F026C009F00450242442
:101B7000F36E05502520F46E06506DDA020E61DA20
:101B80000800F550026E036AC8C728F0C9C729F0DB
:101B90002D6E03C02EF0CEECA8F024C000F025C0BE
:101BA00001F02450251047E1020EDB5002E0B3ECB7
